:020000040000FA
:040000006FD00400B9
:101000006F1000140000000000000000902000207D
:10101000B2270020A9BDF9F56828002000000000D3
:101020000000000068280020902000200000000040
:101030000000000090200020000000009020002010
:101040000000000090200020902000209020002030
:101050009020002090200020B4300020902000201C
:10106000000000009020002090200020F4280020A4
:1010700090200020CE2800209020002090200020EA
:101080009020002090200020902000209020002020
:101090009020002001A04111B7170040985F3AC688
:1010A000945F3247E39CE6FE324541018280411164
:1010B000814601468145114506C6EF009014B727C9
:1010C000004011472383E780B7F700E003A707D16B
:1010D0006D9B23A8E7D003A707D15D9B23A8E7D08A
:1010E0007300501001000100B240410182800111E3
:1010F000814601468145114506CEEF009010B72785
:10110000004011472383E780B717004083C6E702FA
:1011100003C5E7041307800893F6C60F136535006F
:1011200093E61600733607801376860832C00100F6
:101130000100930570052380B704130680FA23800D
:10114000C70401000100238207022380070402482C
:10115000732808800100010073380780137888081D
:1011600042C2010001002380B7042380C7040100AC
:1011700001002387D7022387A70423800704924610
:10118000F3A6068001000100F336078093F6860877
:1011900036C4010001002380B7042380C704010086
:1011A000010083C6B70493E60602A385D704238013
:1011B0000704A246F3A6068001000100B7F600E08E
:1011C00003A506D11365450023A8A6D003A506D123
:1011D0005D9923A8A6D07300501001000100733759
:1011E0000780137787083AC6010001002380B704FF
:1011F0002380C7040100010003C7B7041377F70D6C
:10120000A385E70423800704B247F3A70780010002
:101210000100F240056182803971B7F5070022DCD8
:1012200081462A843010E105194506DE02D42316D2
:101230000102EF00007DB717004083C6E7041307E3
:10124000800893E63600733607801376860832C42A
:1012500001000100930570052380B704130680FA8E
:101260002380C704010001002382070223800704B2
:101270002245732505800100010073350780137531
:1012800085082AC6010001002380B7042380C70413
:10129000010001002387D70423800704B246F3A688
:1012A000068001000100F336078093F6860836C8F1
:1012B000010001002380B7042380C704010001005E
:1012C00003D50702F176FD16E98E2390D70223801D
:1012D0000704C246F3A606800100010037F500E0CE
:1012E000832605D193E646002328D5D083D607026E
:1012F0006575110593F60660C18EC98EC206C1825E
:1013000073350780137585082ACA01000100238000
:10131000B7042380C7040100010003C5F70013656B
:101320000504A387A7002390D70223800704D24691
:10133000F3A60680010001001165618D1DE9733778
:101340000780137787083ACC010001002380B70497
:101350002380C7040100010003C7B7041367070215
:10136000A385E70423800704E247F3A70780010071
:10137000010037F700E0832707D1DD9B2328F7D052
:10138000730050100100010013078008F337078035
:1013900093F787083ECE01000100B7170040930580
:1013A00070052380B704130680FA2380C704010068
:1013B000010083D60702C606C5822390D702238088
:1013C0000704F246F3A6068001000100F336078009
:1013D00093F6860836D0010001002380B7042380ED
:1013E000C7040100010003D80702F176FD16B3F629
:1013F00006012390D702238007048256F3A60680B5
:10140000010001000DED73370780137787083AD28A
:10141000010001002380B7042380C70401000100FC
:1014200003C7B7041377F70DA385E70423800704E8
:101430009257F3A70780010001005145ED2EF250AD
:10144000625421618280397152D481462A8A0146D0
:101450008145114522DC26DA06DE4AD84ED63714FD
:10146000004045238347E4020347E40493048008D3
:1014700093F7C70F1367370093E71700F3B604809D
:1014800093F6860836C60100010093097005230013
:101490003405130980FA230024050100010023020A
:1014A000040223000404B246F3A6068001000100F2
:1014B000F3B6048093F6860836C8010001002300C5
:1014C000340523002405010001002307F40223074B
:1014D000E40423000404C247F3A7078001000100CD
:1014E00013055002E128B7F700E003A707D11367FF
:1014F000470023A8E7D073B70480137787083ACA58
:10150000010001002300340523002405010001002F
:101510000347F40013670704A307E400230004044F
:101520005247732707800100010073B704801377C7
:1015300087083ACC0100010023003405230024056C
:10154000010001002167336AEA00231044032300ED
:1015500004046247732707800100010003A707D135
:101560005D9B23A8E7D07300501001000100814665
:101570000146814511457121F3B4048093F4840838
:1015800026CE0100010023003405230024050100BC
:1015900001008347640493E717002303F404230046
:1015A0000404F247F3A7078001000100F2506254DF
:1015B000D2544259B259225A216182800111130733
:1015C0008008F337078093F787083EC201000100C7
:1015D000B7170040930570052380B704130680FAFF
:1015E0002380C7040100010083C6B70493F6F60DFB
:1015F000A385D704238007049246F3A60680010042
:10160000010093760502D5CEF336078093F686085F
:1016100036C4010001002380B7042380C704010001
:101620000100B70614007D89558D88C701000100AF
:101630000100010023800704A246F3A606800100F2
:10164000010073370780137787083AC6010001004D
:101650002380B7042380C7040100010001000100BA
:101660003727004093061005A303D7802380070483
:10167000B247F3A707800100010093078008F3B782
:10168000078093F787083ECE01000100B71700409E
:10169000130770052380E704130780FA2380E7040B
:1016A0000100010003C7B70413670708A385E70417
:1016B00023800704F247F3A70780010001000561BA
:1016C000828093760504BDC6F336078093F68608BC
:1016D00036C8010001002380B7042380C70401003D
:1016E0000100B7061400938606047D89558D88C7CE
:1016F000010001000100010023800704C246F3A697
:1017000006800100010073370780137787083ACA03
:10171000010001002380B7042380C70401000100F9
:101720003727004093062005A303D78023800704B2
:10173000D24781B773370780137787083ACC010007
:1017400001002380B7042380C704010001009847EB
:101750001367070C98C723800704E24719BF0111DC
:10176000814601468145114506CE612C93078008CC
:10177000F3B7078093F787083EC601000100B7174B
:101780000040130770052380E704130780FA2380C5
:10179000E7040100010003C76704136717002383F0
:1017A000E70423800704B247F3A707800100010084
:1017B000F240056182804111814601468145114513
:1017C000892413078008F337078093F787083EC4FE
:1017D00001000100B7170040130670052380C704FD
:1017E000930680FA2380D70401000100FD5523965B
:1017F000B70223800704A245F3A50580010001007C
:1018000073370780137787083AC6010001002380E9
:10181000C7042380D7040100010003C767041367CE
:1018200017002383E70423800704B247F3A7078048
:101830000100010001A0BD473305F50201007D153F
:1018400075FD8280411122C426C206C6AA840144C5
:1018500063179400B24022449244410182800504FF
:101860001305803E4204C13F4180DDB7930500026D
:1018700073A0458082457390153492402242B24253
:101880004243D2436244F244025592552256B25624
:101890004257D2576258F25806499649264AB64AE4
:1018A000464BD64B664CF64C065D965D265EB65EA4
:1018B000465FD65F0961730020304111B7170040C1
:1018C000985F3AC6945F3247E39CE6FE3245410199
:1018D0008280B7170040130700032388E70285477B
:1018E00023A2F18673002030411122C406C63704BA
:1018F00000201C408297F5BF3737004083474700E0
:101900009146BD8B6389D70099466394D70083477E
:1019100057407300203083C6118993871600A3882F
:10192000F18803478700973700009387E73BB69716
:101930002380E700B7E70400BC4F0946894503C58B
:1019400061828297F9B72303048015472303E4805B
:1019500001002302A480828083076480E3CE07FE17
:1019600023030480828083076480E3CE07FE03455F
:101970004480828083076480E3CE07FE2302A48034
:101980008280411126C44AC24EC006C61377F50BA9
:10199000AD47AA892E8995446306F7001945653736
:1019A000653F8D444E854537FD59FD1463983401DC
:1019B000B240A24412498249410182801355090173
:1019C0001375F50F453F2209CDB7011126CC06CE80
:1019D000B704080051371545BD37713769372AC636
:1019E000A53F32459377150089EB136515001375F4
:1019F000F50FF240E24405618280FD14E9FC0145E7
:101A0000CDBF397126DC4ADA4ED852D656D45AD2D6
:101A10005ED006DE62CE66CCB7E700E07D5783AAD3
:101A2000070022C603AA470023A0E71823A2E7184D
:101A3000B7170040130770052380E704130780FAE7
:101A40002380E70483C74704930B75FFB684E2073E
:101A500093FBFB0F8546AA892E8B328937240040E1
:101A6000E187015763FA76016308D50089461307B9
:101A700000026313D5000157D98F93F7F70FB71CF6
:101A800000402382FC0411472303E4801305F00F78
:101A90005D3D094CD135636D7C11B7050700DA95C2
:101AA00037870700795563F2E504B3879500636EC5
:101AB000F702370B0800A94733EB65016399F90674
:101AC00089E48144513D26850DA0DA850945553DBF
:101AD00005090345F9FFFD14050B693D81C49377A2
:101AE000FB0FFDF7DD3569FD7D55B7170040130786
:101AF00070052380E704130780FA2380E70403C7F7
:101B00004704418B2382E704F250B7E700E023A0AB
:101B1000571123A24711E25432445259C259325A42
:101B2000A25A125B825B724CE24C21618280A54713
:101B30006395F90685691309F00FB3069900B3742C
:101B40002B01B6941349F9FFB3749900856B33796F
:101B50006901416B9387F9FFB3F7270199E363FCB0
:101B6000340193D94900C147E3E637FF99BF0569BE
:101B7000C1697D19D9B71305800D63886901130503
:101B800000026384790113051008CA85DD3B353DE9
:101B900021DD4E99B3843441D9B7DA852D45D5334B
:101BA000CA94E30099F205097D3BA30FA9FED5BFB6
:101BB0009387F9FF93F7F70F6361FC0C83C71C044D
:101BC00013073008631FF70437070800636BEB0443
:101BD000B3079B00B706100063F5D704334BEB0047
:101BE00089476393F9068980D549E38C04ECDA854B
:101BF0000945413B11090327C9FF91472320E48090
:101C000003076480E34E07FE23033481FD17EDFBD9
:101C1000FD14110B81C49377FB0FE9FF7D3371F540
:101C2000E1B5B717004003C75704B707080013779B
:101C3000070219E3B78707007955E378FBEA330712
:101C40009B00E3FFE7F855B58547E382F9F2DA85B3
:101C50002D45053B9389F4FFE38504E6293393F78B
:101C6000390091EB8326048003270900930749007C
:101C7000E39AE6E43E89CE84F1BFB5476396F90066
:101C80001305900BC93135BDB1471305B00AE38B7D
:101C9000F9FE99476391F904B7050800B365BB00E5
:101CA0002D45C53181448D4BA14975396396740129
:101CB000832704802320F9008504E39834FF8327D9
:101CC000048013172B01635507002312F900D5BBBD
:101CD0002322F900FDB39D476399F902814513055D
:101CE000B0044531BD442320090023220900FD59D9
:101CF0009D3993F77400CA9703C70700FD14398D07
:101D00002380A700E39634FF6DBBA1476392F904DB
:101D10006D398144630D0B008D479304C003630844
:101D2000FB009304000563048B01930440041375C6
:101D3000C507E30895D819453931393905452131A9
:101D400026850D3909453D314931E31C05D669BB6E
:101D500091476399F90013056006F536F53E1305C2
:101D600090090DB7E38F09D4F154A9BBBD660147B3
:101D70001736000013060624938606A6854583477A
:101D8000060093F7F70F91C382800507E3F9E6FE9B
:101D9000973700002380B722DDB77D166206618683
:101DA00093178601E18763D407000145828093176A
:101DB00026003307F500AE9718439C4363E7E7001E
:101DC0007D16E37FF7FC7D55828005458280FD15F9
:101DD000E205E18513978501618793F7F50F634865
:101DE0000700FD15139725002A97584365D71385DB
:101DF00017006205618582803308B5021C4283A802
:101E00000600B335B502C29733B50701AE984695C3
:101E100085486367B5006394A50063E307018148C3
:101E20000C43C6950CC388C21CC28280814713979D
:101E3000870161876343B7008280139727002A9741
:101E4000232007008507E5B781470147939687015F
:101E5000E18663C5B600133517008280939627008C
:101E6000AA9694428507558FD5B793D755408A07D0
:101E7000AA979C4305453315B5007D8D828017F3E5
:101E8000FFDFE702033B2A84993705C59317250036
:101E90003E940327C4FF814711EB7D1516053E953F
:101EA0004205418517F3FFDF6700E33A05838507A5
:101EB000E5B70145C5BF8147139787016187634334
:101EC000C700828013972700B386E50094422A97C3
:101ED000850714C3D5B77D1662066186014793173F
:101EE0008601E18763D507001335170082809317B9
:101EF0002600B306F500AE9794429C437D16B58F3D
:101F00005D8FF1BF8A05AA9501476363B5008280A2
:101F100083A6C5FFF11593D71600D98F9CC11397DF
:101F2000F601E5B72A830148014701456343D7001D
:101F30008280B387050183A80700B30706019C438D
:101F4000C697AA976384F80033B517010507B3084D
:101F50000301620723A0F80061871108C1BF2A832B
:101F600001478147014563C3D70082803388E5007C
:101F700083280800330EE600032E0E003388A840A5
:101F80003308C8416384080133B508018507B308E5
:101F9000E300E20723A00801E1871107E9B717F37F
:101FA000FFDFE70203290111B286B2842E86AA85DB
:101FB0000A8575372A84A6850A85793533348000E9
:101FC000060413351500018D056117F3FFDF670067
:101FD000832817F3FFDFE70243234111AA89AE8A62
:101FE000328BB68402C202C402C60144131C8401AF
:101FF000135C8C4163499C02939B1400FD1B0549B3
:10200000138CF4FFF15C3304890162046184634D35
:10201000740592478E04CE9423AEF4FE410117F36B
:10202000FFDF6700032213192400B30B2B01014AC1
:1020300093172A00D69783A50B00884378003400B5
:1020400050005D3B050A93178A01E187F11BE351BC
:10205000FCFE92474E9905042320F900A2473EC298
:10206000B24702C63EC459B7131A8901135A8A41AE
:10207000131D240093178A01E18763CF97009247CD
:102080000A044E941CC0A24705091379F90F3EC2F9
:10209000B24702C63EC485BFB3079A0313152A0090
:1020A00056950841780034005000050AEA97DA97FF
:1020B0008C439933C1B70000197106C212C416C609
:1020C0001AC81ECA22CC26CE2AD02ED232D436D658
:1020D0003AD83EDA42DC46DECAC0CEC2D2C4D6C648
:1020E000DAC8DECAE2CCE6CEEAD0EED2F2D4F6D638
:1020F000FAD8FEDA9385C1858841E7000500924051
:102100002242B2424243D2436244F24402559255C3
:102110002256B2564257D2576258F258064996494B
:10212000264AB64A464BD64B664CF64C065D965D43
:10213000265EB65E465FD65F096173002030000000
:1021400097210020938181E6174100201301816BC4
:1021500017F5FFFF130545EB97050020938585EAEA
:10216000171600201306C6FD63FAC500832205007A
:1021700023A0550011059105E3EAC5FE17A501004E
:1021800013054542971500209385C5FB13860184EE
:1021900063FAC5008322050023A0550011059105AF
:1021A000E3EAC5FE13850184974500209385852CBD
:1021B0006377B500232005001105E36DB5FEFD42F0
:1021C000739002BC8D4273904280B72200009382CC
:1021D000828873900230970200209382A2E293E2F9
:1021E000320073905230974200009382C2EA73909B
:1021F00012346FB0F46073002030397101436EC641
:1022000019A0397141536AC866CA62CC5ECE19A062
:10221000397101535AD056D252D44ED64AD826DA02
:1022200022DC06DE33016140828241114AC026C2AF
:1022300022C406C68282B24D4101024D924C224C0C
:10224000B24B4101024B924A224AB2494101024932
:1022500092442244B240410182803D432A87637305
:10226000C3029377F700BDEFADE5937606FF3D8A95
:10227000BA960CC34CC30CC74CC74107E36BD7FEDF
:1022800011E28280B306C3408A0697020000969648
:102290006780A6002307B700A306B7002306B70090
:1022A000A305B7002305B700A304B7002304B700B4
:1022B000A303B7002303B700A302B7002302B700AC
:1022C000A301B7002301B700A300B7002300B700A4
:1022D000828093F5F50F93968500D58D9396050131
:1022E000D58D61B793962700970200009696868257
:1022F000E78086FA9680C1171D8F3E96E374C3F877
:10230000A5B73367B500FD530D8B79E7B7877F7F9E
:102310009387F7F710419441B372F6003363F600E8
:10232000BE92B3E262006397720C6318D606504106
:10233000D441B372F6003363F600BE92B3E262009A
:102340006398720A631BD60410459445B372F60075
:102350003363F600BE92B3E262006391720A631EB9
:10236000D6025045D445B372F6003363F600BE92F0
:10237000B3E26200639A72086311D602104994496D
:10238000B372F6003363F600BE92B3E26200639369
:1023900072085105D105E30FD6F61317060193977E
:1023A0000601631CF7001357060193D70601330596
:1023B000F7409375F50F91E982804183C18333051E
:1023C000F7409375F50F91E182801377F70F93F73C
:1023D000F70F3305F74082800346050083C60500EA
:1023E000050585056313D60065FA3305D64082805E
:1023F00011059105E312D6FE014582802105A10554
:10240000E31CD6FC014582803105B105E316D6FCFC
:10241000014582804105C105E310D6FC014582805B
:10242000B717004003C777051377E70FA38BE704BF
:10243000130700F8A38DE7043D47238CE704130737
:102440005003A38CE70403C7A7051377D70F238D89
:10245000E7048280B717004003C7E7040D894111E4
:102460001377C70F498F93068008F3B6068093F65B
:10247000860836C601000100930670052380D70444
:10248000930680FA2380D704010001002387E70424
:1024900023800704B247F3A7078001000100410130
:1024A0008280B717004003C7E7020D8941111377F7
:1024B000C70F498F93068008F3B6068093F6860807
:1024C00036C601000100930670052380D7049306E9
:1024D00080FA2380D704010001002387E7022380CC
:1024E0000704B247F3A70780010001004101828081
:1024F00041112A83014E930E407E130F0019930F52
:10250000400663E56E129308001913034006B37882
:102510001503854E0D4FA14F337365020D89133599
:10252000150063EFBE121308F6FF79467298420851
:10253000135808013307C70213D61700BE07329796
:102540006146B3F6C60213068070B386C60236979C
:10255000A166F58F42075D8FB716004083C7F6026C
:1025600093F70708A303F1000346710083C7F6023F
:1025700093F70708E394C7FE83477100B71600403E
:1025800093F7F70F6388071293078008F3B7078064
:1025900093F787083EC401000100B7170040930677
:1025A00070052380D704930680FA2380D7040100A6
:1025B000010023AA070383C6170393E60608A3882E
:1025C000D70223800704A247F3A707800100010078
:1025D0001166B71700407D16D45BC85F938547032B
:1025E000A98EF18EF5FA93068008F3B6068093F66D
:1025F000860836C601000100930670052380D704C3
:10260000930680FA2380D7040100010098C103C714
:10261000170313670704A388E70223800704B24760
:10262000F3A7078001000100410182807D13336818
:10263000E3039308E016630E08003368F30393087E
:10264000D016630808009378330093B81800938875
:10265000D81633081E01131E0801135E0E0155B56E
:102660006393E5030548638608000148630303009C
:102670002A8871087298FD15131E0801C205135EA1
:102680000E01C18179BD13F8150063F4BF0079080C
:10269000D5B713381800E5BF83C7F60293F70708CC
:1026A000A303F1000346710083C7F60293F70708FE
:1026B000E394C7FE8347710093F7F70FF1DFE9B5A5
:1026C00031714AD966CB06DF22DD26DB4ED752D5E3
:1026D00056D35AD15ECF62CD6AC96EC7AA8C02D8D2
:1026E000EF00901C2A8993078008F3B7078093F7BF
:1026F00087083EDA01000100B71700401307700594
:102700002380E704130780FA2380E7040100010017
:1027100003C7F7021377770FA387E70203C7F70210
:1027200013678700A387E70223800704D257F3A724
:102730000780010001000545AD33130780C1334711
:10274000E902116A93070AE893065002BD69930BE8
:10275000A004814A014B13048008930470057D1A7C
:10276000B347F9023307D7023EC0FD873ECC9387BB
:1027700009A69309803E3347F7023AC27D873AC4DF
:10278000334739038549B399990193D93940B30641
:10279000D702B30B7703B3C6F602B3CBFB0236C640
:1027A000FD8636C893D6FB4136CEB7460F009386DA
:1027B00006243349D9028566938606FAB3969601B4
:1027C000B389E902130760553309D9029306001053
:1027D000B389E9023349D902B3C9F9029316390022
:1027E00036CA37190040FD8636D0930D090493D7B9
:1027F000F9413ED2F336048093F6860836DC0100B8
:102800000100930770052380FD00930680FA238062
:10281000DD00010001008346390593F6860FA30908
:10282000D9048346390593E61600A309D904238009
:102830000D00E256F3A6068001000100130C80FA99
:10284000116DF336048093F6860836DE0100010030
:10285000930770052380FD0023808D010100010096
:1028600083463905216693E60602A309D9048356F7
:102870000905B3E6A6012318D90483560905D18EAC
:102880002318D90423800D00F256F3A60680010018
:1028900001008346390593F60602638A061803464B
:1028A0003905218A6DDE0818EF00100473360480A4
:1028B00013768608B2C20100010023809D002380A8
:1028C0008D0101000100B717004003C637051376DC
:1028D000F60DA389C70403C6370513660602A3894C
:1028E000C704835609052166B3E6A6012318D90457
:1028F00083560905D18E2318D90423800D009646EE
:10290000F3A60680010001008346390593F606020E
:102910006386061483463905A18AEDFE97F0FF1FF2
:10292000E7806077AA8636D497F0FF1FE780A0760D
:10293000A256E30AD5FE835609054255B3E6A60121
:102940002318D904C12783463905A18AEDDE035631
:1029500009058346290582473376CA00B306DA02A1
:1029600093D5F641B296B388F640E24733B8C60035
:102970002E983308F840A247B3B616013308D84062
:1029800063C70701631DF800924763FA1701C24746
:10299000634DF80E63950701B24763E8F80E894668
:1029A00063E7660FF2469315180013D3F8015E86AD
:1029B00013951800B365B30042D646D4EF602125C5
:1029C0003258050B137BFB0F634700016312083875
:1029D000A258638F083613081500B336A800B695C1
:1029E00013D6F5013298B336C800AE9613581800C6
:1029F000FE06B3E606017336048013768608B2C677
:102A00000100010023809D0023808D010100010051
:102A10000356C902B296C206C1822316D902238088
:102A20000D00B646F3A606800100010019BDF3367D
:102A3000048093F68608B6C00100010023809D0043
:102A400023808D01010001008346390593E60602CB
:102A5000A309D90423800D00864605BDF336048002
:102A600093F68608B6C40100010023809D002380F0
:102A70008D01010001008346390593E60602A30992
:102A8000D90423800D00A646A5BDE30D0BF0F33657
:102A9000048093F68608B6C801000100930680FA08
:102AA00023809D002380DD0001000100834639055D
:102AB00093F5FC0F93F6860FA309D90483463905D5
:102AC000CD8EA309D90423800D00C646F3A6068047
:102AD00001000100130580FA034639059306390504
:102AE0001D8A631496297336048013768608B2CC47
:102AF00001000100130680FA23809D002380CD0091
:102B00000100010003C606001376F60D2380C600FF
:102B100003C60600136606022380C6008356090515
:102B20001166D18E2318D904835609052166D18EEA
:102B30002318D90423800D00E646F3A60680010081
:102B40000100130680FA8346390593F6060263886E
:102B5000062483463905130C3905A18AFDDA0818C5
:102B60006123F336048093F68608B6D00100010095
:102B7000930680FA23809D002380DD000100010080
:102B800083460C00116693F6F60D2300DC008346A5
:102B90000C0093E606022300DC0083560905D18E63
:102BA0002318D904835609052166D18E2318D90428
:102BB00023800D008656F3A606800100010013064F
:102BC00080FA8346390593F606026385062083461C
:102BD0003905A18AEDFE97F0FF1FE780C04B2A8CD4
:102BE00097F0FF1FE780204BE30C85FF8356090514
:102BF00011664255D18E2318D904292383463905FD
:102C000013063905A18AFDDAF336048093F68608A7
:102C1000B6D401000100930680FA23809D00238032
:102C2000DD00010001008346060093F6F60D230047
:102C3000D60023800D00A656F3A6068001000100F1
:102C40008356090503462905D247B376DA003306D1
:102C5000CA021305800C9355F6413696330DF640A3
:102C60008257333CD6002E9C3336A601330CFC40F1
:102C7000330CCC403308850392564E86B335A503FA
:102C80003305A503C295EF50917863468001631E1A
:102C90000C16630C0D16130615003335A6002E9581
:102CA0009356F5013696B335D600AA959396F5015D
:102CB00005828585D18E6346B000639D051A638BBE
:102CC000061A0356C90215823305D6003336C500ED
:102CD000B2956348B000639105241306F00F637D3D
:102CE000A622894663F3561593078008F3B7078039
:102CF00093F78708BED601000100371700409307FD
:102D000070052300F704930780FA2300F7040100FD
:102D100001008356C70289678117D58FC207C18317
:102D20002316F70223000704B657F3A70780010014
:102D30000100FA506A54DA544A59BA592A5A9A5A2E
:102D40000A5BFA4B6A4CDA4C4A4DBA4D29618280D3
:102D50001308F5FF3335A800FD152E951356F50120
:102D60003298B336C800AA9651B1F336048093F670
:102D70008608B6CA0100010023809D002380AD00B3
:102D80000100010083463905CD8EA309D9042380B3
:102D90000D00D646F3A606800100010035BBF336D0
:102DA000048093F68608B6CE0100010023809D00C2
:102DB0002380CD00010001008346390593E6060219
:102DC000A309D90423800D00F646F3A6068001006E
:102DD000010095BBF336048093F68608B6D2010055
:102DE000010023809D002380CD0001000100834667
:102DF000390593E60602A309D90423800D009656EF
:102E0000F3A60680010001006DBB9306F5FF33B504
:102E1000A600FD152E959355F501AE96B3B5B600F7
:102E2000AA951396F501858269B5F336048093F669
:102E30008608B6D801000100930680FA23809D0021
:102E40002380DD00010001008356C90205660116DA
:102E500093F6F60FD18EC206C1822316D9022380C3
:102E60000D00C656F3A6068001000100850A93FAFC
:102E7000FA0F49B233E6B60045C20356C90233051C
:102E8000D0403338A000B305B040B385054115826A
:102E90006345B000D1E16371A608894663F0560529
:102EA00093078008F3B7078093F78708BEDA01001D
:102EB0000100B7170040130770052380E7041307CC
:102EC00080FA2380E7040100010003D7C7027D8B4D
:102ED0002396E70223800704D65781BDF33604808A
:102EE00093F68608B6DC01000100930680FA238081
:102EF0009D002380DD00010001008356C9020566A4
:102F0000011693F6F60FD18EC206C1822316D9029E
:102F100023800D00E656B9B793078008F3B7078002
:102F200093F78708BEDE01000100371700409307C2
:102F300070052300F704930780FA2300F7040100CB
:102F400001000356C70293975600B297C207C18388
:102F50002316F70223000704F657C1BB914763EE1F
:102F6000B70217870100130767988A05BA959C4135
:102F7000BA978287B717004003A7470B1345F5FFA1
:102F8000698F23AAE70A03A7070B698F23A8E70A1B
:102F900003A7070A798D23A0A70A8280B7170040EC
:102FA00083A6470B1347F5FFF98E23AAD70A83A6FA
:102FB000070B558D23A8A70A83A6070A758F23A0A0
:102FC000E70A8280B717004003A7470B498F23AA5F
:102FD000E70A03A7070B1345F5FF45BFB7170040E6
:102FE00083A6470B1347F5FF758F23AAE70A03A7AC
:102FF000070A598D4DB7B717004003A7470B498FF4
:10300000EDB7914763EEB702178701001307478FAB
:103010008A05BA959C41BA978287B717004003A7E3
:10302000470D1345F5FF698F23AAE70C03A7070D8A
:10303000698F23A8E70C03A7070C798D23A0A70CA1
:103040008280B717004083A6470D1347F5FFF98E1E
:1030500023AAD70C83A6070D558D23A8A70C83A6FA
:10306000070C758F23A0E70C8280B717004003A7D9
:10307000470D498F23AAE70C03A7070D1345F5FF5A
:1030800045BFB717004083A6470D1347F5FF758F5F
:1030900023AAE70C03A7070C598D4DB7B7170040BB
:1030A00003A7470D498FEDB7B71700408847420582
:1030B00041819377050491EB9377F5013755E8014A
:1030C000130505803345F50282809377050C1307BD
:1030D00000046397E7009377F50137459C1CCDB753
:1030E0002165130505D0828037E700E01C43544377
:1030F000A183E206D58F1CC1FD572320F718232298
:10310000F718828013178500B7E700E023A0E710C7
:10311000618123A2A7108280B7F700E08847CC47DF
:103120008280814737370040A14663C4C70032859B
:1031300082800345B740E38EA6FE3385F500034544
:10314000050085072304A740CDB797070020938784
:10315000E7659C43173700201307C7313E95636E20
:10316000E500173700201307E7496368A700170732
:103170000020232DA7623E858280FD57EDBF4111BF
:1031800022C406C62A840D372947B307E502B24098
:103190008D83B3D7870222449507B3D7E702373729
:1031A0000040C207C1832316F70041018280716588
:1031B00041111305052006C6D937B737004013075C
:1031C00070F82381E7000D47A381E700130700048F
:1031D000A380E70005472387E700B24041018280D2
:1031E00037370040834727001A0593F7F703C98F45
:1031F00093F7F70F2301F7008280B737004003C72A
:10320000170019C9D98DA380B70003C7070013673A
:1032100087002380E700828093C5F5FFF98DA380A6
:10322000B7008280B73700402147B736004091E1B0
:10323000828003C6B700E30CC7FE05050346F5FF11
:10324000FD15C2052384C600C181D5B7411122C432
:1032500006C62A84913D2947B307E502B2408D8313
:10326000B3D7870222449507B3D7E7023737004028
:10327000C207C1832316F740410182807165411165
:103280001305052006C6D937B7370040130770F875
:103290002381E7400D47A381E74013070004A38083
:1032A000E74005472387E740B24041018280CC4197
:1032B000411106C6328503C6150083C505002206E6
:1032C0004D8E42068D654186138875A263080611EE
:1032D000634BC804138845A2630C060B634AC800FD
:1032E000938535A2630FB60623900600294669A888
:1032F000138855A26301060D938565A2E316B6FEF9
:103300008D451D4663E2E5081146198E63F3C7003B
:103310003E86B7E704002390C600FC47979501005E
:1033200093854522B9A8138895A2630F060F634AB7
:10333000060D1388A5A2630C0611938505A5E31558
:10334000B6FA99451D4663E1E504198E63F3C7009B
:103350003E86B7E704002390C600FC479385818032
:103360000DA09D451D4663E1E5022146198E63F3DC
:10337000C7003E86B7E70400FC472390C60093854C
:103380000184BA9582970146B2403285410182801C
:10339000AD451D46E3EAE5FE3146198E63F3C700ED
:1033A0003E86B7E704002390C600FC4797750100EE
:1033B00093850558F9B7B1451D46E3E7E5FC354669
:1033C000198E63F3C7003E86B7E704002390C6005A
:1033D000FC47977501009385A55665B78D451D4639
:1033E000E3E4E5FA1146198E63F3C7003E86B7E7BA
:1033F00004002390C600FC4797950100938545156E
:1034000049B78D451D46E3E1E5F81146198E63F392
:10341000C7003E86B7E704002390C600FC47979597
:1034200001009385A514B1BFA5451D46E3EEE5F463
:103430002946198E63F3C7003E86B7E70400239040
:10344000C600FC47977501009385C54D1DBFB54566
:103450001D46E3EBE5F23946198E63F3C7003E865D
:10346000B7E704002390C600FC47977501009385D9
:10347000654A01BFB7E7040003A3071397060020BE
:10348000938646D54146A54517050020130585CBF3
:1034900002832D4559EF03C5050009476317E50869
:1034A00003A84500411106C60347180032850346AC
:1034B000080022074168518F930828FE630817030C
:1034C00063E9E80005186303070523900600294512
:1034D0001DA8130648FE630BC7021518E31707FF64
:1034E00015463E87637BF602154705A83E8691C3C5
:1034F0000546B7E70400FC472390C6004206CC45CA
:10350000418282970145B240410182801306700FCB
:103510003E876374F6001307700FB7E7040023902B
:10352000E600FC4713160701D9BF239006000545A6
:1035300082808280416779176302E504411122C4C9
:1035400006C685472A84639DF500B7E704002285F7
:103550002244B24003A387139385C18441010283AF
:1035600089476399F500B7E7040083A7070B8545F2
:10357000829761DDB240224441018280828079716C
:1035800022D452CC2E842A8A977501009385853DDA
:10359000177501001305C53E06D63AC626D24AD095
:1035A000B68432894ECEEF50D131A6851775010011
:1035B0001305053EEF50F1302945EF509134834714
:1035C000840093F70702F1E3834904008947054526
:1035D00032476394F908544083C7160083C6060037
:1035E000A207D58FC166138616FE638CC7028D169F
:1035F000638DD7068D66938626902945639FD704F1
:10360000B7E70400A285225403A34714B250F2493D
:10361000A6864A86925402595285624A8547456178
:1036200002832D451DEB9307700F354563E7970225
:10363000B7E70400FC4748441306700FCA85829719
:103640008149938781859C43014581CB9C4391C7E8
:103650004E852686CA8582970145B25022549254DF
:103660000259F249624A456182802D457DF79307F0
:10367000700F3545E3E397FEB7E70400FC47484485
:103680001306700FCA8582976DBF2145F9B74111A6
:1036900022C437E404008327841326C2AA84416528
:1036A00006C69385C1847D1582978327C40A1705B2
:1036B0000000130565E88588829795C003230413ED
:1036C0002244B240924497060020938666C2414647
:1036D000C545170500201305A5B041010283B2407E
:1036E0002244924401454101828009C523ACA18452
:1036F000014582804545828011476360A70A97761D
:1037000001009386E6240A0536951841411106C644
:103710003697AE87B28502871307700F6145639BAA
:10372000E700B7E70400FC471306700F1385C18B51
:1037300082970145B2404101828005476145E39B84
:10374000E7FEB7E70400FC47054613858184CDB743
:103750001307700F6145E39FE7FCB7E70400FC47E0
:103760001306700F1385419BE1B71307700F614576
:10377000E392E7FCB7E70400FC471306700F1385DC
:10378000C1AA7DB715476145E396E7FAB7E704009C
:10379000FC4715461385018561BF094582804111AB
:1037A00026C2B7E4040083A7C41322C44AC006C6D5
:1037B0002E849385C1842A898297058905C5970738
:1037C00000209387E7A183D7A70BA28503A3440D0D
:1037D0002310F4002244B24092444A850249014633
:1037E00041010283B24022449244024949454101C9
:1037F000828011456FE0DFEC411193962500AA8588
:103800002D4506C697F0FF1FE780A01FB240014577
:1038100041018280011122CC06CE3714004026CA15
:103820004AC84EC652C483447405034AB40583494A
:10383000840503499405EFE0BFBE8347A40593F4D4
:10384000F40F137AFA0F93E71700230DF40493F99A
:10385000F90F1379F90FB717004003C7A705058BB8
:103860006DFF03D5C705A38D4705238C3705A38CB2
:103870002705A38B9704F2406244D2444249B249DF
:10388000224A0561828041119397050122C406C630
:1038900026C2C1872E8463D00702B7E40400FC541B
:1038A000829719C1BC5482972165218DB240224470
:1038B00092444101828093F7150013C51500FDF76E
:1038C0009397250163D30702B7E4040083A7C41EBE
:1038D00082970537BC4C37F60200130606E089656F
:1038E00003C5018682970965C9B7939715010145FC
:1038F000E3DE07FA1775010013054510EF50B1100C
:10390000B7E70400BC4F13060064916503C5018648
:103910008297116559BF2D71232A9110FD74E98C8E
:10392000232C811023282111232631112A84AE89CA
:103930003289930600100A86A6852D45232E111084
:1039400097F0FF1FE780E00B13154401B7E7040071
:10395000FC4751810A0513962900CA850A9582976A
:10396000A68585660146254597F0FF1FE78060091B
:103970000A86A68593060010294597F0FF1FE78069
:1039800040088320C111032481118324411103299C
:1039900001118329C11015618280B7F7070003C7A1
:1039A0000701411106C622C426C24AC0A547631AB0
:1039B000F7009537B2402244924402490145410143
:1039C000828013942500AA843289A286AA850146A2
:1039D000254597F0FF1FE780C002A2864A86A6858C
:1039E000294597F0FF1FE780C001E9B71D71A2CC00
:1039F00037E404005C5C485886CE49469775010060
:103A0000938545FB829701E9177501001305C5FBF6
:103A1000EF50617F01A0B7F600E0795798CAFD57D3
:103A2000DCCA0567B7E700E023A0E7101306F00241
:103A300090C223A0E71801000100370700201847B3
:103A400013060004814523AEE1844157A38AE74071
:103A50003C4408088297971700209387A7E83EC840
:103A6000856713870740231AE1001D673ACC3707A3
:103A70000105130707109387B7D33ACE2312F1023B
:103A80001307B00F97F7FFFF938747692310E102F1
:103A90003ED8094797070000938707D82301E10222
:103AA0003EDC17070000130767D5970700009387D0
:103AB00087D4B7F50700BAC23EDE17070000130728
:103AC00007EE970700009387C71B81463000E1058A
:103AD0001945BAC43EDA97F0FF1FE78080F2180854
:103AE0008147994630003E96034606008507050744
:103AF000A30BC700E398D7FEC24791C70357410104
:103B000085676373F70001A0B7E7040083A7470A3E
:103B100008088297AA8501C917750100130505ECED
:103B2000EF50215A01A0F640664425618280411180
:103B300026C2B7E4040083A7040806C622C41705FA
:103B40000000130585D48297138401862300A40006
:103B50008520E12A03450400224403A38405B240E2
:103B60009244130600328965410102834111930793
:103B70008008F3B7078093F787083EC6010001006D
:103B8000B7170040130770052380E704130780FA76
:103B90002380E70401000100C8DB23800704B2474B
:103BA000F3A707800100010023A201864101828062
:103BB000797106D622D413078008F337078093F76C
:103BC00087083EC201000100B71700409305700549
:103BD0002380B704130680FA2380C7040100010084
:103BE00083C6F70293F6A60FA387D70223800704A4
:103BF0009246F3A606800100010073370780137711
:103C000087083AC4010001002380B7042380C70459
:103C10000100010003C7F70213672700A387E7022B
:103C200023800704A247F3A7078001000100054590
:103C3000EFE03F877D3E0147814681470546854548
:103C40001305407EEFE0DF8A37E404003C4468005F
:103C5000514681458297B707C0A83EC8B787E80399
:103C6000938707D03ECA97F7FF1F938707C53EC6C5
:103C70007C5868008297B2502254456182800111BD
:103C800022CC06CE930730031304D5FC63E7A700CC
:103C90003704C0A81304D4FC2A946800EFF0CFC402
:103CA00097E0FF1FE780203FB307A4406376A4009E
:103CB000B707C0A8A297898F3747F6A681171307C1
:103CC00007C6637AF7003245EFF0CFC30945F240EB
:103CD0006244056182802285513D3245EFF08FC2FA
:103CE000373700408347574093F707048DCF9387BA
:103CF00041869C430D45E1FF1165690597E0FF1F73
:103D0000E78080510545EFE0EFF497E0FF1FE78083
:103D100080382AC497E0FF1FE780E037A247E30B13
:103D2000F5FE01456DB7010075BF4111130780080D
:103D3000F337078093F787083EC401000100B717E7
:103D40000040930570052380B704130680FA238092
:103D5000C7040100010083C6E70093E686002387BD
:103D6000D70023800704A246F3A6068001000100C5
:103D700073370780137787083AC601000100238054
:103D8000B7042380C7040100010003C717031367AA
:103D90000702A388E70223800704B247F3A707803E
:103DA00001000100B7E700E03707001023A0E7108B
:103DB000410182804111977501009385E5331775A4
:103DC00001001305E5BB06C6EF50A12F17750100D2
:103DD0001305054DEF50E12EB240294541016F50CA
:103DE00041324111977501009385453217750100E5
:103DF000130505B906C6EF50C12C17750100130550
:103E0000E548EF50012CB240294541016F50612F28
:103E1000411122C406C6834705002A849DC39775B5
:103E200001009385653417750100130565B5EF50E2
:103E300041294C40177501001305C55AEF50612800
:103E40001DA058411DE7977501009385E531177551
:103E500001001305E5B2EF50C126177501001305E7
:103E6000E559EF5001262244B240294541016F50E7
:103E70004129A1679386D7036311D7029775010083
:103E80009385852E17750100130585AFEF506123CB
:103E90001775010013058557E9B7ED079775010000
:103EA0009385852C17750100130585AD6319F700FF
:103EB000EF50212117750100130585565DB7EF50AE
:103EC00041204C40177501001305855785BF4111EE
:103ED000977501009385C52417750100130545AA40
:103EE00006C6EF50011EB240294541016F506121C5
:103EF000797122D426D24AD02E842A898145B2846F
:103F00004800714606D6EFE04FB597F7FF1F93873D
:103F1000A75DDC4783D70700231421012313F10099
:103F2000EF20206C9547A305F1009307401F3EC684
:103F3000FD572305A100230AF100EF20007C26860F
:103F4000A2854800EF20406CB2502254925402598E
:103F5000456182802399018823880188B7E704009E
:103F6000BC47411106C6414681451715002013057F
:103F7000A5958297EF109055EF1050340145EF2032
:103F8000F07A03C7417A9307F00A631BF70093079F
:103F9000F00889451385417A2392F17AEF30E023C6
:103FA000EF30E03581453705040023A401882392D2
:103FB000018823830188239F0186239E0186239104
:103FC000018823960188EF2000250145EF30C029A4
:103FD0009775010093854517177501001305459ADC
:103FE000EF50210E177501001305C54BEF50610D01
:103FF000B240294541016F50C110411122C406C68B
:1040000026C293F715002E846389070C814617F6A4
:10401000FF1F1306E64A854503D58187EF8020728E
:1040200005C5977501009385E51217750100130505
:104030002595EF50010917750100130565B4EF5080
:1040400041082945EF50E10B9775010093858510D4
:10405000177501001305C592EF50A10617750100F1
:10406000130545B3EF50E1052945EF50810917F5D8
:10407000FF1F130565475C4505472390E700EFF0F8
:104080006002977501009385E50C17750100130513
:10409000258FEF500103177501001305E5B0EF50B0
:1040A00041022945EF50E105930710F82382F17A88
:1040B00083D74187A382F17A1385417AA183914501
:1040C0002383F17AA383017AEF3020111345140082
:1040D000B240224492444101828093F72500D1C32B
:1040E00003D7418825CF9386818894429777010032
:1040F0009387473D03C66188814517050020130556
:10410000A57CEF400071AA8431C9977501009385A1
:10411000250B177501001305A586EF40917AA6853A
:10412000177501001305C5A9EF40B1792945EF4086
:10413000517D23920188930710F82382F17A83D767
:104140004187A382F17AA1832383F17A91458D4738
:104150001385417AA383F17AEF30200813452400B8
:1041600085BF93F74500A1CF97750100938545055D
:10417000177501001305C580EF40B1741775010074
:104180001305C5A5EF40F1732945EF4091779307DB
:1041900020F82382F17A83D7E187A382F17AA18381
:1041A0002383F17A8547A383F17AEF2000551385A5
:1041B000417A9145EF3060021345440011BF93F7F7
:1041C00085009DCB97750100938585FF17650100DC
:1041D0001305057BEF40F16E17750100130545A12E
:1041E000EF40316E2945EF40D17123920188EF40B5
:1041F000206F13458400E9BD93F70501A1CF8545E4
:1042000003D5E187EF00313997750100938545FBB0
:10421000176501001305C576EF40B16A17750100F7
:104220001305459EEF40F1692945EF40916D9307D5
:1042300030F82382F17A83D7E187A382F17A13855C
:10424000417AA1838D452383F17AEF2010791345BC
:104250000401BDBD93F70502B1CF977501009385A9
:1042600025F6176501001305A571EF4091651775D7
:1042700001001305659BEF40D1642945EF4071684B
:10428000930740F82382F17A83D7C187A382F17A1A
:10429000A1832383F17A8547A383F17A239E018644
:1042A000EF20A0451385417A9145EF201073134507
:1042B000040239BD93F70504D9CF977501009385A2
:1042C00025F0176501001305A56BEF40915F177589
:1042D00001001305E596EF40D15E2945EF4071627C
:1042E00083C7417A1307700A6384E7041307800ABF
:1042F0006380E7061307600A6395E702930760F897
:104300002382F17A83D72188A382F17AA183238340
:10431000F17A8547A387F17AB1451385417AEF2079
:10432000D06BEF20803D13450404239101884DB3E9
:10433000930770F82382F17A83D72188A382F17AD8
:10434000A1832383F17A8547A384F17A9945F1B754
:10435000930780F8C5B793F705080145E38A07D6A8
:10436000977501009385C5E5176501001305456143
:10437000EF403155177501001305058EEF4071545C
:104380002945EF4011589307A0F82382F17A83D78B
:10439000C188A382F17AA1832383F17A8547A3831D
:1043A000F17A23960188EF2040351385417A9145B3
:1043B000EF20B0621345040821BB411122C4977558
:1043C00001009385A5DB2A84176501001305455B71
:1043D00006C6EF40114F4C4017750100130505FE4E
:1043E000EF40314E2945EF40D15103470400930778
:1043F000F00F6319F70297750100938525D81765AB
:1044000001001305E557EF40D14B4C4017750100F3
:104410001305C5FBEF40F14A2244B2402945410152
:104420006F40314EB24022444101828085CD41111E
:1044300022C4176501001305A5542E849775010049
:104440009385C5CE06C6EF40D147A28517750100FA
:1044500013050503EF40F1462244B24029454101CE
:104460006F40314A8280411122C426C22E84AA8420
:1044700097750100938545CC1765010013054550DC
:1044800006C6EF4011441775010013052500EF40E3
:1044900051432945EF40F146977501009385C5C901
:1044A000239C9186176501001305854D8544239A49
:1044B0008186239B918623998188EF40914083D503
:1044C0002189177501001305E5FCEF40913F29454F
:1044D000EF40314323889188EF10405E2285EF2022
:1044E000F0240545EF20505897F7FF1F9387C7FF2B
:1044F000DC4703D70700C167FD176310F7022244AA
:10450000B7E70400B240924403A3870503C5818640
:104510001306000A854541010283B24022449244B9
:1045200041018280011122CC37E404005C5C06CE9C
:1045300026CA3546977501009385C5D717750100C2
:1045400013054566829701E9176501001305C54704
:10455000EF40714B01A097F7FF1F9387675F3EC441
:10456000B7F507008567938707C081461386C18624
:10457000E10519453EC697E0FF1FE78080487C446F
:1045800019469385C186170500201305252D8297AE
:1045900034001386C186977501009385251C177515
:1045A00001001305251DEF30507FAA8415C99775AA
:1045B00001009385E5BF176501001305653CEF40D9
:1045C0005130A685177501001305C5CFEF40712F37
:1045D0002945EF401133F2406244D24405618280A4
:1045E000EFA02016177501001305C5C4EF30801A1F
:1045F000EF706004EF00F12217F5FF1F130585EB44
:10460000EF00D10F177501001305C5C3EF0031236B
:10461000AA84EF302075EFC04048EF209142EF4070
:104620005011EF307054EFE03025977501009385FD
:1046300025B8176501001305A53489C8EF40712816
:10464000A68517750100130525CA49B7EF407127E4
:1046500017750100130585CBEF40B1262945EF40C2
:10466000512AEFE0D007EFB00032630D050C85450D
:1046700037050400EF10303A97750100938545B374
:10468000176501001305C52FEF40B1231775010011
:10469000130545C9EF40F1222945EF40912697F7D0
:1046A000FF1F9387A7D483D707002399F1888547F5
:1046B0002388F188EF10405CEF10404003D521893A
:1046C000EF20D00683C7F188B9EFA3030100832749
:1046D000441713067100854513055030829797756E
:1046E00001009385E5AC1765010013056529EF40CE
:1046F000511D17750100130525C5EF40911C294573
:10470000EF40312097750100938585AA1765010058
:1047100013050527EF40F11A177501001305C5C8E9
:10472000EF40311A75B597750100938565A8176537
:1047300001001305E524EF40D1181775010013059A
:1047400025C465BF97750100938585A6176501008F
:1047500013050523EF40F11617750100130585D4E5
:10476000EF4031162945EF40D1190145EF20D02FF8
:1047700051BF411122C437E404008327041A06C63E
:104780008297EF20700383270408170500001305A4
:10479000058782972384A18617F5FF1F1305C5D4CB
:1047A000EF2000212244B2404101ADBB411122C49F
:1047B00091462A84170600201306C6079D652D45DD
:1047C00006C697E0FF1FE780C023B7F7070003C7BF
:1047D0000701A5476313F70001A0930600100146E7
:1047E0009D65254597E0FF1FE780A02197070020E2
:1047F000238287042244B240914617060020130604
:1048000066039D652945410117E3FF1F6700631F8C
:10481000B7E704001171FC47CED79389417AA2DD36
:10482000CAD986DFA6DB2E8432892E86AA854E85DC
:10483000829783C70900130780029387E70793F7DE
:10484000F70F636CF772176701001307671B8A077E
:10485000BA979C43BA9782878D47977501009385D5
:104860006597176501001305A511630BF400EF4070
:104870005105176501001305A554EF409104CDA221
:10488000EF4031041765010013050555EF40710332
:104890002945EF401107930720F811469385417A87
:1048A0004A852382F17AA383017AEFF06FE42A84A8
:1048B0000DC5977501009385E591176501001305F6
:1048C000250CEF401100A2851765010013058554E2
:1048D000EF40217F2945EF40D10297750100938574
:1048E000658F176501001305A509EF40817D1765E8
:1048F000010013056553EF40C17C2945EF4071006D
:104900004165930730FA05469385417A7D152382E8
:10491000F17AEFF0EFDD2A840DC5977501009385DC
:10492000658B176501001305A505EF408179A28508
:10493000176501001305054EEF40A1782945EF40AA
:10494000417CB7E70400BC4F0566130606C8A145C5
:1049500003C581868297FE506E54DE544E59BE596F
:104960001161828091476301F4029775010093857C
:104970006586176501001305A500EF408174176572
:1049800001001305A54DD5BDB7E70400FC4F9145C7
:1049900003C581868297977501009385A583176566
:1049A00001001305E5FDEF40C17117650100130516
:1049B000A54CEF4001712945EF40A174EF10F05371
:1049C0009145C1A285476301F40297750100938563
:1049D0006580176501001305A5FAEF40816E176524
:1049E00001001305E54A51BD239F2187B7E7040065
:1049F0000566BC4F130606C8C14599BF8D476301C4
:104A0000F402976501009385E57C176501001305A5
:104A100025F7EF40016B1765010013052549B1BD6E
:104A2000930740F811469385417A4A852382F17AAB
:104A3000A383017AEFF0CFCB2A84E30E05F09765CC
:104A400001009385257917650100130565F3EF4093
:104A50004167A285176501001305C53BEF406166FC
:104A60002945EF40016AC5BD9147E31CF4F8B7E75B
:104A70000400FC4F9305000203C581868297976569
:104A800001009385257517650100130565EFEF405B
:104A90004163176501001305E54221BF894763E1C2
:104AA0008702976501009385E5721765010013057C
:104AB00025EDEF400161176501001305E54175BB68
:104AC00083C4617A83C7517A9765010093858570A5
:104AD000A204176501001305A5EADD8CEF40615EB5
:104AE000A2851765010013056540EF40815DC20492
:104AF0002945EF400161C1849305D4FF93960401D9
:104B0000C1824A8693F5F50F1385717AEF102074F0
:104B1000E35390E4930750F82382F17A83C7390076
:104B200022869385417A85074A85A383F17AEFF03F
:104B30002FBC2A84E30105E297650100938585690E
:104B4000176501001305C5E3EF40A157A28517754E
:104B500001001305E59119B7894763E1870297655D
:104B600001009385256717650100130565E1EF4096
:104B70004155176501001305253901B3EF10F037D2
:104B8000A2851385417AEF204065F1B38D4763011B
:104B9000F402976501009385E5631765010013052D
:104BA00025DEEF400152176501001305A537F1B16D
:104BB000B76602000146B7750200054597E0FF1F82
:104BC000E78020E4930760F82382F17AA383017AD7
:104BD0009307002623A4F17AE5779387072123968C
:104BE000F17A3146A387A17A9385417A4A85238752
:104BF000017AEFF0EFAF2A84E30F05D49765010047
:104C00009385455D17650100130585D7EF40614B1E
:104C1000A285176501001305653289B5B1476301A7
:104C2000F402976501009385E55A176501001305A5
:104C300025D5EF400149176501001305E53135B968
:104C4000B7E70400FC4F9305000403C581868297F3
:104C5000EF10B02AB14535B7914763E187029765F8
:104C600001009385255717650100130565D1EF40B5
:104C70004145176501001305E52F01B183C4817A11
:104C800083C7717AA204DD8C8E04B77702006D149D
:104C9000BE942286A685176501001305E52EEF4018
:104CA0004142B7E70400FC4722869385917A2800A9
:104CB000829793160401C1823000A685094597E0CA
:104CC000FF1FE78000D42A8419C51765010013056A
:104CD000652DEF404153930770F819469385417A4B
:104CE0004A852382F17AA384817AEFF06FA02A8427
:104CF000E30305C6976501009385C54D176501005F
:104D0000130505C8EF40E13BA285176501001305B7
:104D1000652AA9B399476301F4109765010093854B
:104D2000654B176501001305A5C5EF40813917656F
:104D300001001305A52991B6914763E187029765A4
:104D400001009385254917650100130565C3EF40F0
:104D50004137176501001305E52805B683C4817A3C
:104D600083C7717AA204DD8C8E04B77702006D14BC
:104D7000BE942286A685176501001305E527EF403E
:104D80004134B7E70400FC4722869385917A2800D6
:104D9000829793160401C1823000A6850D4597E0E5
:104DA000FF1FE78000C62A8419C517650100130597
:104DB0006526EF404145930780F819469385417A6F
:104DC0004A852382F17AA384817AEFF06F922A8454
:104DD000E30305B8976501009385C53F176501009A
:104DE000130505BAEF40E12DA285176501001305F3
:104DF000A523ADB199476301F4029765010093853E
:104E0000653D176501001305A5B7EF40812B1765B8
:104E100001001305E52295B4B7E70400FC4F9305A4
:104E2000000403C581868297EF10300D994591BB30
:104E30008D476301F402976501009385A5391765D5
:104E400001001305E5B3EF40C12717650100130505
:104E5000A52025B41765010013050521EF40A13AEF
:104E60001305C01297E0FF1FE780C09D0145EFE0EA
:104E7000AFA70D45EFF09F93294597E0FF1FE7800F
:104E8000609C97E0FF1FE780808DF1B49947630134
:104E9000F402976501009385E5331765010013055A
:104EA00025AEEF400122176501001305A51CF1B2E4
:104EB00003C7917A83C7817A22075D8F9166BA967C
:104EC000C2061166C1821306F6EF8D476363D602F0
:104ED00097E7FF1F938747619C4B03C6717A9386C0
:104EE000C70039C603D607004DCA8907E39CD7FE21
:104EF00089471307A0F811469385417A4A85238292
:104F0000E17AA383F17AEFE0BFFE2A84E30505A4EA
:104F1000976501009385052C17650100130545A6CB
:104F2000EF40211AA285176501001305E5153DB66E
:104F300003D607006300E60A8907E39BF6FE8D4768
:104F40004DBF91476302F402976501009385852860
:104F5000176501001305C5A2EF40A11617650100F2
:104F6000130505146FF07F91B7E70400FC4F93051C
:104F7000000803C58186829791B4976501009385E7
:104F80006525176501001305A59FEF40811317657F
:104F90000100130565126FF05F8E2390E70017E59F
:104FA000FF1F13056554EFE080119765010093859D
:104FB0006522176501001305A59CEF408110176558
:104FC000010013056510EF40C10F2945EF40611343
:104FD000814705B72390070017E5FF1F1305C5504C
:104FE000EFE0E00D976501009385C51E1765010090
:104FF00013050599EF40E10C176501001305450EF7
:10500000D9B7411122C406C6834705002A849DC32F
:10501000976501009385C51717650100130545962F
:10502000EF40210A4C40176501001305A54AEF40E7
:10503000410965A05841B707CF009387777D631179
:10504000F706976501009385A51417650100130500
:105050002593EF4001071C448356E4008355C400A8
:1050600003C607001765010013054548EF406105B9
:105070002945EF4001090357E40083D721896307DD
:10508000F7008355C4000844EFE0CF990356E400CD
:105090008355C40008442244B24041016FF04FF7E9
:1050A000B707CC009387777D631FF70297650100F0
:1050B0009385050E176501001305858CEF4061008F
:1050C0001C448356E4008355C40003C607001765DB
:1050D00001001305A541EF30D17E2244B24029459D
:1050E00041016F400102B707CE009387777D6302CD
:1050F000F702976501009385A5091765010013055F
:105100002588EF30117C4C401765010013054533AD
:1051100039BFB2402244410182805171CAD137E97E
:1051200004008327C904A2D52E8686D7A6D32E8451
:10513000AA851385417A829783C7417A1307700A3B
:10514000638BE70C636CF7001307600A6382E70464
:10515000BE502E549E540E596D6182801307800AF2
:105160006380E7121307900AE394E7FE8D47630913
:10517000F416976501009385A507176501001305CF
:105180002580EF301174176501001305A59C15A04B
:105190008D476306F40297650100938565051755F1
:1051A00001001305E57DEF30D1711765010013058E
:1051B000A593EF3011712945EF30B17451BF854788
:1051C00017650100130505942380F188EF40A103C2
:1051D000B7750200B76602000146054597E0FF1F5C
:1051E000E7802082930760F82382F17AA383017A13
:1051F0009307002623A4F17AE57793870721239666
:10520000F17AB1452387017AA387A17A1385417A80
:10521000EF10B07C35BF914763E1870297650100CD
:10522000938505FD1755010013058575EF307169EC
:10523000176501001305058FADBF83C4817A83C74D
:10524000717AA204DD8C8327C9046D1422869385AC
:10525000917A280082978E0493160401B775020094
:10526000C1823000A695094597D0FF1FE78060797D
:10527000930770F82382F17A9945A384A17A79B7CC
:10528000914763E1870297650100938565F617559D
:1052900001001305E56EEF30D162176501001305BB
:1052A000E58901BF83C4817A83C7717AA204DD8C4A
:1052B0008327C9046D1422869385917A28008297EA
:1052C0008E0493160401B7750200C1823000A695C2
:1052D0000D4597D0FF1FE780C072930780F859BF34
:1052E0001765010013054588EF30F1711305C012F1
:1052F00097D0FF1FE78000550145EFD0FFDE0D4539
:10530000EFF0CFCA294597D0FF1FE780A05397D071
:10531000FF1FE780C0442DBDB7E704004111FC47E3
:1053200026C29384417A2E8606C622C44AC02E84A1
:105330002A89AA852685829797650100938505EDC0
:10534000175501001305C563EF30B15783C5417A86
:10535000176501001305C591EF30B1562945EF30AF
:10536000515A83C7040041479387070693F7F70F05
:105370006363F746175701001307C7728A07BA9786
:105380009C43BA9782879D476303F40297650100A7
:105390009385C5E7175501001305855EEF307152FF
:1053A000176501001305458DEF30B15155AA83C72C
:1053B000517AADC783D7817A03D7617AC207D98F73
:1053C00023A4F18883C7640097650100938505E4F1
:1053D000175501001305C55A2383F188EF30714E2C
:1053E000938781888C4303C6618817650100130584
:1053F000658AEF30114D2945EF30B150A382017A13
:105400002244B24092440249930700F82382F17A81
:105410009D451385417A41016F10305CEF30E057B4
:105420002393A17A935705012A842384F17A935711
:1054300085010145A384F17AEF30E0562385A17AF6
:1054400097650100938585DC1755010013054553C9
:10545000EF30314703C6A17AA28517650100130515
:10546000E58441BFCD476301F40297650100938550
:10547000E5D9175501001305A550EF309144176584
:105480000100130525840DB737E404007C44414630
:105490009385517A17F5FF1F13050543829717F57A
:1054A000FF1F13056542EF008076092D83C7617BDE
:1054B00003C7517BA20703238405D98F2392F18868
:1054C0001306000A89452244B2409244024903C5AA
:1054D0008186410102838D476301F40297650100D3
:1054E0009385C5D21755010013058549EF30713DED
:1054F000176501001305C58C45BD03C4617A83C7D8
:10550000517A97650100938565D0220417550100F3
:10551000130505475D8CEF30D13AA2851755010080
:105520001305C57BEF30F1392945EF30913D0D462C
:105530009385417A2285EFE0BF9BAA8415C99765C0
:1055400001009385A5CC1755010013056543EF3085
:105550005137A6851755010013058579EF3071364F
:105560002244B24092440249294541016F307139C9
:10557000239F8186B7E70400116603A387051306FE
:1055800006E8914589B78D476301F40297650100EC
:105590009385C5C7175501001305853EEF3071325D
:1055A000176501001305859001B503C4617A83C7AF
:1055B000517A97650100938565C52204175501004E
:1055C0001305053C5D8CEF30D12FA28517550100E6
:1055D00013054573EF30F12E2945EF3091320D461A
:1055E0009385417A2285EFE0BF90AA840DC197652B
:1055F00001009385A5C11755010013056538EF30EB
:10560000512CA685175501001305057181BF239EF6
:105610008186B7E70400116603A38705130606E831
:10562000930500024DB5894763E187029765010044
:105630009385C5BD1755010013058534EF307128DA
:10564000176501001305458985B383C4617A83C753
:10565000517A97650100938565BBA2041755010037
:1056600013050532DD8CEF30D125A68517550100D5
:105670001305056CEF30F1242945EF30912822867F
:105680009385417A2685EFE0BF862A846304051658
:1056900097650100938585B7175501001305452EC1
:1056A000EF303122A285175501001305A5697DB59C
:1056B000854763F18714834519002244B240924420
:1056C0000249B335B0002380B18817550100130596
:1056D000A56841016F30F11EA2852244B240924478
:1056E0004A85024941016FF05FA399476301F402C3
:1056F00097650100938585B117550100130545286D
:10570000EF30311C176501001305C59671B903C44C
:10571000617A83C7517A97650100938525AF22048A
:10572000175501001305C5255D8CEF309119A28531
:10573000175501001305C563EF30B1182945EF3047
:10574000511C19469385417A2285EFE06FFAAA84AD
:105750000DC197650100938565AB175501001305D1
:105760002522EF301116A685175501001305456156
:10577000F5B323968188B7E70400116603A3870574
:10578000130606E8930500083DBB854797650100B1
:105790009385C5A7175501001305851E6309F400FD
:1057A000EF303112175501001305C55EF5BEEF301D
:1057B0005111175501001305655FEF309110294510
:1057C000EF3031142244B2409244024923920188BE
:1057D00041016F30E01097650100938525A31755AF
:1057E00001001305E519EF30D10D17650100130510
:1057F000A58C5DBEB24022449244024941018280A0
:10580000411106C622C4EFE0AFEE9377F50F95CBBA
:105810002A84976501009385E5A0175501001305BB
:105820002516EF30110A9375F40F17650100130563
:1058300025C4EF3011092244B240294541016F309F
:10584000510CB24022444101828001114EC683D6E0
:105850002189B28903D6818226CA4AC806CE22CCC3
:10586000AA842E89CD2183C70189A9C703C4440016
:1058700083C7340017650100130585CB22045D8CB6
:10588000EF3031044A86A68522859D3F638B09024D
:1058900083C7E1889DC76306090283C7018895E332
:1058A0006244F240B249CA8526854249D244056124
:1058B0006F10B01217650100130505C8EF30B11461
:1058C000F1B7F2406244D2444249B2490561828054
:1058D000834755008345450017650100130505C43E
:1058E000A207DD8D6F30E17D17650100130505C24C
:1058F0006F3071118D4763FAB708011126CA06CEC1
:1059000022CC0344350083C4F18897650100938558
:1059100065C3B3378000A387F18809C49765010088
:10592000938505C317650100130505C3EF30617941
:1059300083C7F18863839700212C83C7F1889DC3B7
:1059400085472306F100B7E7040083A747177000D7
:105950008545130550308297176501001305C5C0B2
:10596000EF30710A9967938757EE2316F1006800AC
:1059700085479145A30781002307F100EF10F0054B
:10598000F2406244D244056182808280894763FE8E
:10599000B706011122CC06CE26CA834425008547CE
:1059A0002A846396F404914763FEB70203454500D9
:1059B0008347340022055D8D2394A18209299967CC
:1059C000938767EE2314F100834734002305910089
:1059D000A305F10083474400954528002306F10004
:1059E000EF10A07FF2406244D24405618280FDF84E
:1059F0009967938767EE2314F10083D78182A3050B
:105A0000F10023050100A183C1BF828001119967C4
:105A100022CCD517138401892314F1008347040095
:105A200026CA938421892305F10083D70400280026
:105A30009545A305F100A18306CE2306F100EF10E2
:105A4000C07903D6040083450400176501001305DF
:105A500025B3EF300167F2406244D2440561828091
:105A60009D677971D9172316F10083C7018906D67E
:105A70002307F1009DCBB7E70400FC47414697F5AB
:105A8000FF1F938565E41305F10082976800CD45FB
:105A9000EF10A07483C5018917650100130545B196
:105AA000EF302162B25045618280B7E70400BC4705
:105AB000414681451305F1008297C9BFB7670203CC
:105AC0006971938757AA3EC4856793871770231619
:105AD000F1009387018983C7070023248112A3075C
:105AE00001002307F1009387218983D7070037E45A
:105AF0000400232611122318F1009387818283D793
:105B00000700414648082319F1007C4497F5FF1F20
:105B1000938585DB8297F1452800F5222312A102A7
:105B20007C442C002810794682973C44130561047C
:105B30001306900D8145829730109305700F014533
:105B4000EFD09FBB8320C112032481125561828054
:105B5000B7C7A55A01119387C7333EC483C7F188DD
:105B60003EC6B7F7070003C7070106CE22CCA547FC
:105B70006313F70001A01164930504F0930600106D
:105B80000146254597D0FF1FE780A0E73000930529
:105B900004F0A146294597D0FF1FE78080E683C522
:105BA000F18817650100130565B1EF308151F240AE
:105BB00062440561828001119165A14630009385A0
:105BC00005F02D4506CE97D0FF1FE78080E32247E2
:105BD000B7C7A55A9387C7336310F702B245176555
:105BE00001001305E5A0B335B000A387B188EF30FD
:105BF000414DF24005618280814517650100130522
:105C000065A1A3870188EF30C14B9937DDB7B7C7CE
:105C1000A55A79719387F7353EC6B7E70400FC476C
:105C2000AA8506D622D4414608088297B7F707000E
:105C300003C70701A5476313F70001A0116493058B
:105C400004E8930600100146254597D0FF1FE78022
:105C500040DB7000930504E8D146294597D0FF1F2B
:105C6000E78020DA17650100130505A9EF30A15977
:105C7000B25022544561828079719165D14670009D
:105C8000938505E82D4506D697D0FF1FE78060D79E
:105C90003247B7C7A55A9387F73517650100130533
:105CA000659F6310F702B7E70400FC4717F5FF1F75
:105CB000130585C141460C0882971765010013053D
:105CC000659BEF304154B25045618280B7F70700C1
:105CD00003C70701A5476313F70001A091654111B0
:105CE000930600100146938505E8254506C697D022
:105CF000FF1FE78000D1B240176501001305858DB5
:105D000041016F304150C16769768146FD17050634
:105D10001397060141836364B7003E858280330791
:105D2000D50003470700B98F214713F81700858373
:105D300063050800B18FC207C1837D171377F70F82
:105D40006DF78506F1B749C1A547054763FFB7065B
:105D500083471500034705003168A207D98F1397C1
:105D60008700A183D98FC207C1831308C85505478F
:105D7000639D0705411106C622C426C203442500BF
:105D8000914763FD8702930754006399F502A301CD
:105D9000C50021822302C5009304340091C6A302EA
:105DA000D500A1822303D5002A84A685A93F269485
:105DB0002300A4002181A300A4000147B240224493
:105DC00092443A854101828005473A858280B7C76F
:105DD000A55A01119387E7343EC42AC6B7F70700D6
:105DE00003C7070106CE22CC26CAA5476313F700D6
:105DF00001A091642A84938504EE93060010014665
:105E0000254597D0FF1FE780C0BF3000A14693858E
:105E100004EE294597D0FF1FE780A0BEA285176535
:105E200001001305A58BEF30C129EFF03FC9F24007
:105E30006244D2440561828001119165A14630001F
:105E4000938505EE2D4506CE97D0FF1FE78060BBFA
:105E50002247B7C7A55A9387E7346312F702B245C2
:105E6000175501001305057D2394B182C205C18138
:105E7000EF302125EFF09FC4F24005618280D147C9
:105E8000D145175501001305E57C2394F182EF30CD
:105E9000412303D58182253FC5B7011126CA06CE0D
:105EA00022CC93F71500AE849DC7AD67371700402D
:105EB0009387A7AA1CC3B7E70400BC4F13060019B9
:105EC000854503C56182829713C51400F240624480
:105ED000D2440561828093F72500638B0710976594
:105EE0000100938565852D464800EF30211283C55A
:105EF0001189854793C4240063EDB70299C983C70C
:105F0000E18891CF8545170500201305A5DDEF1029
:105F1000C02C13950401A3880188418145BF4165C8
:105F20000546970500209385E5DB7D15EFF05F8D35
:105F3000CDB7170400200344E4DA9707002083C795
:105F400077DA22045D8CAD67C2059387B755C181AE
:105F50006302F40863E48702A9679387A755630285
:105F6000F40883C7E1888DE741652E867D15970586
:105F70000020938525D7EFF0BF88A9A0B16793874C
:105F8000C755630EF400B5679387D755E31BF4FC40
:105F900017050020130505D5EF10202425A0054680
:105FA00017050020130505D4EFF03F8A83C7018948
:105FB00091EB4800EF30E12C93150501C1814800B9
:105FC000EFD04FA6A285175501001305E574EF30F9
:105FD000410F81B7170500201305C5D0EFF05F8F83
:105FE000D5B7170500201305E5CFEFF0FF8FD9BF18
:105FF00093F745000145E38B07EC175501001305A6
:10600000E572EF304120EF10003113C544007DBD33
:10601000411122C437E404005C5C06C6354697553E
:10602000010093852529176501001305A5B78297FF
:1060300001E9175501001305E570EF30C11C01A0FF
:106040008327041C82972A840545EF80E06EEF10B9
:106050008162EF10C140EF7070232285B24022446C
:10606000410182801567B71700401307575598C341
:10607000D8439D66558FD8C3D843FD76758FD8C356
:10608000D8431367F70FD8C335671307C7CC98C336
:10609000828041111305800406C622C426C24AC06C
:1060A00097C0FF1FE780805185457D55EFC01FEBEE
:1060B00085457D55EFC0FFF4371400408327840ADF
:1060C0008D451305002093E707202324F40AEFC031
:1060D000FFE8B7E40400EFD06F9AC8581309840CA6
:1060E0001304C40CEF30211217650100130585ABB2
:1060F000EF3061118327C4FF8545414593E70708C9
:10610000232EF4FEEFC0FFEF8D4513050008EFC00E
:106110005FEFEFD0CF890145EFD08F8C85450545E6
:106120008947238AF188EFD04F8D37070004B7E7FE
:1061300000E023A0E710EFD07F8BEFD05F9FC93D39
:10614000EFF07FA7EFF05FCFEFE0AFE28D450D6599
:10615000EFC03FEB170500201305C5C885671CC5B8
:1061600089672320250140C12326250100C95CC978
:1061700083A7841E829783A70408170500001305D0
:1061800005D282972383A182BC4C13060064854507
:106190008297C93D97C0FF1FE78000750145828047
:1061A000B7F7070003C70701A547AE866316F700D8
:1061B0009397450191C301A0AA850146254517D3B0
:1061C000FF1F670003844111B2862E86AA852D45E4
:1061D00006C697D0FF1FE780C082B240014541014B
:1061E00082809307000463E6C7021D71A2CC2A8453
:1061F000080886CE32C6EF207161B2461008A2852B
:10620000294597C0FF1FE780C07FF640664425619F
:10621000828039558280411126C2AE848D4522C4C8
:1062200006C62A84EFC0FFDDB717004099C803A552
:10623000C70C418D23A6A70CB240224492444101D1
:10624000828003A5870C418D23A4A70CF5B7834753
:10625000050003471500A207D98FC2076177C187E0
:10626000130727206397E7008345250037050400BF
:106270005DB782809387818918429C4383D645000D
:106280000345070083C5C700035646006396A50073
:1062900083D5E700638DD502011106CE2386A700C2
:1062A0002397D700B705CF00DC4B9385757D050795
:1062B0007D162EC2230001003AC42316C100231705
:1062C000D10099C30A858297F2400561828082805D
:1062D000DC4DDC4B91CBB7E70400904503A3870569
:1062E000914503C5C189028382806D713C083EC619
:1062F000B707E500232291103EC8AA843C083285E6
:10630000232611103ECA23248110232021112E8917
:10631000EF2050622A84975501009385E54A17457E
:1063200001001305E565EF20D159A285175501003D
:1063300013058559EF20F1582945EF20915CB705E9
:10634000CB009385757D6800EF10603EA2856800E4
:10635000EF20F053014781467000CA852685EF1073
:10636000805D15C52A84975501009385E54517453D
:1063700001001305E560EF20D154A28517550100F7
:1063800013054555EF20F1532945EF209157832000
:10639000C11003248110832441100329011051618D
:1063A00082809387818918429C43797122D406D6D2
:1063B0000348070083C807012A8483D64500035594
:1063C00046006396080183D82701638DD80223888D
:1063D000070105072399D7003708CC00DC4B1308C9
:1063E000787D3ACC1307F5FF42CA23080100231E2B
:1063F000E100231FD10099C7080832C62EC4829736
:106400003246A2452285D535B2502254456182805C
:106410006D713C083EC0B707E5003EC23C083EC473
:106420002326111023248110232291102317010009
:106430002318010023190100231A0100231B010066
:1064400097D7FF1F83D7470E99E3C167FD17231620
:10645000F10097D7FF1F83D7470D81EB9387818981
:106460009C439C43DC4783D7070017D4FF1F1304CA
:10647000A40B584C2317F10083574400484B2318B2
:10648000F10005ED975501009385053B1745010087
:106490001305054FEF20F142175501001305053B89
:1064A000EF2031422945EF20D1458320C11003243C
:1064B0008110832441105161828097D7FF1F83C7C9
:1064C000170789EBB7E70400BC5782975C4C23AAF7
:1064D0000700E1BFFD1797D6FF1FA38AF6040356F6
:1064E0000701834704014C470A85230BF100EF2085
:1064F0003038938781899C430147814688430A86C7
:106500006C00EF104043AA841DC997550100938584
:10651000A532174501001305A546EF20913AA6853F
:106520001755010013054533EF20B1392945EF20F8
:10653000513D584CB7E70400BC57484B79B797D743
:10654000FF1F83C7D7FEF5D7B7E70400BC4F104441
:10655000854503C5C189829789BF5C4EDC4BB9C7AD
:10656000B1C5411122C417450100130565412E84B0
:10657000975501009385852A06C6EF209134A285A0
:10658000175501001305852FEF20B1332945EF2062
:106590005137B7E704002244B24003A3870503C57F
:1065A000C189130640069145410102838280411151
:1065B00022C417D4FF1F130424F51C4C06C689C738
:1065C000DC4399C34C488297584CB7E70400BC574A
:1065D000484B82975C4CB240224423AA07004101F9
:1065E00082801387A182834707009306F00B8507FB
:1065F00093F7F70F63E7F6002385F1820345070061
:106600008280930700F8CDBF835745006384070E4F
:1066100001114AC817D9FF1F130909F152C4032AEF
:10662000C90106CE22CC03274A0126CA4EC656C24D
:10663000F15721EF1307D00DFD576368C704B7E981
:10664000040083A709072A841305860042054181B7
:10665000B284AE8A8297232AAA000325C9015C4925
:106660009DEF9755010093856519174501001305A6
:106670002531EF2011251755010013056528EF205E
:1066800051242945EF20F127DD57F2406244D244DE
:106690004249B249224A924A3E85056182809387E7
:1066A0004400B705CF002319F5009385757D3105AA
:1066B000EF10E0070325C901834564003105EF2091
:1066C000101D0325C9012686D6853105EF20501AF5
:1066D0007146A2854A85EF207113504409CA83A7E9
:1066E0008905854503C5C1898297814779BFEFF048
:1066F0003FD2E5BFFD573E858280411126C297D427
:10670000FF1F938464E2D84C22C437E404003C5455
:10671000484B06C68297DC4C0323C4052244B24092
:10672000924423AA070003C5C1898545410102831C
:10673000411126C2938481899C4006C622C44AC066
:10674000C9C7DC43D9C35CC12300B5002A8497556F
:1067500001009385E5051745010013056522EF202B
:1067600051162945EF20F1199C4023A4070023A2CC
:10677000070097D7FF1F938727D9DC4FDC4B81C7D2
:106780002955EFF0DFE297D7FF1F9387E7D9DC4F5A
:10679000DC4B91C39D3737E904008327C905894540
:1067A00003C5C18982978327C905914503C5C1895E
:1067B00082979C4003A3470163090300228522447A
:1067C000B2409244024941010283B24022449244C1
:1067D0000249410182800111328506CE22CC26CAAF
:1067E0002E84EF203015AA8497550100938585FFEC
:1067F000174501001305C518EF20B10C03078400ED
:106800000356640083554400A686175501001305FE
:10681000E508EF20110B2945EF20B10E97D7FF1F98
:1068200083C7E7CE639897000145EFF05FD88145B5
:106830000A85FD3DF2406244D244056182806D715B
:1068400023248110232611102322911093F7450051
:106850002E84638107123C083EC0B707E5003EC2A4
:106860003C083EC42317010023180100231901002E
:10687000231A0100231B010097D7FF1F83D7C7C826
:1068800099E3C167FD172316F10097D7FF1F83D740
:10689000C7C781EB938781899C439C43DC4783D79F
:1068A000070017D7FF1F130727C62317F100544F00
:1068B000835747002318F100DC4A95EF97550100F4
:1068C000938585F6174501001305850BEF20617F41
:1068D00017550100130585F7EF20A17E2945EF200C
:1068E0005102134544008320C110032481108324E6
:1068F00041105161828097D7FF1F83C757C125552B
:10690000BDC7FD1717D6FF1FA303F6C003D60601A8
:1069100083470701CC460A85230BF100EF20407521
:10692000938781899C4317D7FF1F1307E7BD97669D
:106930000100938666C688430A866C00EF00B07F2C
:10694000AA8445D197550100938505EE17450100AE
:1069500013050503EF20E176A68517550100130501
:10696000A5EFEF2001762945EF20A1792685EFF0EC
:106970001FC485BF93F725009DC3B7E70400BC473C
:1069800041468145280882972555EFF05FC22808C7
:106990009305F00FEFF0DFD913452400A9B793F763
:1069A00015000145A9D3EFF0BFA61345140025BF7C
:1069B0005C4D411106C688C323ACF188B7E70400DB
:1069C00083A70708170500001305A5E78297B240C3
:1069D000238EA18801454101828083C7918A85EF7A
:1069E000C16703D5C18AF9176307F502011193073F
:1069F000700F2316F100B7E7040083A7870D06CEBA
:106A000003C601836C00829701E58547A384F18A60
:106A1000F24005618280828083C7918A91E375BFCD
:106A2000828041119397050122C406C626C2C18700
:106A30002E8463D10706B7E70400FC5703C5018322
:106A40008297AA8415CD034705009307F0076300DA
:106A5000F7049306000B6310D70203474500631C3D
:106A6000F7008355850017550100130565FD23992F
:106A7000B182EF200165B7E70400BC5726858297F5
:106A80002165218DB2402244924441018280835588
:106A90002500D1BF93F715009DC3B7E7040083A776
:106AA000471A17D6FF1F130626AA97F5FF1F9385CF
:106AB000653803C50183829713451400E1B793F746
:106AC000250089CFB7E70400BC4F13060064894551
:106AD00003C501838297134524006DB793F78500A2
:106AE0009DC3B7E7040003A8871A1307401F83C795
:106AF0000183814613064006994503D5C18A029851
:106B00001345840041B793F745000145A5DFB7E47D
:106B1000040083A7041803D5C18A8297BC4C1306CE
:106B20000064914503C5018382971345440099BFD2
:106B300083D7C18A6390A7022397B18A2398C18A19
:106B40002399D18A2E8617550100130565F3BE855A
:106B50006F20215717550100130505F46F20A16A16
:106B600003574500011106CE22CC83D7C18A1755A1
:106B70000100130565F2631BF704C167F91723A62B
:106B8000F18A37E4040023A8018A7C4C894503C5B7
:106B9000018382977C4C914503C501838297DD4731
:106BA0002399F182A384018A83C7F18895C7854719
:106BB000A307F100832744171306F1008545130549
:106BC0005030829717550100130545E0EF20A1636F
:106BD000F24062440561828083C701891755010034
:106BE000130585E3E5F78547A307F10083274417DD
:106BF0001306F100854513055030829717550100A3
:106C0000130505DFE1B77D15954763E5A71817570D
:106C10000100130767D80A053A951C41011122CCDF
:106C200006CE26CABA972E8482871755010013050F
:106C300025E7EF20415D31A203C725009947631D79
:106C4000F7002E85EFF0DFF1834564001755010052
:106C5000130505E6EF20E14623870188175501005B
:106C60001305C5E6F9B703C7250095476315F70275
:106C7000C16703D7C18AF91703D5A5006305F702D9
:106C8000B7E7040083A7C7178297175501001305BC
:106C9000E5E4EF20415785472387F1881755010028
:106CA000130545E679B72396A18A83D7E500B7E4B3
:106CB000040009662397F18A83D70501130606901D
:106CC00003C501832398F18A83D72501A145239920
:106CD000F18ABC4C8297BC4C13060064914503C5F5
:106CE00001838297DD472399F182A384018AEFF023
:106CF000DFCE0356E4008355A400175501001305A9
:106D000025DFEF20013C41BF17550100130545E089
:106D10000DB783C525009147639AF502854717553E
:106D20000100130565E0A307F100EF20C14DB7E7AF
:106D3000040083A747171306F1008545130550305B
:106D40008297F2406244D244056182809947639EF3
:106D5000F5002285EFF0DFE0834564001755010060
:106D6000130505D5EF20E135E9BF9547639FF50091
:106D70008347140017550100130505DBE39B07EA61
:106D800017550100130505DC6DB5175501001305F6
:106D9000E5DBC9BF82806D71232481102326111089
:106DA00023229110328401CD89476306F5028320A6
:106DB000C110032481108324411051618280175532
:106DC0000100130565D9AE84EF20E143A285268535
:106DD000EFE08FD4E9BFB7E70400FC4728008297B3
:106DE00017550100130505D8EF20E14183478100C5
:106DF00029C01307000B638EE7001387A7051377DD
:106E0000F70F8D4663E7E602A2852800EFE0EFB0BA
:106E100079BF8547E3FD87F8834591001745010059
:106E2000130585F3B335B0002380B188EF206129C5
:106E3000BDBF03479100A207D98F35671307D75508
:106E4000638DE7066366F7022D671307B755638105
:106E5000E70631671307C7556386E70429671307F9
:106E6000A7556392E702A2852800EFE0FFA781B74C
:106E700039679306E7656383D70663E9F60013076E
:106E8000E7556388E704A285280099B73D67930614
:106E9000F755638AD7041307F766E396E7FEEFE03A
:106EA0003FBC31B70146A2852800EFE01F9A01B729
:106EB000A2852800EFE0DFA1DDBD8947E3F987EE79
:106EC0009305E4FFC205C1811305A100EFC08FB592
:106ED000F9BDA2852800EFE0FFA1D1BDA285280061
:106EE000EFE0DFAAE9B5EFE07FB2D1B5411122C4EE
:106EF00017C4FF1F13040467AA8617560100130660
:106F000026AB2285C14506C6EF20A13003574400B9
:106F100097C7FF1F938707662393E7000357640013
:106F20002394E700B240224441018280011106CE41
:106F300022CC6D3F37E404008327841417C6FF1F5B
:106F400013064662D545014582978327841793052A
:106F5000F1001305503082978347F100A1C7A307C2
:106F60000100832744171306F100854513055030AF
:106F700082978327441717C6FF1F1306A65FCD45C8
:106F80001305703082978547A307F10083274417C4
:106F90001306F1008545130550308297F240624494
:106FA000056182808327441717C6FF1F1306865C7E
:106FB000CD4513057030D5B7130101DE232C812098
:106FC00037E4040083270408232E1120232A91206C
:106FD0002328212123263121170500001305A5A40C
:106FE000829713890183994785442300A9002318B8
:106FF000F100975501009385A5A593074006174515
:1070000001001305E5972314F110230491009389DF
:107010002189EF20010B83D50900175501001305C5
:10702000E599EF20010A2945EF20A10D03D50900BC
:10703000EFF0DFEB83274417300085451305503010
:1070400082978327441717C6FF1F1306A652CD4504
:107050001305703082978327441717C6FF1F130646
:10706000664FB54513056030829783274417100893
:1070700089451305103182978327441730028945CB
:1070800013052031829783274415930500050D458C
:107090008297832744159305000511458297A30124
:1070A000910023029100230491002324011023085E
:1070B00001008327841630029145130570408297A2
:1070C00083278416130631008545130500408297F7
:1070D0008327841650008545130510408297832727
:1070E000841610088545130520408297832784164F
:1070F00030008545130550408297832704157D5540
:107100008297832744137D5582977D55EFC02FD8F2
:107110008327440C8297EFC0EFB58327841417C6EA
:10712000FF1F13062644D54501458297894713065C
:10713000700F814508082302F100EFB00F928D47D0
:107140001306700F814528022308F100EFB0EF907D
:1071500091472304F11093878183984383C74700A5
:107160003AC42306F100EFE07F95500085450545C0
:10717000EFC08FD810089305700F0945EFC0CFD727
:1071800030029305700F0D45EFC00FD730009545C5
:107190001145EFC06FD6C1671387C18AF9171CC3A9
:1071A000232207001385C182EFC02FD48327C41D7B
:1071B0001385018A82973C480345090085458297DB
:1071C0008320C1210324812183244121032901211A
:1071D0008329C1201301012282800111C16726CABF
:1071E00006CEAA8422CC03D5C18AF9176302F5041E
:1071F000A1C183D721838D46514763F6F600F51769
:107200001397070141836365B70237E404008327BE
:1072100084122E862315B10001478146ED458297E1
:107220002AC601ED1755010013058583EF10B17DC6
:10723000F2406244D244056182807C440356A1003E
:10724000A68582972C0003D5C18AEFC04FD56DD19A
:107250001755010013050582EF10F17A8327C41238
:10726000ED4528008297E9B7011106CE22CC2DC941
:10727000854717C7FF1FA304F72E97C7FF1F23815A
:10728000072E37E40400832784179305F1001305C4
:10729000503082978347F100A9CBA30701008327D1
:1072A00044171306F1008545130550308297832754
:1072B000441717C6FF1F1306E629B54513056030AE
:1072C00082978547A307F100832744171306F1002F
:1072D0008545130550308297F240624405618280F3
:1072E00097C7FF1FA38D072649BF8327441717C6DB
:1072F000FF1F13062626B54513056030E9BFC16799
:1073000003D5C18AF9176307F500B7E7040003A3A3
:10731000C7170283828001118547A30701002384D8
:10732000F18AB7E7040083A7471706CE1306F100DA
:107330008545130550308297F24005618280EFA2A7
:107340003FED2A8408452E89B28909C900C19705F5
:1073500000009385C5746105EF00810181447D5A69
:10736000EF10C00963C3A4048144EF10200A63C670
:10737000A40497F7FF1F9387A7AC9C43DC47B30790
:10738000F94091872302F400638109048327C9002F
:10739000B307F4409587A302F4001C4C89C79C47AF
:1073A00099C3228582976FA0FFE95C44139714006C
:1073B0008504BA972390470165B71C4813971400BA
:1073C0008504BA97239007004DB7832789000547A6
:1073D000B307F4409587A302F40083570400638E3B
:1073E000E7028DC309476384E7040D47E397E7FA93
:1073F000975701009387C7C91CCC97570100938703
:1074000027CA11A897570100938707901CCC97575C
:107410000100938767905CC849B79747010093873D
:10742000A77B1CCC974701009387077CEDB7975744
:1074300001009387A7CA1CCC97570100938707CBFD
:10744000D9BF85E1EFA27FDE004618448347940050
:1074500075839D8B6315F700EF00501C48C46FA027
:107460001FDF8280EFA2DFDA13893500C164420991
:107470004111AA890144F11413590901054A2EC684
:10748000EF00D077B2456346A400014541016FA0EB
:107490007FDB83A7090013171400BA9783D707006F
:1074A0006388B7006394970063742A010504C1BF21
:1074B0000545E9BFEFA2FFD4AA892E89328BB68495
:1074C0003A8ABE8AEF80204C55C12685EF103036AF
:1074D0008D4763E5A7007D556FA03FD683DB440051
:1074E000EF00D0772A84EF00B0789307740031441E
:1074F0003305850263C5A702EF005076EF001076D2
:107500002A84EF00F0769307740031443305850236
:1075100063CDA702EF0090749307450019A8EF0010
:107520003075330585021307F0179307C017E3572B
:10753000A7FC2D55E3C277FB63000B02D68652866B
:10754000A6854A85EFE0106341BFEF0070723305F6
:1075500085029307C5FFF1BF832749001385C90042
:1075600083D52700EFF01FF071F9B5B76955ADB7B6
:1075700097F7FF1F2398A78C97F7FF1F9387478CD8
:10758000904381470C463307F500420741836393DC
:10759000B70082805446139847008507C29623900F
:1075A000E600D5B797F7FF1F938787899C4303C5EC
:1075B0008700828017F5FF1F0355C5888280EFA2E0
:1075C000DFC6C1671387D7FF6307E5026368A700BB
:1075D000F117630EF50001456FA07FC71387E7FF22
:1075E000630EE500FD171D8D13351500F5B7EF404F
:1075F000003D7D15D5BFEF40801AE5BFEF40E01894
:10760000CDBFEFA29FC24111AA8401442EC6EF0054
:10761000F05FB2456346A400014541016FA03FC33E
:107620009C48131514003E9583570500E387B7FE69
:107630000504E9BF03485500814693F7F60F63E55B
:10764000070181473E858280584593975600BA9737
:1076500003D727006316B70003D70700E304C7FE6C
:107660008506E1BF8346450001479377F70F63E442
:10767000D700814711A81C45131657000507B2977C
:1076800003D60700E313B6FE3E858280EFA25FB803
:1076900093170501C18797EAFF1F938A6A7A63559A
:1076A000F00883A70A00C0479C4703570400198DC0
:1076B000420541816366F500014422856FA09FB8B1
:1076C00012052A94DDBFDC4713944900014A3E9419
:1076D000834744006341FA02014A834754006347E9
:1076E000FA028509C20993D9090183A70A009847BC
:1076F000E3EBE9FCD1B71C4413195A00A6853E9967
:107700004A85EFF01FF011ED050AD9B75C44131953
:107710005A00A6853E994A85EFF0BFEE19E1050AA9
:107720006DBFE30009FC51BFAA8481497DBFEFA270
:10773000DFAF1C452A8481E79307C5001CC51C44A4
:10774000231204001CC09307F00F63E9B70093F500
:10775000F50F2285EF10B0136FA07FAF9394050152
:10776000C167C18063F7F500A6852285EF10D015AB
:10777000E5B7C18193F5F50F2285EF105011A6856D
:107780002285EF101012C9BF97E7FF1F9387476B41
:10779000884382801C4599C797E7FF1F23A2A76AE9
:1077A000014582807D55828097E7FF1F9387476957
:1077B000984383474500484792073E958280EFA251
:1077C000DFA6617100451C183EC6B70780013EC8A0
:1077D0001C183ECA8357440002CE02D002CC231E9E
:1077E000F100834784002A8902D22301F1023C0878
:1077F0003ED402D6EFF05FFB835705002316F1025B
:10780000EF30706B2307A1025C4003556400F183E5
:1078100013F717008347F10252055181F99BD98F65
:10782000A307F102EFE0702639C5AA8403550500CD
:10783000EF80401683D704002AD26800231CF10091
:1078400083D72400231DF1001C4803D647008C4336
:10785000EF1010028347B400CA86174601001306D2
:1078600026318117A305F4006C004810EFE090303A
:107870005D616FA0DF9D2155E5BF1C45B1CF03C5FC
:10788000A700894613576500630BD7028D46630E28
:10789000D70285466300D702130740063305E50289
:1078A00003C7B700418B15CB83C7B700BD8B3355DA
:1078B000F54082801375F5031307803EC5B709674D
:1078C0001375F50313070771D1BF37270900137527
:1078D000F5031307077CD9B701458280EFA2FF9417
:1078E00003A98500630509048347B900AE8493F7B3
:1078F000070E91CF03459900930520030D810505DF
:10790000B305B50288446105EFF0B0320DA02E85B5
:10791000EFF0BFF62A8401CD11238325C900B307F8
:10792000B54063F887002E94B305A440E1FD6FA035
:107930001F928545C1BFEFA25F8F2A8403D5050042
:10794000011132C636C43AC22EC002CA02CC02CEDF
:10795000EF80400482452ACA22852ECCEFF0DFE476
:1079600003570500231EE100EF30F054A2463246D3
:107970009247230FA10036874C08B2862285014624
:10798000EFF05FB305616FA09F8CEFA21F8A61715A
:107990001C183EC6B70780013EC81C183ECA3C08EA
:1079A00000453ED4AA8402CC02CE02D002D202D636
:1079B000EFF09FDF8357050035592316F102EF30B2
:1079C000904F2307A10209C48357440091E721592E
:1079D0004A855D616FA0BF870355640052055181E0
:1079E000EFE0B00A2A8965D58347B40093F7070E04
:1079F00089C713058401EFF0502583574400231EE7
:107A0000F100834784002301F1025C400355090023
:107A1000D98313F7070883471102231CA10093F7AA
:107A2000F707D98FA300F10283572900231DF10026
:107A30005C40F18313F717008347F102F99BD98F5C
:107A4000A307F102EF7010752AD251D18347940039
:107A50006800139757008347B400FD8BD98FA305A7
:107A6000F4001C4803D647008C43EF106060A687E3
:107A7000174701001307C70F740005464C102685F1
:107A8000EFF05FA32A8929D58347B400A685FD8B33
:107A9000A305F400EFF09FE425BFEFA20FF98324C4
:107AA00085FE2A8441112685EFF03FDD834734FFB0
:107AB00093F7070E9DC32AC62685EFF05FD019C93C
:107AC000834734FFB245FD8BA309F4FE81C52285AF
:107AD000EFF0301641016FA08FF76DDD8327C4FFF3
:107AE0002685829765F9834734FF93F7070E81C790
:107AF0002285EFF09015032584FEEFF01FE9D9BF32
:107B0000EFA2AFEF9C4141112A8903C707008947C3
:107B10002E8493566700638CF6020D466382C6047A
:107B20009307F0076302F7022E85EF10A060AA8486
:107B30008149C16B130C490097E7FF1F93874730BA
:107B40009C43984763ECE90241016FA0CFEE03D755
:107B500045008547E3FAE7FE2E85EF108061C1BF3F
:107B600003D74500E3F2E7FE2E85EF10A05CAA8460
:107B70002285EF10805DC204C98C5DBFDC470355D0
:107B8000A900139A49003E9A93170501C187635DC6
:107B9000F00083570A006395A70263E57403832707
:107BA000CA00034D5A001DA0A1672167A98F1307C2
:107BB000F7EFE374F7FE63950900EFF05FA071FD46
:107BC00085099DBF83278A00034D4A00835DA90074
:107BD00003576900216A138BC7003AC6814A33CA2A
:107BE0004D01631E5D0197E7FF1F9387E7259C43C7
:107BF000E1DBA2866286814526858297D1B7A1679F
:107C00009387F7EF930C4BFF63F04703B2455A8518
:107C1000EFF05F8519CD03278B00104719CA104379
:107C20006380C4023107D5BFEE856685EFF07F9D86
:107C300071FD93861A0093FAF60F130B0B0255B7DA
:107C4000835644005C43E3EDF6F622853AC6EF1016
:107C5000603DA1679387D7042A8A035D44003247B9
:107C600063E897008347D90093E707F8A306F90074
:107C70001C4766852286E2858297C1670844FD1706
:107C8000337AFA00529508C02312A40115BF97E772
:107C9000FF1F9387E71A9843814715C3144781470D
:107CA00063FFD500939745004C47BE9519C903C79C
:107CB000550081476375E600DC451606B2973E85A0
:107CC000828003C745008147E37BE6FE16069C459C
:107CD000F5B7EFA2EFD3AA892E8A814497EAFF1F56
:107CE000938A0A1683A70A00984763E4E4006FA00A
:107CF0006FD5DC471394440001493E9413BB140034
:107D000083474400634BF900014913BB14008347C8
:107D10005400634FF9008504F1B7084493175900E4
:107D20005287DA860146A2853E9582990509C9BF28
:107D30004844931759005287DA860546A2853E9536
:107D400082990509E9B7EFA24FCE814517F5FFFFEC
:107D50001305255F97E7FF1F2396070EEFF07FF7C8
:107D60006FA0EFCE97E7FF1F9387870D9C4381CFCE
:107D7000EFA2AFCB814517F5FFFF1305855CEFF050
:107D80005FF56FA0CFCC8280EFA28FC837E40400EC
:107D90008327841241112315E100AE893289368A86
:107DA0003A8681460147ED45AA8482972AC621C5B5
:107DB0000356A100D285EF1061258327C413CE8519
:107DC00026858297058915C58327440D2314210133
:107DD00001462C00268582972A8401C9B7E7040052
:107DE00083A7C712ED4528008297228541016FA025
:107DF0006FC54944E5B76554CDBF5C41FD175CC113
:107E00008280EFA28FC2B7E70400FC5F829795479C
:107E10003305F50281450D816FA06FC3EFA2EFC05E
:107E2000B7E70400FC5F829795473305F5020D81A3
:107E30006FA0EFC1EFA26FBFB7E7040083A7870B66
:107E40000355050082976FA08FC0EFA20FBE0355A8
:107E500005003287AE8617B6FF1F0356C67797E533
:107E6000FF1F9385A5FEEFF03FF26FA04FBEEFA27C
:107E7000CFBBB7E7040083A7C71782976FA02FBDBA
:107E8000EFA2AFBAB7E7040083A7871397E5FF1FF8
:107E90009385C5FB829701456FA06FBBEFA2EFB83A
:107EA000B7E7040083A7C71F814517B5FF1F035518
:107EB000856E82976FA0AFB9EFA22FB7B7E7040026
:107EC00083A7871397E5FF1F938545F9829701459F
:107ED0006FA0EFB7EFA26FB5B7E7040083A7C71F86
:107EE000814517B5FF1F0355057182976FA02FB607
:107EF000EFA2AFB32E85EF600055EF60900D6FA03D
:107F00000FB5EFA28FB2EF60D0176FA04FB45C49EE
:107F1000E1175CC95CC583572501A1072319F5004A
:107F200083570501A1072318F5008280F147330527
:107F3000F50297E7FF1F938767F49C433E95828085
:107F40008D476317F60603D74600854763F2E706B9
:107F5000EFA2AFAD368536842E89EF10A01D39C152
:107F60008357440093140501C18063ED9702228575
:107F7000EF10401CFD14231294009307A002630E1F
:107F8000F5009307B0026301F50293079002631BAB
:107F9000F5002285EFC0B07E31A00146CA8522855A
:107FA000EF80000F6FA0AFAA2285EF001059DDBF50
:107FB000828097E6FF1F9386A6EC9C42014599CFED
:107FC0009843D44217E6FF1F232CE6EA6396D700B6
:107FD00097E6FF1F23A8E6EA1385C7FE8280EFA27B
:107FE000CFA4E9267144330585029145EF706062A4
:107FF00001E565556FA0AFA597E7FF1F23AEA7E684
:108000007526330585029145EF70A0607DD197E715
:10801000FF1F23A5A7E6592E97E7FF1F2398A7E484
:10802000712697E7FF1F2394A7E4974701009387E2
:1080300067B917E7FF1F232FF7E297070000938721
:1080400047ED17E7FF1F2325F7E2014565B7EFA2CC
:10805000CF9DAA8517E5FF1F130545E1EF106021AD
:108060006FA0EF9EEFA26F9CEFF07FFEEF10E0217C
:1080700097E7FF1F9387C7E09C4381CF1387C7FE15
:1080800009CB83D5C7FF17E5FF1F1305E5DFEFF029
:10809000403A6FA0CF9BEFA24F99EFF09FF119C923
:1080A000834785002A8493F7070499E70355E50081
:1080B000EFF05FFB6FA0AF998347C50093044501C4
:1080C00017E9FF1F1309C9DB85E3832709005CC992
:1080D00097E7FF1F23A697DA83274900E1FF97E779
:1080E000FF1F23A197DAF9B7FD172306F5006105F5
:1080F000EF60E07E8307840063CB0704834784003E
:1081000093E707F82304F400B7E704009C5F829725
:108110004205A94741813375F5028347840093F7EF
:1081200007FCC98F2304F4008347D4003E951C400C
:108130002318A40089CF984319CB8347C40050402B
:10814000814585073305F502420541810297832762
:1081500009005CC897E7FF1F23A497D28327490033
:1081600089E797E7FF1F23AF97D08347C400B9D3B0
:108170008355040117E5FF1F130505D1EFF0602BB0
:1081800015BFEFA28F8A97E7FF1F938727F59C47BC
:1081900001448583858B81EFAE84B2853A86EF10EA
:1081A00020142A8409C5EF10200B829408CC228564
:1081B0006FA0EF89EFA2CF8541112E8932C6AA891F
:1081C000712C324713060502CA8697050000938575
:1081D00025D617E5FF1F130565C9EFF09FFA2A841E
:1081E00029CD9304C50065261946AA852685EF008A
:1081F000306885452685EF00106517450100130599
:10820000259A4E95834505002685EF0050685C4809
:1082100031468145A1075CC85CC483572401E1173E
:108220002319F40083570401E1172318F4001C4CB0
:108230003E85EFA08F82A3042501228541016FA016
:108240006F80EF929FFE4111AA842EC632C4EF10B8
:108250000003004DB2452246834784000CC050C045
:1082600093F7F70393E707042304F40023180400AB
:108270002685EF00707E83479400A9462317A4004B
:1082800013D7370005073307D7029D8B85072306D1
:10829000F400A306E40083C70401D8488507230F30
:1082A000F7FE17E7FF1F1307A7BD5843232A040053
:1082B000930744011DEB17E7FF1F2325F7BC17E7C2
:1082C000FF1F232FF7BA17E4FF1F1304E4BB228517
:1082D000EFF0A00B1C44858B5D8D09E5814522855F
:1082E000EFF0201541016F909FF61CC317E7FF1FA9
:1082F000232AF7B8C9BFEF925FF397050000938573
:1083000065C40145EFF0DFBE01456F905FF4EF9269
:10831000DFF1EFF01FBF6F909FF38347C500A1E728
:10832000EF92BFF02A840355E500EFF05FD215C944
:108330008347840093F7F7FB2304F4001C4091C7A4
:10834000DC4381C74C4001458297EFF09FC617E59B
:10835000FF1F130565B3EFF0400F0355E400EFF086
:108360007FD06F90DFEE8280EF923FEC97E7FF1FA8
:10837000938707B197050000938525D217E5FF1F66
:10838000130585B023A0070023A20700EFE0507E6D
:108390006F90FFEB1C4D91CBDC4381CBEF92FFE85C
:1083A0008345070082976F909FEA828097E7FF1FBF
:1083B0009387C7AF9C4303C50700828097E7FF1FE1
:1083C0009387C7AE9C4303C51700828097E7FF1FC2
:1083D0009387C7AD9C4303C52700828097E7FF1FA3
:1083E0009387C7AC9C4303C54700828097E7FF1F74
:1083F0009387C7AB9C4303C53700828097E7FF1F75
:108400009387C7AA9C4303C55700828097E7FF1F45
:108410009387C7A99C4303C56700828097E7FF1F26
:108420009387C7A89C4303C57700828097E7FF1F07
:108430009387C7A79C4303C58700828097E7FF1FE8
:108440009387C7A69C4303C59700828097E7FF1FC9
:108450009387C7A59C4303C5A700828097E7FF1FAA
:108460009387C7A49C4303C5B70011E11D458280D3
:1084700097E7FF1F938787A39C4303C5C7008280AC
:1084800097E7FF1F938787A29C4303C5D70082808D
:1084900097E7FF1F938787A19C4303C5E70082806E
:1084A00097E7FF1F938787A09C4303D5070182802E
:1084B00097E7FF1F9387879F9C4303C5270182800F
:1084C00097E7FF1F9387879E9C4303D547018280D0
:1084D00097E7FF1F9387879D9C4303D567018280A1
:1084E00097E7FF1F9387879C9C4303D58701828072
:1084F00097E7FF1F9387879B9C4303C5A701828053
:1085000097E7FF1F9387879A9C4303C5B701828033
:1085100097E7FF1F938787999C4303C5C701828014
:1085200097E7FF1F938787989C4303C5D7018280F5
:1085300097E7FF1F938787979C438857828097E729
:10854000FF1F9387A7969C4303D5C702828097E7B6
:10855000FF1F9387A7959C4303D5E70219E11305F5
:10856000800C828097E7FF1F938747949C4303C545
:108570000703828097E7FF1F938747939C43C85B5D
:10858000828097E7FF1F9387E7918843828097E770
:10859000FF1F938767918843828019E17D55828010
:1085A000F5DE984265DFFDD917E7FF1F130707B314
:1085B0001847AA877155058B6319072203C5070061
:1085C0001547E37DA7FC03C737001305F0057D17AA
:1085D0001377F70FE364E5FC03C35700E30003FCE4
:1085E00083C86700E38C08FA03C777004945791709
:1085F0001377F70FE364E5FA03C7A70011481305E3
:10860000F7FF1375F50FE36BA8F803CE97000D483D
:108610001305FEFF1375F50FE362A8F803C8B70052
:108620006309080065181378F80F1305600DE367F8
:1086300005F703C5C700794879151375F50FE36F82
:10864000A8F403C8D7000D457D181378F80FE36729
:1086500005F503D80701930E401751184208135827
:108660000801E3ED0EF303C8E7007D181378F80F57
:10867000E36605F303C827017D181378F80FE36F4D
:1086800005F103C88700C54E75181378F80FE3E7A6
:108690000EF103D86701856E938EBEE06D18420817
:1086A00013580801E3EC0EEF03D847016D18420898
:1086B00013580801E3E40EEF03D887017918420844
:1086C00013580801E36C05ED03C8A7017D18137862
:1086D000F80FE36505ED03C5B7011D487D1513755A
:1086E000F50FE36DA8EA03C5D70171487915137535
:1086F000F50FE365A8EA03D5E7011308E00F7D1540
:1087000042054181E36CA8E803C507024948791591
:108710001375F50FE364A8E8C85301C937C83400DE
:108720005915130858BFE36BA8E603A8870237C59D
:108730003400130555BF5918E36205E717D5FF1F2D
:108740002324C57603C6050117D5FF1F2320F57620
:108750000545E375C5E403D82501D0493376060302
:10876000E31E06E203C61501E30A06E217D6FF1F61
:10877000232AB67283C5270001466387A50003C676
:108780001700F1453306B60283C707039305C002FD
:1087900072971A071307C70516031A979608469784
:1087A000B387B70241553E97329742074183636EC4
:1087B000E802EF929FA73685EF60D06FEFD0B0212F
:1087C0002A84EF80B01D2A94EFC090252A94EF7080
:1087D00040072A94EFF0BF802A94EF2050632A9438
:1087E000EF50406622956F909FA68280EF92FFA384
:1087F0004111A307A100EF80801E9305F10017052A
:108800000000130565B9EFF0CFCC014541016F9031
:108810001FA4EF921F9F17E4FF1F1304248C03284B
:10882000840079599368180097E4FF1F23AC148BD8
:1088300013781800631E0800BA84BE89368B328A0A
:108840002E89AA8AEFE01FD67D15269509E53159B4
:108850004A856F909F9EEFE0FFD47D152695A16716
:10886000E357F5FE97E7FF1F938747BE98433E8C7B
:10887000814B11C70145EFC0B03E933B15004A85BF
:10888000DA865686D285EF7070372A8911CD1C445E
:10889000F99B17E7FF1F2327F78483270C00CDDB05
:1088A000E3880BFA82976DB7268597E7FF1F23A908
:1088B0000782EFE0FFCB4146CE8517E5FF1F13058A
:1088C000658BEF00A174EFA070080325040BEFA0E7
:1088D000700A0545EFA070100545EFF03FF18DBF20
:1088E00097D7FF1F9387877F9C47858BD5C7EF92CC
:1088F000DF9317E5FF1F1305258697D7FF1F23AFCB
:10890000077C97D7FF1F23AD077C97D7FF1F23ABAB
:10891000077CEFE09033EF40C002EFE0F00AEFE0B9
:10892000700F97D7FF1F9387E7799C4381C7054551
:10893000EF60B03397D7FF1F938787629C4389C747
:1089400041657D15EF50A06BEFC0703AEFA0F000CD
:1089500097E7FF1F9387878D9C43139717016354F5
:108960000700EFC0A04597E7FF1F23A5078097E703
:10897000FF1F23A3078097E7FF1F23A1078097D737
:10898000FF1F23AF077EEFF09F984923EFF0AFBBA7
:10899000EFC080676F90BF8B828097D7FF1F938750
:1089A000E77388438280EF925F88EF60B07EEF705C
:1089B00080006F90DF89EF92BF852A8493041402B0
:1089C00001112E85B289A685214636C63A89EF0067
:1089D00081611DE1B24638082686CE8513059404D0
:1089E000EF40604321462C084A85EF00C15F1335F4
:1089F000150005616F901F850145E5BFEF92FF826D
:108A00009305450617D5FF1F1305854AEFE0702231
:108A10006F90FF83EF927F8141112EC6EFF00FC060
:108A2000B24588C141016F909F82EF926FFEAA8488
:108A30002E84EF605078AA8985452285892D83C7C9
:108A4000E4011389940899E313890403CE852285F0
:108A50003D2D2146930519022285192D97D7FF1F19
:108A60009387C7678C432285EF00E0682146938592
:108A700084022285F52B6F90EFFCEF928FF839710D
:108A8000EFC0E04E9305400645EDEF60D06F630EFA
:108A9000051097D7FF1F83C7674313B7170097D6F3
:108AA000FF1F2385E642014489CFC16417D9FF1F08
:108AB0001309C9629309400EFD14EFF03F98634813
:108AC000A408EFF0AFB54169B7290900096AFD7A3A
:108AD0002A8B81447D199389F97B130A0A71938A41
:108AE0008AC7EFF0BF9563D5A4041304400EB38783
:108AF000840217D7FF1F1307675E0324070B3E94FA
:108B00008357C4016386270918403307EB4063EAA3
:108B1000E900834744008507B3874703D697636915
:108B2000F706014681450945EFF0CFE8AA8B29E118
:108B3000EF20105A8547631FF504896593850571F9
:108B400017D5FF1F1305C536EFE0B00EA1A8B30778
:108B500034030327090BBA9703D7C70163089700AB
:108B600003C75700A38207002382E7000504B1B7BB
:108B70009305C5002285EFF05FEB5E852286973571
:108B8000010093852503EFF0CFEB5E85EF00E06FEA
:108B9000850481BF97D7FF1F938747549C478D83D8
:108BA000858BC1FF21616F904FE9014685450945DD
:108BB00002D002D202D402D6EFF0CFDFAA847DD158
:108BC000EFC0203A1389C4002A8481454A85C12117
:108BD0000C4041464A856929832944006388090875
:108BE0004E8502D802DA02DC02DEEF0081692ACE6D
:108BF000141005462C0808184ECCEF406019137568
:108C0000F50F2DE58355840093E525004A856D29F0
:108C100011460C104A85A929014697350100938514
:108C2000E5F92685EFF0EFE12685EF0000665C4070
:108C3000B5DB014685450D45EFF0CFD7AA843DD180
:108C400048401389C400EF00C1632AC64A85C5267F
:108C50003246636AC5004C404A8519290146814560
:108C60002685EFF00FDE26850D252DBF8355840068
:108C700071BFEF928FDB97D7FF1F938727469C47E3
:108C800019CD93E7870017D5FF1F1305652217D766
:108C9000FF1F2329F744EFE060786F904FDBDD9BE7
:108CA00017D7FF1F2320F744EF2090427DF517D5FB
:108CB000FF1F1305E51FEFE04079C5B7EF926FD4B2
:108CC0004169AA892E8AB28A368BBA8B814417DC15
:108CD000FF1F130CAC40930C400E7D19EFF00FF604
:108CE00063C4A40001442DA03384940383270C0B98
:108CF0003E948357C401638027055A87D6865286DF
:108D0000CE8513050403EFF01FCB11C523800B00A4
:108D100022856F908FD28347F40191CF5A87D686F0
:108D20005286CE8513059408EFF0FFC809C5854724
:108D30002380FB00F1BF850455B783574500638D41
:108D40000716EF92EFCC01112A84ED2619C585474D
:108D5000630AF50405616F90EFCEEFC040217DF905
:108D6000835744004947ED9BE396E7FEC1452285C2
:108D70004524AA842285F52E0357440002CE91474C
:108D80002A896317F700228539293C082ACC3ECE70
:108D9000EFC0201D5C55DDDF74084A86A6850545B9
:108DA00082974DBF03574400D147E3F5E7FA032A02
:108DB0000400C169014997DAFF1F938A2A32130B15
:108DC000400EFD19EFF08FE76344A90C2285032ABA
:108DD00004008D26A1452A8922851D2CAA8422857E
:108DE000D92614402A86AA8978082685CA85EFF0F4
:108DF000FFECAA8425D103C7F40189476315F70066
:108E00008347C101A1DB5546D28513856400EF007D
:108E1000E11F0145EF60103801C583D7C401B1EBF4
:108E200097D7FF1F9387872B9C47935519008589F8
:108E300013D73700058B11CB8983858B6397B700D8
:108E400001452EC6EFF0FFE2B2454E85EF60703C63
:108E50000346C1012A84937519002685EF7070318D
:108E600031C92685EF607037268511C00145EF6056
:108E7000D061EF20F0258547E31EF5EC83C7540051
:108E80001307F00FE388E7EC8507A382F400D9B558
:108E9000B304690383A70A0BBE9483D7C401638913
:108EA00037015546D28513856400EF00C11371D197
:108EB000050909BF5DDC5DBF8280EF926FB5EF6091
:108EC000902C11CDC164014417D9FF1F130909214A
:108ED0009309400EFD14EFF06FD6634AA40017D536
:108EE000FF1F1305E5FCEFE060536F90AFB533054E
:108EF00034038327090B3E958357C501638697008A
:108F000023120500EF60702D0504F1B797D7FF1FFE
:108F10009387C71C9C478D83858B99EBEF92EFB0AD
:108F200017D5FF1F1305C5F8EFE020526F902FB241
:108F30008280EF928FAF97050000938545B417D5D7
:108F4000FF1F1305E5F6EFE0A0426F904FB0EF92E0
:108F5000CFAD8841B7E70400BC5B05054205418100
:108F6000829709C585472300F50005056F902FAE50
:108F700083C7F5FF2E858507A38FF5FE828083C703
:108F8000F5FFFD1793F7F70FA38FF5FE99EBEF921F
:108F9000CFA9B7E70400BC571385F5FF82976F9000
:108FA0000FAB82801C41035745008D8FBA951CC1C1
:108FB0002312B5003E85828093D78500A205144117
:108FC000DD8D835745001387E6FF18C189072312FB
:108FD000F50013D685004111238FB6FEA38FC6FE80
:108FE0004101828018419307F7FF1CC18357450058
:108FF00085072312F500A30FB7FE82808357450033
:109000008D8F2312F5001C41BE950CC12E858280E8
:10901000AA8703D7470008410D8FAA952392E7003E
:109020008CC38280184108453305A740828083574E
:109030004500035765001D8F1C4108453385A74037
:109040003305A7408280EF924F9E41112EC62A849D
:10905000EFF0FFFDB2456373B50001A083574400F4
:109060000840BE952312B4003E9541016F902F9E9B
:10907000EF92AF9B41112E84B28532C6EFF0BFFC58
:109080003246A285EFF0907841016F904F9CEF92AD
:10909000CF992E848545EFF01FFB230085006F904C
:1090A0000F9BEF928F9841112317B1008945EFF084
:1090B0009FF98347E1002300F5008347F100A300F7
:1090C000F50041016F90AF98EF922F9693D78500EE
:1090D000A2054111DD8D2317B1008945EFF0BFF6E0
:1090E0008347E1002300F5008347F100A300F5006A
:1090F00041016F90CF95EF924F931397850193D7CE
:109100008501C166938606F0D98F13D78500758FC8
:10911000D98FA2053707FF00F98D4111DD8D2EC6CD
:109120009145EFF05FF26C001146EFF0306E4101B7
:109130006F90EF91EF926F8F1C41854503C407003C
:10914000EFF0DFEB22856F908F90EF920F8E1C4136
:109150004111894503C7070083C717002307E100B2
:10916000A307F100EFF09FE90355E10041016F9083
:109170000F8EEF928F8B1C414111894503C7070069
:1091800083C717002307E100A307F100EFF01FE7F3
:109190008357E100410113D58700A2075D8D420589
:1091A00041816F90CF8AEF924F880C4141112A8400
:1091B00011466800EFF0906591452285EFF01FE4BD
:1091C000B247C166938606F01397870113D58701CE
:1091D000598D13D78700758F598DA2073707FF0068
:1091E000F98F5D8D41016F908F861C45BE950CC136
:1091F0008280AE87944391E6584101EF0CC15CC177
:10920000828003C7570013671700A382E700B68761
:10921000D5B70CC3EDB7AA87084119CD1841D4437F
:1092200098C36313D500D8C32A87034657009376A3
:10923000160081E6232007008280944381CA8C4275
:1092400003A847008CC363930601CCC3799A14C367
:10925000A302C7003687D1BF1C45DC471D8DB777F9
:10926000DBB6938777DB09853305F502420541813B
:109270008280F147B385F50248452E958280834769
:10928000450085072302F5008280EF821FFA2A84B9
:1092900019E06F80DFFB83474400E5DFFD1793F79C
:1092A000F70F2302F400F5F71C4403D72700050746
:1092B0002391E700DC4399C3228582974C4889CDEE
:1092C00083475400898B99E71C4422859C479C4323
:1092D0009C478297232A04000040232004004DBFAE
:1092E000EF82BFF48357250041112EC691E7014458
:1092F000228541016F80BFF5035705008147F14684
:10930000E307F7FEB385D702404585072E948345D2
:10931000440008C4F5F5B247AA8481E7232A040073
:1093200009A81C456C0022859C439C43829748C831
:109330005DDD85472312F400B24723200400231883
:1093400004002319F4005C485CC483D72400FD1793
:109350002391F40071BFEF825FED97D7FF1F9387D2
:1093600027B7884323260500232405004105EFE0A5
:10937000C00D6F80DFEDEF825FEB17D4FF1F13048A
:1093800024B51C40411189CF9C472300B5002AC653
:109390005CC1EFF05FFC1C40DC4399C3324582970F
:1093A00041016F80DFEA034745001DEB584DAA8756
:1093B0007D550DCBEF827FE71CC3DC4797D6FF1F9F
:1093C00023A8E6B0F156130507012390D7009705AF
:1093D000000093858501EFD0B07901456F803FE7AC
:1093E0007D5582808280EF825FE401116146814574
:1093F0002800EF809FE697D7FF1F938767AD9C43B8
:1094000028009305F00FDC473EC6EFF0DFF605615C
:109410006F80FFE397D7FF1F938787AB9C43D847A5
:10942000A1679387C7026312F70A397106DE22DC4F
:1094300026DA80004AD84ED652D456D23285B2842B
:10944000EFF05FCFAA892685EFF03FD02318A4FC68
:109450002685EFF09FCF2319A4FC2685EFF0FFCEE1
:1094600083D744000A8A231AA4FC858393F7F70F55
:10947000230EF4FC8607BD0793F7073F3301F14045
:109480008A8A01498347C4FD6365F902CE851305C5
:1094900084FC232C54FDEFF01FEE5281130104FCD9
:1094A000F2506254D2544259B259225A925A21610E
:1094B00082802685EFF07FC993171900D69705099A
:1094C0002390A7001379F90F75BF828097D7FF1FEC
:1094D000938707A09C43D847A1679387A70263108F
:1094E000F70A397106DE22DC26DA80004AD84ED629
:1094F00052D456D23285B284EFF0DFC3AA892685D2
:10950000EFF0BFC4FD572318A4FC26852319F4FCF3
:10951000EFF0BFC383D744000A8A231AA4FC8583D3
:1095200093F7F70F230EF4FC8607BD0793F7073F69
:109530003301F1408A8A01498347C4FD6365F9021A
:10954000CE85130584FC232C54FDEFF0DFE252811D
:10955000130104FCF2506254D2544259B259225AB7
:10956000925A216182802685EFF03FBE9317190041
:10957000D69705092390A7001379F90F75BF82804C
:1095800097D7FF1F9387C7949C43D847A167890744
:109590006318F708397106DE22DC26DA80004AD823
:1095A0004ED652D456D232853289EFF0BFB8AA894E
:1095B0004A85EFF09FB9835749000A8A2318A4FC13
:1095C000858393F7F70F230CF4FC8607BD0793F709
:1095D000073F3301F1408A8A8144834784FD63E574
:1095E000F402CE85130584FC232A54FDEFF0BFD886
:1095F0005281130104FCF2506254D2544259B259C0
:10960000225A925A216182804A85EFF01FB49397C3
:109610001400D69785042390A70093F4F40F75BF28
:10962000828097D7FF1F9387A78A9C43D847A1675B
:109630009387E7046312F70A397106DE22DC26DA23
:1096400080004AD84ED652D456D23285B284EFF03A
:109650007FAEAA892685EFF05FAF2318A4FC26858C
:10966000EFF0BFAE231AA4FC2685EFF01FAE83D720
:1096700044000A8A2319A4FC858393F7F70F230E6D
:10968000F4FC8607BD0793F7073F3301F1408A8A50
:1096900001498347C4FD6365F902CE85130584FC47
:1096A000232C54FDEFF03FCD5281130104FCF25006
:1096B0006254D2544259B259225A925A216182803C
:1096C0002685EFF09FA893171900D69705092390D8
:1096D000A7001379F90F75BF828097C7FF1F938783
:1096E000277F9C43D847A1679387C7046310F70A75
:1096F000397106DE22DC26DA80004AD84ED652D4F2
:1097000056D23285B284EFF0FFA2AA892685EFF007
:10971000DFA3FD572318A4FC2685231AF4FCEFF0E1
:10972000DFA283D744000A8A2319A4FC858393F718
:10973000F70F230EF4FC8607BD0793F7073F3301AD
:10974000F1408A8A01498347C4FD6365F902CE85E9
:10975000130584FC232C54FDEFF0FFC1528113014B
:1097600004FCF2506254D2544259B259225A925ACD
:10977000216182802685EFF05F9D93171900D697AF
:1097800005092390A7001379F90F75BF828097C749
:10979000FF1F9387E7739C43D847A167DD07631BCF
:1097A000F702EF829FA8797132853284EFF09F989B
:1097B0002AC62285EFF07F992311A1022285EFF0BE
:1097C0007F97B2452300A1022808EFF0DFBA456178
:1097D0006F80FFA7828097C7FF1F9387676F9C43A7
:1097E000D847A16793878704631BF702EF82FFA323
:1097F000797132853284EFF0FF932AC62285EFF02B
:10980000DF942311A1022285EFF0DF92B2452300FD
:10981000A1022808EFF03FB645616F805FA3828008
:1098200097C7FF1F9387C76A9C43D847A167938751
:10983000A704631CF700EF825F9F01112800814598
:10984000EFF07FB305616F809FA0828097C7FF1FF5
:10985000938707689C43D847A16793875702631192
:10986000F702EF829F9C01113285EFF0BF8C230835
:10987000A10081452800EFF01FB005616F803F9D7A
:10988000828097C7FF1F9387A7649C43D847A1672F
:109890009387E702631FF702EF823F990111328538
:1098A0003284EFF09F8AAA842285EFF01F8A8547D1
:1098B00019E52285EFF01F884205B337A000280084
:1098C0008145231891003ECAEFF0FFAA05616F8021
:1098D0001F98828097C7FF1F9387875F9C43D84755
:1098E0009947631FF704EF825F9479713285328460
:1098F000EFF05F842AC62285EFF03F852310A10296
:109900002285EFF03F832301A1022285EFF09F82A1
:10991000A301A1022285EFF0FF812302A10222858B
:10992000EFF05F812313A1022285EFF0BF80B245E3
:109930002314A1022808EFF01FA445616F803F9116
:10994000828097C7FF1F9387A7589C43D847A1677A
:109950009387C703631FF704EF823F8D79713285C8
:109960003284EFF02FFD2AC62285EFF00FFE231080
:10997000A1022285EFF06FFD2311A1022285EFF0F5
:109980006FFB2302A1022285EFF0CFFAA302A1020E
:109990002285EFF02FFA2303A1022285EFF08FF941
:1099A000B245A303A1022808EFF0FF9C45616F8038
:1099B0001F8A8280EF827F8701112A84EFF08FF760
:1099C000AA842285EFF06FF82285EFF00FF8035795
:1099D00044008D4763F5E7002285EFF00FF72285FD
:1099E000EFF0AFF62800A685EFF0FF9805616F80D5
:1099F0001F8697C7FF1F9387A74D9C43D847A16732
:109A0000FD076319F700EF825F823285EFF09FFA5E
:109A10006F80FF83828097C7FF1F9387674B9C43AC
:109A2000D847A167E5076311F706EF821F807971B8
:109A300032853284EFF00FF02AC62285EFF0EFF086
:109A40002285EFF08FF02310A1022285EFF0EFEFD7
:109A5000520551812311A102228523020102EFF058
:109A60006FEDA302A1022285EFF0CFEC2303A10248
:109A70002285EFF02FECB245A303A1022808EFF0F6
:109A80009F8F45616F80AFFC828097C7FF1F9387D0
:109A900027449C43D847A1679387E7036319F700DE
:109AA000EF82AFF83285EFF0FFF06F804FFA8280DF
:109AB00097C7FF1F9387C7419C43D847A1679387E8
:109AC00047046314F702EF824FF6797132853284CE
:109AD000EFF04FE62AC62285EFF02FE7B2452808BF
:109AE000EFF07F8945616F808FF6828097C7FF1FF7
:109AF0009387073E9C43D847A167938787026316E5
:109B0000F702EF828FF2797132853284EFF08FE2C3
:109B10002AC62285EFF00FE2B2452300A1022808F1
:109B2000EFF07F8545616F808FF28280EF82EFEFEB
:109B30000111EFF02FE0AA852800EFF0DF83056127
:109B40006F80EFF097C7FF1F938787389C43D847F4
:109B5000A167D1076319F700EF822FED3285EFF08F
:109B6000FFFC6F80CFEE828097C7FF1F9387473639
:109B70009C43D847A167C5076319F700EF82EFEA56
:109B80003285EFF0BFFA6F808FEC828097C7FF1F9E
:109B9000938707349C43D847A167B9076319F70037
:109BA000EF82AFE83285EFF07FF86F804FEA828076
:109BB00097C7FF1F9387C7319C43D847A167AD075D
:109BC0006319F700EF826FE63285EFF03FF66F80A2
:109BD0000FE8828097C7FF1F9387872F9C43D84742
:109BE00089476310F702EF824FE40111328532C8D2
:109BF000EFF04FD4AA852800EFF0EFF705616F80F2
:109C00000FE5828097C7FF1F9387872C9C43D84717
:109C1000A1678D076317F702EF822FE101113285EB
:109C20003284EFF02FD113066100AA844C00228504
:109C3000EF20D00C2800A685EFF0EFF305616F80D0
:109C40000FE1828097C7FF1F9387C7289C4381CB72
:109C5000DC4391C7EF826FDD82976F804FDF828098
:109C6000EF82AFDC79713C08AE843ED2A165B707C4
:109C70000A002A843ED448103C08DD053ED636C48E
:109C800032C63AC2EFD0BFAA12474810BA85EFF0E9
:109C90000FC032464810B285EFF0AFC0A246481060
:109CA000B685EFF0CFBE501001478146A6852285CC
:109CB000EFD07FC845616F808FD9EF820FD7011138
:109CC0007C000329C501AE843ECAA165B707070021
:109CD0002A843ECC48087C00C5053ECEEFD03FA587
:109CE0008345D9004808EFF08FBA500801478146F4
:109CF000A6852285EFD03FC405616F804FD5EF82E6
:109D0000CFD283C7950093F7F707A384F500EFF050
:109D1000DFFA6F80CFD3EF824FD179713C08AE84E8
:109D20003ED2A165B70709002A843ED448103C08FA
:109D3000938545043ED632C636C4EFD05F9FA24617
:109D40004810B685EFF0AFB432464810B285EFF058
:109D50004FB5501001478146A6852285EFD0BFBD83
:109D600045616F80CFCEEF824FCC83C79500411104
:109D70002A8493F7F707A384F50032852EC6EFF007
:109D8000CFBC85672AC4637CF500EF50B040224603
:109D9000B24509E9114781462285EFF07FEC410188
:109DA0006F80EFCA01478346F501FDB7EF824FC6CA
:109DB00001113C003ECAB7070A003ECC3C003ECE33
:109DC00083C79500AA89328593F7F707A384F50026
:109DD0002E84EFF08FB785676371F504A165AA84BF
:109DE000938585044808EFD09F942685EF50903ADC
:109DF0002A891DE591454808EFF06FA9A685480816
:109E0000EFF02FAACA854808EFF06FA801478146F6
:109E10005008A2854E85EFD01FB205616F808FC2BA
:109E200081454808EFF0AFA603490902C1BFEF82A0
:109E30002FBE79711C103ECAB7070F003ECC404DB3
:109E40001C10AA84AE894808994532C636893ECE90
:109E5000EFD0FF8D32464808B285EFF04FA3630480
:109E60000902A5454808EFF00F9E2546CA85EFF088
:109E7000E019500801478146CE852685EFD0BFAB5B
:109E800045616F802FBC8355C4024808EFF06FA175
:109E90000355E402814515C185478545630FF500EB
:109EA000C167FD179305F00F6309F5007D15EF50AD
:109EB00020749305150093F5F50F4808EFF02F9DDA
:109EC000834504034808EFF08F9C8345140348083A
:109ED000EFF0EF9B835524034808EFF08F9C8355E8
:109EE00044034808EFF0EF9B69B7EF820FB483C7D4
:109EF00095008146014693F7F707A384F500EFF03C
:109F00001FF36F80CFB4EF824FB279713E841C1083
:109F10003ECA2E89B7070F00A1653ECCFD051C1077
:109F2000AA84480842C03AC23ECE36C432C6EFD0F8
:109F30001F8032464808B285EFF06F95A246480868
:109F4000B685EFF00F9612474808BA85EFF06F9587
:109F500002486304080291454808EFF0CF8E11468D
:109F6000A285EFF0A00A500801478146CA852685E0
:109F7000EFD07F9C45616F808FAD89454808EFF039
:109F80008F8C834704002300F50083471400A3004F
:109F9000F500D1BFEF82CFA783C7950001112A8AB0
:109FA00093F7F707A384F5003285AE8432C6EFF04D
:109FB000CF9932462A893285EFF0CF978567637F44
:109FC000F900AA894A85EF50F01C2A8419E9114743
:109FD00081464A86A6855285EFF09FC805616F804D
:109FE0006FA69387E9FF93F7F70F0547E368F7FE3E
:109FF0008347F50195E78947E382F9FE8346F4013B
:10A00000528501474A86A685EFF09FC5A167D9070B
:10A0100048083ECC230A010002CEEFF0BFC27DBF4C
:10A02000639CE7008947639CF90093071020231F76
:10A03000F500EF50901AD9B70947E391E7FC8D4737
:10A04000E39EF9FA2285EF50D03B97C7FF1F938715
:10A0500067079C4399E797C7FF1F938767F09C4367
:10A0600089C703D50400EF60300C231F040022854C
:10A07000C9B7EF828F9B01113C003ECAB7070B00A6
:10A080003ECC3C003ECE83C795002A89328593F7AB
:10A09000F707A384F500AE84EFF02F8B931705012B
:10A0A000C187635EF004A1652A849385E5024808B0
:10A0B000EFD0EFE7A2854808EFE0BFFE97C7FF1F8C
:10A0C000938707EA9C439DEF01449375F40F48087A
:10A0D000EFE0FFFB9355844093F5F50F4808EFE060
:10A0E0001FFB9355044193F5F50F4808EFE03FFA45
:10A0F000014781465008A6854A85EFD0DF83056178
:10A100006F80EF94416585460546A2857D15EF3049
:10A1100070675DD95105EFD04027130440063344E2
:10A12000850265B7EF826F900111B70706003EC642
:10A1300083C7950021642A8993F7F707A384F50064
:10A14000AE8428009305A4040AC40AC8EFD02FDE09
:10A15000300001478146A6854A85EFD0CFFDEFE06C
:10A160002FF813049404480822CC230A010002CEDD
:10A17000EFF05FAD05616F808F8DEF826F89C164F5
:10A180002A89014497C9FF1F938949F5130A800260
:10A19000FD14EFE0AFAB6345A40001456F808F8AEB
:10A1A000B307440303A7C90ABA9703D70700630696
:10A1B000970083D72700638427010504D9BF05458D
:10A1C000F1BFEF82EF842A8A2E8999C123A005006E
:10A1D0008149814497CAFF1F938A0AD0614BEFE0FF
:10A1E0002FAD63C5A4004E856F80CF853384640393
:10A1F00083A70A003E948357040099E7630409008B
:10A20000232089008504E1BF4146D285130544001F
:10A21000EFE0705D65F9A289F5B7EF727FFF3971E4
:10A220007C083ED4B7070A003ED67C083ED883C7D8
:10A2300095002A8A328593F7F707A384F5002E89C3
:10A2400032C6EFE09FF085676373F5063246AA8455
:10A250003285EFE03FEE8547AA8963EAA704A1654E
:10A26000938585042810EFD08FCC2685EF5080721F
:10A270002A8429E191452810EFE07FE1A685281086
:10A28000EFE03FE2CE852810EFE07FE00147814616
:10A290003010CA855285EFD00FEAA1679387770403
:10A2A00048183EDC230A010202DEEFF0BF9921616B
:10A2B0006F705FF981452810EFE07FDDA6852810DB
:10A2C000EFE03FDE97C7FF1F938707189C4391C7B6
:10A2D000228563870900EFB0600C8345040265B7EF
:10A2E000EFB0200BDDBFEF72BFF283C795004111C5
:10A2F000AA8993F7F707A384F5003285AE84328AE2
:10A30000EFE0BFE48567637BF5022A89EF50806840
:10A310002A84914621C18347F50105476383E702FB
:10A3200091C70D47636EF702AD462DA09305050357
:10A3300003250A004146EFE0104B1DE141016F701B
:10A340007FF09305950803250A004146EFE0B049E8
:10A35000814679F94A86A6854E85EFF0DF9BF9BFE5
:10A3600083250A0013059408EF60600119C1C146F6
:10A37000D5B797C7FF1F9387E7D49C4399E797C743
:10A38000FF1F9387E7BD9C4389C72285EF60A054D8
:10A3900079FD8547A30FF4002285EF80B05D22850B
:10A3A000EF50A0634E8581464A86A685EFF0BF96A2
:10A3B000A1679387570448003EC42302010002C6E8
:10A3C000EFF05F88A5BFEF72DFE383C7950041110F
:10A3D000AA8993F7F707A384F50032852E89B28AFC
:10A3E000EFE0BFD685676370F50CAA84EF50805A02
:10A3F0002A841DE9416B014A97CBFF1F938B0BCE3B
:10A40000130C400E7D1B19A833048A0383A70B0B82
:10A410003E948357C401638D6703050AEFE00F8202
:10A42000E344AAFE954639A88357C5016392970273
:10A430009305050303A50A004146EFE0D03A99468B
:10A4400011E181462686CA854E85EFF0DF8CA1A8F2
:10A4500083A50A0013050403EF507072C1467DF115
:10A460002285231E9400EF80F0502285EF50E056A5
:10A4700097C7FF1F938747FD9C438DCB23000402A2
:10A480002285EFA090614E8581462686CA85EFF031
:10A490009F88A1679387070448003EC423020100F8
:10A4A00002C6EFF02FFA41016F703FD989472300B0
:10A4B000F402D1BF397106DE22DC4AD8800052D4C2
:10A4C00056D25AD026DA4ED65ECE2E8A32892A8BC2
:10A4D000EFD0DFF30605710541998A8A3301A14067
:10A4E000232224FC231404FCEFD05FF283479A005C
:10A4F0000605350593F7F7072315A4FCA304FA0016
:10A500004A85232624FCEFE05FC493170501C18729
:10A510006340F0025681130104FCF2506254D2549D
:10A520004259B259225A925A025BF24B21618280FF
:10A53000AA844A85EFE07FC1AA894A85EFE0FFC07F
:10A54000A1659385C5022A89130544FCEFD02F9E8F
:10A550002685EFD0AF93854501C94A86CE85EFD0D9
:10A560006F8DAA8B15ED8945130544FCEFE03FB2D2
:10A57000A685130544FCEFE0DFB2CE85130544FC4D
:10A58000EFE03FB2CA85130544FCEFE09FB10147FD
:10A590008146130644FCD2855A85EFD0CFB99DBFC2
:10A5A0008145130544FCEFE09FAEA685130544FCEE
:10A5B000EFE03FAFCE85130544FCEFE09FAECA85C8
:10A5C000130544FCEFE0FFAD8144EFD03FE4E3D05E
:10A5D000A4FC83A70B0113971400BA9783D5070037
:10A5E00089C5130544FCEFE0DFAB8504F9BF797141
:10A5F00006D622D44AD000184ECE52CC56CA26D205
:10A600005AC8AE893289AA8AEFD05FE0060569058B
:10A6100041990A8A3301A140232A24FC231C04FC0B
:10A62000EFD0DFDE83C7990006052D0593F7F70706
:10A63000231DA4FCA384F9004A85232E24FCEFE00B
:10A64000DFB093170501C187634FF00052811301FA
:10A6500004FDB250225492540259F249624AD24A3D
:10A66000424B45618280AA844A85EFE01FAEA16516
:10A670009385A5022A89130544FDEFD04F8B2685CB
:10A68000EFD0CF80854519C5CA85EFC0BFFD2A8BA5
:10A690000DE98945130544FDEFE07F9FA68513056D
:10A6A00044FDEFE01FA0CA85130544FDEFE07F9F46
:10A6B00001478146130644FDCE855685EFD0AFA7EE
:10A6C00071B78145130544FDEFE07F9CA685130516
:10A6D00044FDEFE01F9DCA85130544FDEFE07F9C1C
:10A6E0008144EFD0BFD2E3D5A4FC83270B0113979D
:10A6F0001400BA9783D5070089C5130544FDEFE020
:10A700005F9A8504F9BFEF725FB283474500404D01
:10A71000D5E7FD574DC0834694000947636DD708C0
:10A720000346B400854663E8C6088306E40063C4B4
:10A7300006085C45F9562390D70097B7FF1F83C7DB
:10A74000E77999E3A304E40097C7FF1F9387478144
:10A750009C4381E78947A306F40097C7FF1F9387AF
:10A76000A7CE9C4381E789472306F40097050000A4
:10A7700093854505AA8413050401EFC0703FFD577A
:10A78000231AF40281471CDC014897B7FF1F23A35B
:10A79000877497B7FF1F93872774232E040304C081
:10A7A0008043EFD0FFD061463306C5028145228544
:10A7B000EF70BFAA81473E856F707FA9FD57E5BF47
:10A7C000EF72BFA62A8403554502EF50A01C09E58D
:10A7D000231E04006F70BFA78357E401E5DF9305D4
:10A7E00004FF1715010013052577EFB01063DDB7DF
:10A7F000EF72BFA32E89A16541119385E5032A84D9
:10A8000036C432C6BE843AC2EFC07FF212472285F8
:10A81000BA85EFE0DF8732462285B285EFE07F8898
:10A82000A2462285B685EFE0DF87630D09009145DA
:10A830002285EFE05F811146A685EFE0207D410192
:10A840006F70FFA089452285EFE0EFFF83C704000A
:10A850002300F50083C71400A300F500CDB7EF7205
:10A86000DF9C83C79500444D054793F7F707A38402
:10A87000F5001C42411183C70700636DF7042E8465
:10A880002A8985CC03C7D4006309F70217B7FF1FD5
:10A890001307076D184301CFA386F400EF80902BB8
:10A8A00083C7D40089E741657D15EF30407583D7B4
:10A8B0002403918B99C3EFB0B0624A85A285EFF073
:10A8C000CFBFA167C10748003EC42302010002C6F2
:10A8D000EFF04FB741016F709F97EF721F9503D74D
:10A8E00045008D47AA8441112E8432892E8563ED5F
:10A8F000E700EFE09F85AA85230009002685EFC0C9
:10A900007FD641016F70BF94EFE03F842AC6228555
:10A91000EFE0BF83B24585472A862300F9002685EC
:10A92000EFC05FD1F9BF397106DE22DC26DA800084
:10A930004ED652D456D24AD85AD05ECEAE89B284C0
:10A94000AA8AEFD0BFAB06051305250241990A8AF2
:10A950003301A140232224FC231404FCEFD01FAABE
:10A9600083C7990006054D0593F7F7072315A4FC47
:10A97000A384F9002685232624FCEFE00FFD93171E
:10A980000501C1876340F0025281130104FCF250BB
:10A990006254D2544259B259225A925A025BF24B33
:10A9A00021618280AA8B03AB0400EFC03FCE35E962
:10A9B00083D7440001498544F11793B71700A301D9
:10A9C000F4FC834734FCA165BDC79385E5041305FA
:10A9D00044FCEFC0DFD5A685130544FCEFE02FEB68
:10A9E000DE85130544FCEFE0CFEB834734FC1146D2
:10A9F00091E30946DA85130544FCEFE06FE78144F3
:10AA000063080900416B7D1BEFD05F9F63C8A40200
:10AA100001478146130644FCCE855685EFC0BFF141
:10AA2000A5B7A685130634FCEFF03FEB9334150071
:10AA30002A89860479B79385C50451BF8327C90045
:10AA400013971400BA9783D5070063866501130531
:10AA500044FCEFE00FE5850445BFEF728FFA797192
:10AA60001C103EC4B7070F003EC61C103EC883C76B
:10AA70009500AA8A328593F7F707A384F500AE897B
:10AA80003284EFE08FEC93170501C1876350F00625
:10AA90002A8A2285EFE06FEB2A895285032B040076
:10AAA000EFC0DFBE39E58357440081440544F11708
:10AAB00093B71700A303F10083457100DA8722875B
:10AAC000CA8652862800EFF0BFD201478146300087
:10AAD000CE855685EFC03FE6A1679387D703480828
:10AAE0003ECC230A810026CEEFF0CF9545616F70F2
:10AAF000CFF4A28513067100EFF03FDEAA8409446B
:10AB000045DD3544E30A55FB4A85EFF00FE70D4478
:10AB100045D50144EFD09F8E634BA400C16B014427
:10AB2000FD1BEFD0BF8D634EA400154471B7DC440C
:10AB300013171400BA9783D707006381270305040E
:10AB4000D1BFD84493171400BA9703D707006319ED
:10AB50007701239027012685EF80C0540144A9BFC7
:10AB60000504C1B7EF72CFEA83C7950041112A8A65
:10AB700093F7F707A384F50032852E893284EFE03E
:10AB8000CFDC93170501C187635BF004AA89228596
:10AB9000EFE0AFDB2311A1004E85832A0400EFC054
:10ABA000FFAE29E18357440085440144F11793B770
:10ABB0001700A300F1000348110003572100D687B6
:10ABC0005285CE862686CA85EFF0EFB3A167F107DE
:10ABD00048003EC42302910022C6EFF0AF86410137
:10ABE0006F704FE6A28513061100EFF01FCF2A8485
:10ABF000894471D18357210011678544BA97C207F0
:10AC00001167C1831307F7EFE367F7FA97B7FF1FE1
:10AC10009387474B9C4391C7854513052100EF401F
:10AC2000300E8355210022858144EFC09F9D41D580
:10AC3000231005002285EF808048B5BFEF726FDCDE
:10AC400083C7950041112A8B93F7F707A384F5007A
:10AC500032852E8A3284EFE04FCF93170501C187EA
:10AC60006359F004AA8A2285EFE02FCE2A895685FF
:10AC7000832B0400EFC09FA121E18357440081444E
:10AC80000544F11793B71700A301F1000348310001
:10AC9000DE875A854A87D6862286D285EFF0AFA610
:10ACA000A167ED0748003EC42302810026C6EFE0FD
:10ACB0007FF941016F706FD8A28513063100EFF064
:10ACC000DFC1AA84094479D19167CA97C207116785
:10ACD000C1831307F7EF0544E36AF7FACA85EFC0AB
:10ACE0005F92014445F58149EFD04FF263DBA90043
:10ACF000984893971900BA9703D7070015E7239050
:10AD00002701EFD0AFF01544E382A9F82685EF8044
:10AD1000003B97B7FF1F9387E73A9C430144BDD799
:10AD20004A85EF4040769DB785097DBFEF724FCED3
:10AD300079713E847C083EC82E8AB7071400A1654D
:10AD40003ECAE5057C08AA89080836C4428932C68D
:10AD5000BA8AC6843ECCEFC09F9DCA850808EFE042
:10AD60000FB332460808B285EFE0AFB3A246630ED8
:10AD700009029D450808EFE00FAD1D468145EF70C3
:10AD8000CFCD63870A0691450808EFE0CFAB1146A7
:10AD9000A685EFE0A027100801478146D2854E85A1
:10ADA000EFC07FB945616F70EFC9B6850808EFE065
:10ADB0004FAF1C400808D8439355C7018589120737
:10ADC0005183B205D98DEFE0CFAD1C40080883C593
:10ADD0008700EFE0CFAB1C40080883C5A700EFE079
:10ADE0000FAB1C40080883C59700EFE04FAA51BF86
:10ADF00089450808EFE02FA583C704002300F5006C
:10AE000083C71400A300F50079B7EF726FC083C742
:10AE100095004111AA8993F7F707A384F5003285BD
:10AE2000AE843284EFE06FB293170501C187635798
:10AE3000F0042A89032A0400EFC05F8519E98357CB
:10AE400044000548F11793B71700A307F1008146A6
:10AE500021A81306F100A285EFF03FA81DC11C45F3
:10AE60009DC383D6470001480347F100930785003F
:10AE7000D2884A86A6854E85EFF05FEB41016F7060
:10AE80006FBC0948E9B71D48D9B7EF726FB8657153
:10AE90005C083EC4B7077B013EC65C083EC883C75A
:10AEA00095002A8A328593F7F707A384F500AE89C7
:10AEB000EFE04FA88357E100C5C389452800EFC0E4
:10AEC0001F8781452800EFE08F9CEFC0FF8B97B76D
:10AED000FF1F938767579C4317B4FF1F0344040069
:10AEE000AA843334800099C31364240097B7FF1FEA
:10AEF000938707079C4399C31364440097B7FF1FC8
:10AF00009387471C9C4399C31364840083D5040032
:10AF100028000149EFE0EF9883D524002800EFE0F6
:10AF20004F9883D544002800EFE0AF97EFD00FC9CA
:10AF300093150501C1812800EFE0AF96A285280096
:10AF4000EFE02F969C44636CF90001478146300086
:10AF5000CE855285EFC03F9E59616F70AFAEDC4425
:10AF60001314490028003E94EFE06F8C834744009F
:10AF70000347540089070607BA978607E36EF5FC76
:10AF8000835524002800814AEFE0AF9183454400B7
:10AF90002800EFE0CF8F834554002800EFE02F8F8B
:10AFA0008347440063C9FA00814A8347540063CF52
:10AFB000FA00050941BF1C4413975A002800BA97AC
:10AFC00083D50700850AEFE0CF8DD9BF032BC400DE
:10AFD00093975A0028003E9B83552B00850AEFE08B
:10AFE0004F8C83550B002800EFE0AF8B7DBFEF72D5
:10AFF000CFA35C4993E717005CC9EF8020336F70E3
:10B000000FA5EF728FA22E848145EFF08F9B05C1B3
:10B0100083570500FD172310F50009C48357250049
:10B020002310F400EFF0BFFC01456F704FA23145D3
:10B030006DDC23100400D5BFEF728F9D83C7950090
:10B0400041112A8A93F7F707A384F50032852E89E8
:10B050003284EFE08F8F93170501C187635EF004A0
:10B06000AA89C1452285EFD0BFFA2A8B4E85832A53
:10B070000400EFC0AFE121E5835744002311010034
:10B080000544F11793B71700A300F100814403486A
:10B09000110003572100D6875285CE862286CA85A5
:10B0A000EFE07FE6A1679387170248003EC42302C2
:10B0B000810026C6EFE01FB941016F70AF981306FB
:10B0C0001100A285EFF07F81AA8409E52311010018
:10B0D000094475BF930521005A85EFF09FF283570D
:10B0E00021002A84CDD797B7FF1F9387A7FD9C43E4
:10B0F00091C7854513052100EF408040835521000D
:10B1000026853144EFC0EFCF59D1231005002685A5
:10B11000EF70F07A0144A5BFEF722F9141112E8993
:10B120006C00AA8402C6EFF0CF8909CD0357050051
:10B1300005072310E500EFF09FEB81473E854101B5
:10B140006F70EF903247954775DBCA852685EF20F3
:10B15000D008C147E34405FE3244854741462310E9
:10B16000F40083570900A685130544002311F40059
:10B17000EFD0D0692285C1B7EF728F8983C7950060
:10B180004111AA8A93F7F707A384F5003285AE89A7
:10B190003284EFD09FFB93170501C187635EF004F3
:10B1A0002A8AC1452285EFD0BFE6AA845285032BA7
:10B1B0000400EFC0AFCD21E5835744002311010007
:10B1C0008544F11793B71700A300F1000144034829
:10B1D000110003572100DA875685D2862686CE8550
:10B1E000EFE07FD2A1679387070248003EC42302A5
:10B1F000910022C6EFE01FA541016F70AF84A285C8
:10B2000013061100EFF06FED2A8409E52311010008
:10B21000894475BF268593052100EFF0FFEFAA84CE
:10B220005DF5835521002285EFC0AFBD4DF1014989
:10B23000EFD0CF9D635DA900184893171900BA9706
:10B2400003D707001DE7035721002390E700EFD045
:10B25000EF9B6302250397B7FF1F9387A7E69C43E5
:10B2600089C703552100EF4000222285EF70306529
:10B27000B9BF050975BF954499BF05C19307F00F84
:10B28000630FF500C547630CF5009307F5FF05450F
:10B290003315F50042054181828001458280416578
:10B2A0007D158280B9E1EF625FF8034506033284C1
:10B2B000EFF0BFFC9305803EB305B502C205C18126
:10B2C00091C90357E402854763F6E70013050401BB
:10B2D000EFC020168357E40241677D176385E700BE
:10B2E000FD172317F4026F609FF68280EF627FF1F3
:10B2F000004283C79500444D0349140093F7F707B4
:10B30000A384F50083470400220911673369F9001B
:10B31000A167B347F90041112A8BAE8A63ECE70CB1
:10B32000834724001307C00EB91793F7F70F637113
:10B33000F70E03473400C14763ECE70C8347440032
:10B340001307E00793C707086373F70A834984006C
:10B3500083477400A209B3E9F900856763F9F90826
:10B36000034A6400834754004E85220A336AFA0078
:10B37000EF40406245C123962403834B3400137A87
:10B38000FA00239A3403238874032399440393898E
:10B390000401631A090023A60402239804024E85BF
:10B3A000EFC0A00A1DA0034924004A85EFF0FFEC7E
:10B3B0002397A402834744004E85A388F402E381C7
:10B3C0000BFEE30F09FCEFC06005EF70907981463A
:10B3D0000146D6855A85EFE09FA5A167938797031D
:10B3E0003EC423020100480002C6EFE0BF854101D0
:10B3F0006F60BFE48544A2862686D6855A85EFE035
:10B400001FA3A167938797033EC423029100E1BF66
:10B41000BD44D5B79144C5B7EF629FDF01111C0849
:10B42000404D3EC2B7070F003EC41C083EC62A89E5
:10B43000AE89EFC01F9D585C1C5C634CB70A6394D7
:10B44000E50063E8A70A3385A740B3B7A700B305B3
:10B45000B7401306803E81469D8DEFD0407B93140C
:10B460000501C180A1659385C5034800EFC02FACDD
:10B4700081454800EFD0BFC1835504044800EFD098
:10B480005FC2835524044800EFD0BFC1814599C8ED
:10B49000C167FD179305F00F6386F4002685EF4022
:10B4A0002015AA854800EFD09FBE0355440481456E
:10B4B00011C9C167FD179305F00F6305F500EF4053
:10B4C0002013AA854800EFD09FBC83456404480040
:10B4D000EFD0FFBB834574044800EFD05FBB500042
:10B4E00001478146CE854A85EFC0EFC405616F6094
:10B4F0007FD5814485BFEF625FD383C7950093F703
:10B50000F707A384F500EFF03FF16F605FD4EF62BF
:10B510003FD083C795004111404D93F7F707A384AF
:10B52000F5002A8A3285B284AE89EFD01FC22A8BF9
:10B530002685EFD09FC12A892685EFD0BFBF9317FC
:10B540000B0163CA0702E177CA97C207C18311677B
:10B5500063E3E70293070910C207C1831307B00F23
:10B56000637BF70093170901C187AA8A6348F0003B
:10B57000C54763FA570141016F60DFCCEFC08F838D
:10B58000E31B25FFF5B763060B0263040902814440
:10B5900063870A02B7077F0023106405231124057F
:10B5A0007CC05685EFF07FCD9304803EB3049502B6
:10B5B00039A0B7077F00232004047CC081440355D1
:10B5C0002404EFB0101095CCEFC0BF83269593D71D
:10B5D000F44133379500AE97BA9708DC5CDCCE8532
:10B5E0005285EFF07FE399E023220404A16793875B
:10B5F000B70348003EC42302010002C6EFE08FE417
:10B600009DBF814701481CDC232E0403C9BFEF62A4
:10B61000DFC1EFC0FFE9E1473305F5029145EF30A7
:10B62000507FE55711C597B7FF1F23A7A78A81470A
:10B630003E856F60DFC1854717B7FF1F2300F78A7C
:10B640008280EF629FBE97B7FF1F9387A7888043D2
:10B650002DC083570404639EA70483572404639A70
:10B66000B7043689B284EFC0CFF95C5C63C3B7041A
:10B670006395B7001C5C63EEA7028347640463F321
:10B68000F400A6872303F4048347740463F397004C
:10B69000A687A303F4048357440441677D17638599
:10B6A000E70085072312F4043C4481C7CA85268538
:10B6B00082976F60DFB997B7FF1F9387A7819C437D
:10B6C000014599C303C587008280EF621FB601114F
:10B6D000B70707003EC683C79500584D0AC493F7C5
:10B6E000F7070AC8A384F5002A89AE8401CB1C425F
:10B6F00083C707002304F700EF70D045216493054A
:10B7000054022800EFC0AF82EFF0FFFAAA852800AC
:10B71000EFD0FF97300001478146A6854A85EFC0EC
:10B720008FA113044402480822CC230A010002CE50
:10B73000EFE04FD105616F609FB1EF621FAF011164
:10B740007C003ECAB70707003ECC7C003ECE83C7D4
:10B7500095002E84AA8493F7F707A384F500A165CA
:10B76000938555024808EFB09FFCEFF0DFF4AA85FF
:10B770004808EFD0DF91500801478146A285268511
:10B78000EFC06F9B05616F609FAC97A7FF1F93870A
:10B7900067749C43094599C303C59700828097A7A6
:10B7A000FF1F938727739C43094599C303C5D7009F
:10B7B000828097A7FF1F9387E7719C43014599C338
:10B7C00003C5A7008280EF62BFA40111B70708007C
:10B7D0003EC683C79500404D0AC493F7F7070AC8D1
:10B7E000A384F5002A89AE8429C01442854703C783
:10B7F000060063EEE7068347940009468149638E9D
:10B80000C700B307F740A304E400B339F00083C7CF
:10B8100016002305F400EF70F03303572403058B63
:10B8200009C763840900EFA0B06B2164930584020B
:10B830002800EFB0DFEFEFF05FF5AA852800EFD02A
:10B840001F85EFF01FF7AA852800EFD05F8401471E
:10B8500081463000A6854A85EFC0EF8D130474023F
:10B86000480822CC230A010002CEEFE0AFBD0561FB
:10B870006F605F9DEF627F9B01117C003ECAB7073E
:10B8800008003ECC7C003ECE83C795002E84AA845F
:10B8900093F7F707A384F500A1659385850248080F
:10B8A000EFB0FFE8EFF07FEEAA854808EFD02FFE5B
:10B8B000EFF03FF0AA854808EFD06FFD5008014730
:10B8C0008146A2852685EFC00F8705616F603F988E
:10B8D00097A7FF1F938707609C43014599C303C542
:10B8E000B7008280EF627F940111B70707003EC660
:10B8F00083C79500404D0AC493F7F7070AC8A3848D
:10B90000F5002A89AE8405C41C42054783C7070099
:10B91000636AF7040347B400630BF700A305F40060
:10B92000EF7050238347B400A9C3EFD00FD921642F
:10B930009305B4002800EFB09FDFEFF07FF9AA85F0
:10B940002800EFD0CFF4014781463000A6854A8514
:10B95000EFB07FFE2904480822CC230A010002CE62
:10B96000EFE04FAE05616F609F8EEFD02FDAC1B769
:10B97000EF62BF8B01117C003ECAB70707003ECCC7
:10B980007C003ECE83C795002E84AA8493F7F707E8
:10B99000A384F500A165AD054808EFB05FD9EFF0CD
:10B9A0003FF3AA854808EFD08FEE50080147814643
:10B9B000A2852685EFB03FF805616F605F8997A784
:10B9C000FF1F938727519C43094599C303C5C700AF
:10B9D0008280EF629F8501117C00AE843ECAA16522
:10B9E000B70707002A843ECCD1057C0048083ECE2C
:10B9F000EFB0FFD3EFF0BFFCAA854808EFD02FE9E6
:10BA0000500801478146A6852285EFB0DFF2056127
:10BA10006F60FF83EF627F8183C7950093F7F7071D
:10BA2000A384F500EFF0FFFA6F607F82EF624FFEB4
:10BA300083C795000329C501411193F7F707A38434
:10BA4000F5001C4283C90700854763EC370597B7AB
:10BA5000FF1F9387679F9C432E84AA8495C7EFF0AE
:10BA60001FF689476302F502630009028347C90094
:10BA7000638C370123063901EF70D00D83572903FA
:10BA8000898B99C3EFA0D0452685A285EFF07FF47E
:10BA9000A167CD0748003EC42302010002C6EFE0C3
:10BAA0006F9A41016F600FFA97A7FF1F9387874234
:10BAB0009C431D4599C303C5E7008280EF62EFF602
:10BAC0000111B70707003EC683C79500584D0AC449
:10BAD00093F7F7070AC8A384F5002A89AE8405C73F
:10BAE0001C4283C7070093968701E18663C806045A
:10BAF00085466385D7048346E7006386F6002307FF
:10BB0000F700EF70300521649305E4002800EFB0E2
:10BB10001FC2EFF07FF9AA852800EFD04FD7014769
:10BB200081463000A6854A85EFB0FFE0350448081D
:10BB300022CC230A010002CEEFE0CF9005616F60B6
:10BB40000FF1EF628FEE01117C003ECAB7070700CC
:10BB50003ECC7C003ECE83C795002E84AA8493F70A
:10BB6000F707A384F500A165B9054808EFB03FBC0D
:10BB7000EFF09FF3AA854808EFD06FD15008014736
:10BB80008146A2852685EFB01FDB05616F602FEC33
:10BB9000EF620FE8AA84014417A9FF1F1309C933F4
:10BBA000E149EFC0FF906344A400014519A83305A3
:10BBB0003403832709003E9583572500639597003A
:10BBC00011056F602FE80504E9BF032E85006304AB
:10BBD0000E1017A3FF1F1303E34E03230300631587
:10BBE00003002943639A060E03234E0163150300E5
:10BBF0001D436393070EEF62CFE0C689428A3E89F8
:10BC0000BA8AB684328BAE8B2A84A1E903554E00E2
:10BC100009E501431A856F604FE2A167A98F11679B
:10BC200063F7E700EFF0DFF68145EFF08FBD0844E2
:10BC3000B70700E05841F98F18455CC1B707001FEE
:10BC4000F98F1CC55C4981C76105EFB01000E38224
:10BC500009FC2285EF70606E6DBF3285EFA0E06257
:10BC60000D434DD91C44116703D54700A167A98F27
:10BC700063F7E700EFF0DFF18145EFF08FB80323C2
:10BC8000840093164B01D1828347B30003566300AF
:10BC90008588FD8BA305F300FD777D8E558EFD769F
:10BCA000FD16B204F18E83274301C58E2312730162
:10BCB0002313D3002304530123052301A3044301C9
:10BCC000D9D72285EFB07FBBAA850844B5DD6105D1
:10BCD000EFB02076ADBF1D431A858280EF624FD34F
:10BCE0000569AA84AE89328A0144FD5A7D19EFC0E4
:10BCF000EFF06345A40001456F60CFD4D84493179B
:10BD00001400BA9703D70700631B3703239057012A
:10BD100063050A002685EF70E0389C448DC383D705
:10BD20006700B3F72701639C3701D2880148814738
:10BD300001478146014681452685EFF01FE905044C
:10BD40007DB7EF62EFCC79711C103EC4B7070F00CE
:10BD50003EC61C103EC883C79500AA8A328593F759
:10BD6000F707A384F5002E893284EFD00FBE931716
:10BD70000501C1876350F006AA892285EFD0EFBC88
:10BD80002A8A4E85032B0400EFB05F9039E5835774
:10BD9000440081440544F11793B71700A303F10051
:10BDA00083457100DA872287D2864E862800EFE02D
:10BDB0003FA4014781463000CA855685EFB0BFB722
:10BDC000A1679387F70348083ECC230A810026CE5B
:10BDD000EFD05FE745616F60EFC6A2851306710083
:10BDE000EFE0BFAFAA84094445DD5285EFE0EFB82C
:10BDF0000D445DD50546D2852685EFF03FEE2A84B9
:10BE000045B7EF628FC283550700034627004111F3
:10BE10002A842E8532C62EC4EFE02FB611C53246D5
:10BE2000A2452285EFF09FEB41016F604FC2EF62A8
:10BE30004FBD83C795004111AA8A93F7F707A384E2
:10BE4000F5003285AE893284EFD02FB0931705010B
:10BE5000C1876357F008C1452A8A2285EFD04F9BDE
:10BE60002A8D2285EFD06FAE2A892285EFD08FAC44
:10BE7000930705F893F7F70F1307E007AA8B637191
:10BE8000F7062285EFD00FAB2A8C2285EFD08FAA40
:10BE9000AA8C5285032B0400EFB04FFF29E583578E
:10BEA0004400231101008144F11793B71700A30048
:10BEB000F100054403471100835621009387840055
:10BEC0005685DA8822885286CE85EFE03FE6A16764
:10BED000E90748003EC42302810026C6EFD09FD662
:10BEE00041016F608FB513061100A285EFE0FF9E40
:10BEF000AA8409E52311010009446DBF93052100BF
:10BF00006A85EFF06FA12A8455F583552100935679
:10BF1000C9001316490185486688E2875E87858ACD
:10BF200051822685EFF07FCA2A8469B7EF626FAD30
:10BF300083C7950041112A8B93F7F707A384F50077
:10BF40003285AE893284EFD04FA093170501C187A7
:10BF50006352F0082A8A2285EFD02F9FAA8A228571
:10BF6000EFD0AF9E2A892285EFD0CF9C930705F8AA
:10BF700093F7F70F1307E0072A8C637DF7042285F8
:10BF8000EFD04F9BAA8C2285EFD0CF9A2A8D528575
:10BF9000832B0400EFB08FEF29E1835744008544E1
:10BFA0000144F11793B71700A301F10003473100D3
:10BFB000930784005A85DE882688D6865286CE85E9
:10BFC000EFE0DFD68D4748003EC42302910022C631
:10BFD000EFD05FC741016F604FA6A2851306310005
:10BFE000EFE0BF8F2A84894471D19356C90013169C
:10BFF000490185486A88E6876287858A5182D685A5
:10C00000EFF0BFBCAA845DB7EF628FA02A8981449C
:10C010000144617A916A17ABFF1F130BAB0AEFC0A3
:10C02000EFBE63C5A40022856F60CFA183270900FE
:10C0300093991400CE9703D50700330745014207B3
:10C0400041836362570311CD03270B0009C7854560
:10C050003E85EF30E04A832709000504CE97239000
:10C06000070085046DBFEFF0BFB283270900050408
:10C07000CE972390070075D58145EFE09FF8D5B79F
:10C08000EF620F9983C7950041112A8A93F7F7074A
:10C09000A384F50032852E893284EFD00F8B93175D
:10C0A0000501C1876354F004AA89832A0400EFB014
:10C0B000EFDD21E18357440085440144F11793B734
:10C0C0001700A301F10003483100D68752850147CC
:10C0D000CE862686CA85EFD01FE3A167F507480004
:10C0E0003EC42302910022C6EFD0DFB541016F604C
:10C0F0006F95A28513063100EFE02FFE2A84894454
:10C1000079D197A7FF1F9387E7FB9C4381CB044915
:10C11000EFC0CFAFAA852685EF30803E130504011E
:10C12000EFF09FEE2285EF609079814469BFEF6266
:10C130004F8D83C795004111AA8A93F7F707A3840F
:10C14000F5003285AE89328423110100EFC0FFFF74
:10C1500093170501C187635CF0042A8AC1452285D3
:10C16000EFC01FEBAA8B5285032B0400EFB00FD258
:10C1700031E18357440085440144F11793B7170018
:10C18000A300F1000348110003572100DA87568508
:10C19000D2862686CE85EFD01FD7A1679387270248
:10C1A00048003EC42302910022C6EFD0BFA941013E
:10C1B0006F60AF88A28513061100EFE00FF22A84AA
:10C1C000894469D197A7FF1F9387C7EF98433E899A
:10C1D00001CB0449EFC08FA3AA852685EF304032FA
:10C1E00013050401EFF05FE2EFC04FA2954459D967
:10C1F000930521005E85EFE03FF2AA8441F51C48DB
:10C200000357210022852390E700EF60506B8327BE
:10C210000900ADDB03552100EF30E026A5B7EF5252
:10C220005FFE83C795004111AA8A93F7F707A3849D
:10C23000F5003285AE893284EFC03FF193170501D6
:10C24000C1876359F0042A8A2285EFC01FF02A892A
:10C250005285032B0400EFB06FC321E183574400E4
:10C2600085440144F11793B71700A301F100034877
:10C270003100DA8756854A87D2862686CE85EFD06A
:10C280009FC8A167F90748003EC42302910022C657
:10C29000EFD05F9B41016F505FFAA285130631001A
:10C2A000EFE0AFE32A84894479D19167CA97C20746
:10C2B0001167C1831307F7EF8544E36AF7FA97A77D
:10C2C000FF1F938727E09843BE8B01CB0449EFC043
:10C2D000EF93AA852685EF30A02213050401EFF025
:10C2E000BFD2EFC0AF92954459D11C4822858144FA
:10C2F00023902701EF60B05C83A70B00ADDB4A857C
:10C30000EF306018ADB7EF525FF22A844105B28476
:10C31000EFF09FCF01C52285EF60705A814601463C
:10C32000A6852285EF70C00B1C4C89C7DC4799C3DA
:10C33000228582976F50BFF197A7FF1F938787B918
:10C340009C43014599C313850701828097A7FF1F6E
:10C35000938747B888438280EF523FED9317C6001A
:10C36000DD8DC2054111C1812A8432C6EFC07FD361
:10C370003246228511829375F60FEFC05FD14101DD
:10C380006F50FFECEF52DFE879713C083ED2B707FF
:10C390000C003ED43C083ED683C79500AE842A8963
:10C3A00093F7F707A384F500A1659385350448103A
:10C3B000EFB0EFB7C165FD15014417AAFF1F130ABF
:10C3C000EAD1930A400EAE892E8B2EC6EFC00F879E
:10C3D0004205931704014181C183B24563E3A7027B
:10C3E000C167FD176385F5004810EFC09FCB501063
:10C3F00001478146A6854A85EFB0EFD345616F506E
:10C400007FE43307540383270A0BBA9703D6C70187
:10C4100063083601638835014810EFF0FFF3DA85D1
:10C42000050465B7B285EDBFEF52BFDD79717C08B9
:10C430003EC8B70711003ECA7C083ECC83C79500B2
:10C44000AA89328593F7F707A384F5002E89EFC0F8
:10C45000DFCF8567637EF502A165AA848905080898
:10C46000EFB0EFAC2685EF30E052133415000A042C
:10C47000A2850808EFC0BFC1A6850808EFC07FC22B
:10C4800035C0014781461008CA854E85EFB0AFCA56
:10C4900045616F509FDAB30754030327CA0ABA975E
:10C4A00003D70700631A970003D62700638A650342
:10C4B0000808EFF07FEADE8505042EC6EFB01FF90D
:10C4C0004205931704014181C183B245E3E5A7FC0E
:10C4D000C167FD17E387F5FA0808EFC09FBC55B7A1
:10C4E000B285D9BFC165FD15014417AAFF1F130A04
:10C4F000EABE930A80022E8BAE8BC1B7EF52FFD2F9
:10C5000018418347170083460700A207D58FD2073B
:10C51000D1832390F50083472700034717008D45FB
:10C52000A207D98F91832310F600EFC03FAD6F5063
:10C530001FD2EF52FFCDC164014417A9FF1F130999
:10C54000E9B993098002FD14EFB05FF06345A400E0
:10C5500001456F503FCF330534038327C90A3E9509
:10C5600083570500E38797FE0504F9BFEF525FCAC2
:10C570002A8AAE89B284B68AEF30C04109E5914774
:10C580003E856F503FCC2A894E85EF9010502A840B
:10C59000638A0A048D476DD503570500C547E3112B
:10C5A00047FF0347F9018546AD47E31BD7FC8347A7
:10C5B000450091CB4146A6855D05EFC0D02281475D
:10C5C00061D1AD4775BF130965012302E500CA8536
:10C5D0002685EF10202D15CDA547E3830AFA230207
:10C5E000040079BF11CD83570500E39A47F941460E
:10C5F000A6851905EFC0301F814759D1994749B722
:10C600004E85EFF01FF32A8495473DD91309550055
:10C610007DBF4146A6852310440123113401130533
:10C620001900EFC0B01E2285EF60B03C814789BF82
:10C63000EF52BFBF79717C003ECCB7070A003ECEF7
:10C640007C003ED083C79500B2842E8493F7F70711
:10C65000A384F5001306A1002A892C002685EFF09B
:10C66000FFE9A16528088D05EFB06F8C90408355D8
:10C67000A100035581008546EFF05FEFAA84AA85EB
:10C680002808EFC0DFA00356A100835581002808C9
:10C69000EFF09FCC300801478146A2854A85EFB074
:10C6A0008FA9854748103ED42302910202D6EFD0CD
:10C6B0006FD945616F50BFB9EF523FB779717C00B8
:10C6C0003ECCB7070A003ECE7C003ED083C7950023
:10C6D000B2842E8493F7F707A384F5001306A10014
:10C6E0002A892C002685EFF07FE1A16528088D05B9
:10C6F000EFB0EF8390408355A10003558100814640
:10C70000EFF0DFE6AA84AA852808EFC05F980356F9
:10C71000A100835581002808EFF01FC430080147AD
:10C720008146A2854A85EFB00FA1481023029102ED
:10C7300002D402D6EFD00FD145616F505FB1EF52F6
:10C74000DFAEEFF0BFE26F509FB09797FF1F938768
:10C75000A77888438280EF525FAD8357250041114F
:10C76000AE842A842307B10017F5FFFF1305A569DE
:10C770006C002316F100EFB0CFD581C42285EF60A5
:10C78000B02DFD572310F400130620028145130538
:10C790005400EF509FAC41016F507FABEF525FA749
:10C7A00079717C003ECCB7070A003ECE7C003ED0BB
:10C7B00083C79500AA89AE8493F7F7073285A384CF
:10C7C000F5001306A1002C00EFF05FD303558100A4
:10C7D0001144EF30201C15C10355A1000144EF9016
:10C7E000D02A01CD035705008357810045446316C5
:10C7F000F7008545EFF03FF60144216993053900C4
:10C800002808EFA0DFF2A2852808EFC05F88035652
:10C81000A100835581002808EFF01FB430080147BC
:10C820008146A6854E85EFB00F9148104AD4230269
:10C83000810202D6EFD00FC145616F50BFA0EF5209
:10C840003F9D9797FF1F9387E7682A8488432E8927
:10C8500015C1035745038357C401631DF700232601
:10C860000502231805024105EFA0303E63040900CC
:10C87000EF60302F814497A9FF1F93892986130AFF
:10C880008002EFB0BFBC63CCA4029797FF1F9387D1
:10C89000276D9C4389C70355C401EF10407663059B
:10C8A00009002285EF6050031306400E8145228562
:10C8B000EF50BF9AFD57231EF4006F50BF98338589
:10C8C000440383A7C90A3E95035705008357C40153
:10C8D0006315F700CA85EFF01FE885045DB7EF52D6
:10C8E0003F9383C795004111AA8993F7F707A38463
:10C8F000F5003285AE84EFC05F8585676370F5040F
:10C900002A89EF302009014411C983D7040031443A
:10C91000638627018545EFF09FF201444E85A2868C
:10C920004A86A685EFD02FBFA167938717044800DA
:10C930003EC42302810002C6EFD0CFB041016F5048
:10C940007F90EF52FF8C9797FF1F9387A7588043E4
:10C950001DCC0145EFA0E05681470148C1641CDCB5
:10C96000232E0403232004041799FF1F13090977BA
:10C9700001449309400EFD14EFB05FAC634BA4007B
:10C9800081451705000013054598EFB08FB46F502F
:10C990007F8B330534038327090B3E958357C501ED
:10C9A000638597008545EFF09FE90504F1B793573C
:10C9B000050113D78700A380F50093170501C183F4
:10C9C000A1832380E5002381F500A381A500828057
:10C9D000EF52BF852300050083C71500A300F500B3
:10C9E00083C725002301F50083C73500A301F500A7
:10C9F00083C745002302F50083C75500A302F50055
:10CA000083C7650093059500A30305002303F50084
:10CA1000230405003285EFF09FF96F505F83EF52DA
:10CA20002FFF4111E9541DC995C993F9C5FF2E8403
:10CA30002A89AA84338AA900B7EA040063149A02F7
:10CA40000D88854401CCB7E704009C5F82972AC615
:10CA500022866C0033053901EFC0405B2685410119
:10CA60006F504FFE83A78A039104829793170501A5
:10CA7000C183A183A38EF4FE93570501238FF4FE97
:10CA8000A183238EA4FEA38FF4FE4DBF63E0D502E5
:10CA9000EF52AFF9B28741113686BE8536C6EFC078
:10CAA000E056B246410136856F506FFA81463685B1
:10CAB0008280838705001387F5003D05FD8793F786
:10CAC0007708834607007D158606B58FA300F5001D
:10CAD0006307B7007D17834717009D83DDB782800A
:10CAE000EF52AFF4B7E7040083A7070932872A861D
:10CAF0003A858297133515006F506FF501CD814748
:10CB000099C9EF528FF24146EFC0405085473E85AC
:10CB10006F50EFF381473E8582801DC5EF52EFF0E5
:10CB2000414681452A84EF504FF341468145130524
:10CB30000403EF508FF20147C1672322040438C871
:10CB40007CC805456F50AFF001458280814729CDF3
:10CB5000A1CDEF528FEDB2842E8913068005814559
:10CB60002A84EF508FEFCA8524C42685EFF01FF981
:10CB7000414681452285EF504FEE3044A285228503
:10CB8000EFF01FF693040401A2852685EFF07FF2F3
:10CB9000A68513050402EFF0DFF12285EFF0FFF721
:10CBA00085473E856F50AFEA3E858280EF524FE663
:10CBB0004111E9541DC995C993F9C5FF2E842A89ED
:10CBC000AA84338AA900B7EA0400639444030D8859
:10CBD000814401CCB7E704009C5F82972AC6228675
:10CBE0006C0033053901EFC06042268541016F506A
:10CBF0006FE583A78A039104829793170501C18388
:10CC0000A183A38EF4FE93570501238FF4FEA18325
:10CC1000238EA4FEA38FF4FE4DBF71CDEF524FDFE4
:10CC2000B28401E605456F50EFE12A842E89014563
:10CC3000FDD93C487848B3E6E700F5D69386F7FF80
:10CC4000B3B7F6007D17032A4404BA9734C87CC8EA
:10CC5000630F0A04C14913050A03B38949412295A8
:10CC6000637B3601B2862E86A685EFF03FE27C40DC
:10CC7000BE9464C045BFCE862E86CE85EFF01FE100
:10CC8000C114D2944E9923220404A287930604016E
:10CC900003C7070003C607038507318FA38FE7FE8D
:10CCA000E398F6FE3044A2852285EFF07FE32699D3
:10CCB000C1493306994063EA9900ADD4A686A6859A
:10CCC00013050403EFF09FDC6DB78147B306F40052
:10CCD0003307F6000347070083C5060085072D8F3D
:10CCE0002380E600E39437FF3044A2852285EFF0ED
:10CCF0003FDFC1147DBF0145828019C9EF52EFD2D9
:10CD0000130680058145EF504FD505456F502FD450
:10CD10000145828081473DC9B5C9EF520FD1FC4121
:10CD200041462E84AA846393C70413860501A28713
:10CD30008146C14503C7070003C507038507298F3F
:10CD40003305D600034505008506298FA38FE7FE2E
:10CD5000E392B6FE3044A2852685EFF07FD8228587
:10CD6000EFF0BFF985473E856F506FCE13850703FF
:10CD70001D8E81452295EF504FCE7C40130700F861
:10CD800013060402A2972388E70255B73E858280E6
:10CD9000EF52AFC96D712E84B284AA85901028001D
:10CDA0003689EFF0BFDA19E9D55705A050400C409D
:10CDB0002800EFF09FE66DD9FD142104E5F82C0062
:10CDC0004A85EFF03FF5814765D13E8551616F504F
:10CDD0000FC8EF528FC541112EC432C62C00054634
:10CDE000EFF01FFB41016F508FC6EF520FC40111CE
:10CDF0002A842EC602C802CA02CC02CEEFC0604806
:10CE0000B2462A86A2850808EFF0BFFC1375F50F1D
:10CE100005616F50CFC3EF524FC17971B2872A8439
:10CE200021462308B10013051101BE853AC436C658
:10CE3000EFC0C01DB246930591013685EFF03FB7B4
:10CE40002285141035460C08EFF0BFF82A842247DB
:10CE500011E521460C103A85EFC0401B2285456143
:10CE60006F50EFBEEF526FBC7171AE84AA850A8518
:10CE70003284EFF0BFC801C90A86A6852285EFF08B
:10CE80003FC6814711E1C5473E854D616F502FBCBC
:10CE9000EF52AFB61D712A8AB289BE8435468547E6
:10CEA000130511012E8CB68A3A8BC28C468D23084D
:10CEB000F100EFC0A01510100C085285231F0100CF
:10CEC000EFF05FFA2A842DE9A147631BFD06930763
:10CED000900591E0E5473546E28513051101139968
:10CEE0000A012308F10013590901EFC0201213575A
:10CEF000890093978A00D98F90080C085285231FC8
:10CF0000F100EFF03FF62A8405E9A1E09387FA00EB
:10CF100091831379F9003EC6631309004149668B7A
:10CF20008144C14B854DB2476397970C6A868C004C
:10CF300033855C01EFC0800D228525616F50AFAF56
:10CF400093079004C9F8A54779B7834701050947B6
:10CF5000C14B2308F10083471105A58FA308F100F9
:10CF600093872400814463EFFB0201471408338652
:10CF7000E6008C08B386E400BA95DA9683C606000C
:10CF800083C505000507AD8E2300D600E390E7FEBC
:10CF900041476398E70490080C085285EFF09FEC36
:10CFA00035D535A8B3069B00BA871008B305F6003F
:10CFB00090083E9603C506000346060085078506D1
:10CFC000298E2380C500E39277FF998F90080C0883
:10CFD0005285BE94EFF01FE98947014749D52A845D
:10CFE000A1BF90083E96034606001408BE96238013
:10CFF000C600850779BFB2478504638B97128147C6
:10D000001808B306F70098083E973386F9000347DF
:10D010000700034606008507318F2380E600E39171
:10D0200077FF90080C085285EFF0DFE34DF93546A5
:10D03000E285130511012308B101EFB0307D13978C
:10D0400004014183939784002183D98F10180C0821
:10D050005285231FF100EFF0FFE051F181471018D6
:10D060003387F9003E960347070003460600B306E0
:10D07000FB008507318F2380E600E39277FF75A0E0
:10D080001808B306F70098083E973386F90003475F
:10D090000700034606008507318F2380E600E3E1A1
:10D0A00027FFCA876398770990080C085285EFF02C
:10D0B0007FDB15F581479800B306F700900818103C
:10D0C0003E973E9603470700034606008507318FCB
:10D0D0002380E600E39177FF3546E28513051101D1
:10D0E0002308B101EFB09072139704014183939725
:10D0F00084002183D98F10180C085285231FF1005A
:10D10000EFF05FD6E31D05EC814710183387F90077
:10D110003E960347070003460600B306FB0085075B
:10D12000318F2380E600E3E227FFC109410BE5BB15
:10D130008147B5B79408BE9683C6060018083E9787
:10D140002300D7008507B9BF638E062CEF52EF8A04
:10D1500059712A84BE89B28B854735461305110261
:10D160002E8B468C4289BA8A368A2300F102EFB0B0
:10D17000F06910180C10228523170102EFF09FCEE2
:10D18000631E0510A1476319FC069307900563937E
:10D190000900E5473546DA851305110293140A01A3
:10D1A0002300F102C180EFB0706693178A0013D795
:10D1B0008400D98F90080C1022852317F102EFF01C
:10D1C0007FCA69ED639009049307FA00BD889183D3
:10D1D00091E0C144C207C183DE8C814A3EC6414D05
:10D1E000B24763EAFA0C6286B3854B018810EFB050
:10D1F000905F4DC53D555DA093079004E39C09F8F1
:10D20000A54749BF834701050947C14C2300F102E7
:10D2100083471105B3C7F900A300F10293872900E2
:10D22000814963EFFC02814618103306D7008C0851
:10D230003387D900B69556970347070083C5050085
:10D2400085062D8F2300E600E390D7FE4147639AC1
:10D25000E70490080C102285EFF0DFC035D53DA81B
:10D26000B3863A01BA871010B305F60090083E96CF
:10D2700003C506000346060085078506298E238020
:10D28000C500E39297FF3387EC4090080C1022858D
:10D29000BA99EFF03FBD8947014741D565616F40BD
:10D2A0009FF990083E96034606001410BE96238010
:10D2B000C600850769BFB247850A93990A01939D05
:10D2C0008A0093D909016399570D85473546DA8558
:10D2D000130511022300F10293D98900EFB0105316
:10D2E000B3ED3D0190000C1022852317B103EFF040
:10D2F0007FB74DF58147A68963E6970626860C0819
:10D300004A85EFB0B05081471810B306F7001008F7
:10D3100098083E973E960347070003460600850798
:10D32000318F2380E600E3E197FE639DA905900815
:10D330000C102285EFF01FB335F181479810B3062A
:10D34000F700900818183E973E96034707000346DB
:10D3500006008507318F2380E600E391A7FF41098E
:10D36000C10CBDBD18089000B306F7003E96338788
:10D37000FC0003470700034606008507318F238022
:10D38000E60095BF98084E97034707001C10CE97FC
:10D390002380E700850951BF85473546DA851305A7
:10D3A00011022300F10293D98900EFB03046B3EDAA
:10D3B0003D0190000C1022852317B103EFF09FAAC6
:10D3C000E31E05EC814718089000B306F7003E966F
:10D3D0003387FC0003470700034606008507318FAB
:10D3E0002380E600E391A7FF41460C084A85EFB091
:10D3F000F04181471810B306F700100898083E97CF
:10D400003E9603470700034606008507318F2380B9
:10D41000E600E391A7FF90080C102285EFF09FA48F
:10D420001DDDADBD7D558280EF423FE001112A84B4
:10D430002E8593055100328902C002C202C402C681
:10D4400093047400EFF0AFD61D46A6851305910036
:10D45000EFB0D03B10088A854A85EFF0BFA019EDE8
:10D4600093071400180883C60700034607008507C2
:10D470000507B18EA38FD7FEE397F4FE05616F40D9
:10D480001FDDEF42FFD82E848C414111AA8983878A
:10D4900015003289914463D30700A1449797FF1F79
:10D4A000938787FA9C43B1C3B5CE8D472310F10013
:10D4B00083C725004A852301F10083C73500A301F6
:10D4C000F10083C745002302F10083C75500A30282
:10D4D000F10083C7650093059100A30301002303B6
:10D4E000F10023040100EFF08FCC0C404A860A853E
:10D4F000EFF00FCE0328040083564400A6881D08D1
:10D5000081470147E51642868A854E85EFF05F9890
:10D510002A8909E5A6852285EFB0FFB24A85410137
:10D520006F405FD24A860A85EFF08FCA7DBFEF4217
:10D530003FCE2E848C414111AA8983871500328900
:10D54000914463D30700A1449797FF1F9387C7EFC8
:10D550009C43B1C3A5CE8D472310F10083C725009E
:10D560004A852301F10083C73500A301F10083C779
:10D5700045002302F10083C75500A302F10083C7D1
:10D58000650093059100A30301002303F100230428
:10D590000100EFF0CFC10C404A860A85EFF04FC37F
:10D5A00083564400032804008A85858EC2061D0820
:10D5B000C1822312D400A68881470147E51642861E
:10D5C0004E85EFF07FB841016F40DFC74A860A857C
:10D5D000EFF00FC0C9B7EF425FC5B335B00001111E
:10D5E00085052A891315F601336515012308B10055
:10D5F0009305110136843AC632C03EC442C2EFF0F0
:10D600000FBBA2471248425593D68700230BF10067
:10D610009305910193578800A30AD100A30BF10051
:10D62000230C0101EFF0AFB8324702460328040093
:10D63000B337E000835644009207914411C2A144DD
:10D640004A85A68842860C08EFF09F842A8909E55E
:10D65000A6852285EFB03F9F4A8505616F403FBF99
:10D66000EF421FBB01113EC68647B335B0008505AA
:10D67000AA891315F6015D8D2308B10093051101E8
:10D6800036843A89B28442C446C2EFF04FB222488F
:10D690009248164593578800A30AF100930591011B
:10D6A00093D78800230B0101A30BF100230C110178
:10D6B000EFF0EFAF3247104083564400B337E0003D
:10D6C000920703280900914891C0A1480C084E8593
:10D6D000EFF09FA7AA8411E5835544004A85EFB077
:10D6E0009F96268505616F40FFB5AA959307F00FB9
:10D6F00017F700001307C7896317B50013C5F7FFB5
:10D700001375F50F828005058346F5FFB58FBA972F
:10D7100083C70700D5B70357450014419307F00F9F
:10D7200017F600001306C686369742074183139505
:10D7300006014181631BE500AD8FB29703C5070069
:10D74000130515F3133515008280850603C5F6FF12
:10D75000A98FB29783C70700D9BFEF421FADB28729
:10D7600036842E86BA86AA853E85BA84EFF06FE6A7
:10D77000634B05002285EFB0D0302A86A686A285AD
:10D780002685EFF00FE56F409FACEF427FA85D71FB
:10D790002A8BAE8A17E500001305057D2C00B284A4
:10D7A000368ABA893E89EFF04FE42A8459E534106D
:10D7B0004146DA852800EFF0CFE12A843DED854728
:10D7C000A303F100A6C2930771002408BEC4A68675
:10D7D00085470D462C18281002DC02DED6C0BEC6D6
:10D7E000EFF00FDB2A8431E983477102A6860D46EC
:10D7F00093F7F7072300FA00C1473EDE2C1889474C
:10D80000281026DCA303F100EFF08FD82A8415E559
:10D810004146A6854E85EFB0607F8D47A6860D46B2
:10D820002C182810A303F100EFF08FD62A8411E5FD
:10D830004146A6854A85EFB0607D228561616F40D3
:10D840007FA0EF429F9E97D7000093876709984378
:10D8500083C7470079712A89AE8417E50000130554
:10D8600025710C083AC42306F100EFF00FD82A8482
:10D8700015E514104146CA850808EFF08FD52A84B3
:10D8800011ED140815462C000810EFF08FD42A84EF
:10D8900011E521462C082685EFB0407722854561A9
:10D8A0006F40FF9AEF427F9897D700009387470316
:10D8B0009C477971AA842E8417E500001305C56B77
:10D8C0000C083EC6EFF06FD20DE514104146A68558
:10D8D0000808EFF00FD011ED140811466C00081085
:10D8E000EFF02FCF19E58347F10193F7F7032300FA
:10D8F000F40045616F40BF95EF423F933688A148E1
:10D9000081470147E546EFF0AFD86F405F94EF42A3
:10D91000DF913688A14881470147E546EFF0DF8275
:10D920006F40FF92EF427F9001112A842E850C08F0
:10D9300032C6EFF08FCB19E9324797E600009386A5
:10D9400026621008C1452285EFF03FE105616F4076
:10D950001F90EF429F8D4111C1472EC032C48A856E
:10D9600009463EC23EC6EFF0AFC241016F403F8E56
:10D97000EF42BF8B4111AE8613061009AA850A85B6
:10D9800002C002C202C402C6EFF0AFC441016F4040
:10D990001F8CEF429F89328797E600009386465E90
:10D9A0002E8693050002EFF05FDB6F405F8AEF4247
:10D9B000DF877971C1472ACC2ED032D42C080D468E
:10D9C00028003ECE3ED23ED602C402C602C802CADB
:10D9D000EFF00FBC45616F409F87EF421F8501113B
:10D9E000AA842E8417E500001305055A8A85EFF0F6
:10D9F000CFBF05E514084146A6850A85EFF06FBD47
:10DA000009ED8347E1010347F101A207D98FCA0756
:10DA1000C9836177D98F2310F40005616F403F837C
:10DA200005C9EF429F809787FF1F9387674F9043F9
:10DA30009785FF1F9385054F1785FF1F1305454ADF
:10DA4000EFB080091785FF1F130585496F403F80A0
:10DA50001785FF1F1305C54882809DC5EF42EFFC67
:10DA60009787FF1F9387C74B944301112E840A8623
:10DA70009785FF1F9385054BEFB0800A0A850294B6
:10DA8000014505616F40AFFC7D558280EF42EFF9A3
:10DA9000EFB080149787FF1F23A4A74817F5FFFF57
:10DAA000130525F8EF90D0406F406FFA1787FF1FDE
:10DAB000130747499317150008433E95FD57231058
:10DAC000F5008280EF426FF62A84084019E16F402A
:10DAD0000FF81C4158401CC06313E5005CC083472D
:10DAE000550023200500F99BA302F500EFB0EFF9E4
:10DAF000E9BFEF42EFF19787FF1F9387A74698434F
:10DB00002A8411CB8347350093F7070289C7035551
:10DB100005008945029713054401EF9010138355C2
:10DB200004000355E400EF20701B485809C5EFB00E
:10DB3000CFF5232A040213058403EFF0BFF88144D4
:10DB4000B149EFA0FF9A63C5A402834734002320A4
:10DB5000040493F727FCA301F4000048EFA05F9AA8
:10DB60001316150081452285EF402FEF6F408FED92
:10DB7000B38734030329040385043E994A85EFF0F3
:10DB80007FF42304090075BF8347350093F707022C
:10DB900099E3014582808357E500E39CB7FEC167A6
:10DBA000FD176316F600054582800545B9A0EF42D2
:10DBB000CFE793170601C187B2842A8401496359CC
:10DBC000F002835705008DCB01456367F6000345DE
:10DBD00084003E953325A6001375F50F39A81C481F
:10DBE00013171900BA9783D70700E38097FC05093C
:10DBF000EFA01F91E345A9FE01456F404FE5EF42BD
:10DC00002FE1AE89AA84EFA07F852A84EFD0BFAA36
:10DC1000AA8601471306840197050000938545E90C
:10DC20001785FF1F13054532EFA0AFD52A8921CDF7
:10DC30008C441304C50022859E0593F50508EFB0BA
:10DC40000FC5CC4083877400E18163D1070493E55D
:10DC500005082285EFB0AFC30D46938544002285A9
:10DC6000EFB00FC183D504002285EFB0EFC583D597
:10DC700024002285EFB04FC503D6490083A50900D3
:10DC80002285EFB0EFBE4A856F40CFDB93F5F507F5
:10DC9000C9B7EF428FD901112A84328532C6EFB05D
:10DCA0006FB4EF903F91835704001787FF1F13074E
:10DCB000E7423246231BF100930700F8A30DF10061
:10DCC0001C471843231AA1008983858BB307F740AB
:10DCD000B28548083ECE231C0100230D0100EFF061
:10DCE0001FF205616F40AFD6EF428FD20041014570
:10DCF00029CC9304C40026853289AE89EFB08FB257
:10DD000095452A8A2685035B0401EFB02FAF26854F
:10DD1000EFB02FC68D45AA8A2685EFB02FAE268597
:10DD2000EFB02FC55C48420A135A0A01D2975CC46F
:10DD300023186401814763983A0146054D813306F3
:10DD400025419337160013F5F70F6F40AFCFEF4221
:10DD50004FCB89692A8BAE8B328AB68A81440144C3
:10DD6000314CFD19EFA0CFF863C9A400EFA04FFB21
:10DD7000018D33B5AA006F404FCC338984038327CC
:10DD80000B003E9963170A008347890085043E947F
:10DD9000D1BF03560A00DE854A8533F6C900EFF08D
:10DDA000BFF47DD10545C1BFEF422FC801112A84C0
:10DDB0007C000355E5003ECAB70707003ECC7C0057
:10DDC0003ECEEF10303D2A8985454808EFB0EFC1BF
:10DDD00099454808EFB02FA7AA844A85EF10B03DB7
:10DDE0002380A4009787FF1F9387472F9C4341669A
:10DDF000130606F09396870113D78701558F93D6A4
:10DE00008700F18E558FA207B706FF00F58FD98FD7
:10DE100011462C00138514003EC4EFB0201F50089B
:10DE2000A382040089452285EFF0BFE609C9AA85CF
:10DE300013058403EFB0EFBB3C4085073CC0056190
:10DE40006F40EFC0EF426FBEEFA08FED2A84050454
:10DE5000EFA00FEC3305A402F14791453305F5021D
:10DE6000EF10207B01E565556F406FBE9787FF1F60
:10DE700023A2A70EEFA0CFEA2A840504EFA04FE962
:10DE80003305A40289450605EF10A07869DD978760
:10DE9000FF1F23A9A70AEFA0AFE82A840504EFA07B
:10DEA0002FE73304A4029787FF1F239F8708EFA063
:10DEB0002FE72A84EFA0CFE5930714003385A7024C
:10DEC0009787FF1F2393A70897E70000938787CFC3
:10DED0001787FF1F232EF706014579B7EF424FB38F
:10DEE000AA842E8901449789FF1F9389291F130A49
:10DEF0008006EFA0EFE16345A40001456F408FB4B9
:10DF00003305440383A709024A86A6853E95EFF0B0
:10DF1000BFC719E10504F1BF0545CDB7EF426FAEAC
:10DF2000AA8A2E8BB28B368C3A8A8144014481496D
:10DF3000978CFF1F938C8C1A130D8006EFA04FDD7A
:10DF400063C7A40011E085494E856F400FAF338948
:10DF5000A40383A70C025E86D6853E994A85EFF01E
:10DF6000BFC219CDEFA0CFDB0544636B4501D2865C
:10DF70006286DA8513050903EFF07FDD11C185495B
:10DF800085046DBFEF42CFA8C16441112A890144C5
:10DF90009789FF1F93898914130A8006FD1436C6DA
:10DFA00032C42EC2EFA0CFD692452246B246634677
:10DFB000A400014541016F40EFA83305440383A746
:10DFC00009023E9509C683473500C18B9DC791C69E
:10DFD0008347350093F707028DC363069900835783
:10DFE000E500639C27010357050001CB63E7E500CB
:10DFF00083478500BA97E3CFF5FA05044DB7EF42A2
:10E000002FA1C1642A8901449789FF1F9389090DB3
:10E01000130A8006FD14EFA0AFCF6344A4006F4045
:10E020006FA23305440383A709023E958357E50099
:10E03000638897006304990063942701EFF07FAB36
:10E040000504D1BFEF426F9B89692A8AAE8A328B61
:10E05000B68B8144178CFF1F130C4C08930C800661
:10E06000314DFD19EFA0CFCA63C4A4006F40AF9C2F
:10E070003389940383270C028355CA015A863E993B
:10E080004A85EFF07FB005CD814D05A03384AD0307
:10E090008327090303D60B00D68533F6C9003E94C7
:10E0A0002285EFF07FC419E5850DEFA06FC4E3CFA3
:10E0B000ADFC31A02285EFF0FFA02304040085040D
:10E0C00055B7EF420F944169AA8A014A178BFF1F87
:10E0D000130BCB007D19C14B054CEFA06FC36344FC
:10E0E000AA006F408F9593098006B3073A038329EE
:10E0F0000B02BE9983D7E900638C270163842A0150
:10E100006398570103A4890311E44E85EFF0DFC93A
:10E11000050AE1B783570401639977079304C400A4
:10E120002685EFA03FF085452A8D2685835C040176
:10E13000EFA0DFEC2685EFA0FFFF62056185635F3E
:10E1400005028D452685EFA07FEB89452685EFA04A
:10E15000FFEA89452685EFA07FEA85452685EFA061
:10E160003FEB83470500094793F7F7076398E700FC
:10E1700099452685EFA0DFE9A30285014848337D54
:10E180002D01231894016A9548C40040B5BFEF42A1
:10E19000CF8937E404008327041D82979787FF1FE8
:10E1A00083C7C7E01755FF1F1305454AA300F500B5
:10E1B0008327441C82978327841C81461306F00F13
:10E1C0008145014582976F408F881787FF1F13078E
:10E1D000E7CD18439785FF1F83C545DD9787FF1F50
:10E1E000938747DB83468703034697036397D500EE
:10E1F0009787FF1F238CC7DA828083C58701034777
:10E20000A7036317B6009787FF1F2381E7DA828091
:10E2100003C687016317C7009787FF1F2388D7D8D6
:10E22000828083C68701130750026319D7009307C2
:10E2300060021787FF1F230BF7D6828083C68701F2
:10E24000130660026315D60093077002DDB783C71B
:10E25000870155BF9787FF1F9387C7D3D44B0947C3
:10E260006385E608EF327FFC1789FF1F1309C9CFCA
:10E270003E8483470900918B9DCFB7E4040083A7B8
:10E28000041D829783A7441C1785FF1F130545CEE5
:10E29000829783A7841C81461786FF1F034646CFBB
:10E2A00081450145829721C183470900ED9B17876E
:10E2B000FF1F230BF7CA8347040093F7F70F85C7A7
:10E2C00091471787FF1F2321F7CEEFF05FECEFF0A8
:10E2D000DFEFB7E70400BC4F414691451785FF1FAC
:10E2E0000345C5CB82976F309FF68280EF32FFF3F4
:10E2F0008D4741116304F504C5476306F502854760
:10E300006310F5029787FF1F2384A7CAB7E70400AD
:10E31000BC4B930500101785FF1F034525C8829746
:10E3200041016F30DFF285471787FF1F2302F7C8CF
:10E33000B7E70400BC4B93050020F1BF9787FF1F90
:10E34000938747C5D44B1147638DE600B7E70400B8
:10E3500083A7071D8297B7E70400BC4B9305000411
:10E360005DBF05491787FF1F232027C583C7070007
:10E3700032C62E8493F7F70FC5D7B7E4040083A7FE
:10E38000041D7D141374F40F8297E37689FCB24563
:10E39000994703C61500E3F0C7FCFC44090617853E
:10E3A000FF1F130525C18297BC48930500081785F8
:10E3B000FF1F0345A5BE829779BFEF321FE717877E
:10E3C000FF1F130727BD4047184B1C409786FF1FB0
:10E3D00023A8F6BC6316E4001787FF1F2324F7BCAD
:10E3E000130584FEEF907FF3035564FFEF903FC663
:10E3F000EFA0BFE96F30BFE5EF323FE39787FF1F24
:10E40000938747B9D84BDC4799C3EFF01FFB85478B
:10E410001787FF1F232AF7B89787FF1F938707A93E
:10E420009C43930500021785FF1F034525B783C74B
:10E4300087031787FF1F230BF7B6B7E70400BC4B12
:10E4400082976F30DFE09787FF1F23A7A7B48280F2
:10E45000EF321FDC37E404007C4CA1451785FF1F19
:10E460000345C5B382977C48A1451785FF1F034527
:10E47000E5B29784FF1F9384E4B18297DC4489E777
:10E48000EFF05FDD6F301FDC03D567FFEF903FBC1F
:10E49000AA897DD5D84891476310F7027C4C9145F5
:10E4A0001785FF1F034585AF82977C4891451785E7
:10E4B000FF1F0345A5AE829703A9490103D40901B3
:10E4C0008947B7E904001787FF1F232FF7AC83A7FD
:10E4D000091D21044204829783C784011755FF1F39
:10E4E0001305C51661191757FF1FA301F71683A758
:10E4F000491C418082979787FF1F238B07AA83A718
:10E50000C91C814609469375F40F4A85829711E923
:10E510009787FF1F83C707BA89C79750FF1FE780F8
:10E52000E084B7E70400BC4F2146A1451785FF1FD3
:10E530000345C5A68297B9B7EF323FCF93F70520C1
:10E5400001112E8481CBEFF03FEB134504200561D0
:10E550006F30FFCF93F70510A9CB9784FF1F9384EB
:10E5600064A3DC48EFF07FC61787FF1F13070794EB
:10E57000184383C78401034787036316F700DC440D
:10E5800099C3EFF09FE385471787FF1F232EF7A05E
:10E59000B7E70400BC4B930500021785FF1F034536
:10E5A000E59F8297134504105DB793F70508ADC743
:10E5B0009787FF1F83C717A0E91719469785FF1F85
:10E5C0009385659F1305D10093F4F70F1789FF1FFB
:10E5D0000349499EEFA0902393970401C1831787B5
:10E5E000FF1F1307A79D231DF100231CF100978730
:10E5F000FF1F9387279A3ACE3ACAD84323060100D1
:10E6000009CBDC439315890154080D46E185680068
:10E6100082971345040825BF93F72500B1CF97874C
:10E62000FF1F93872797D84B89476306F702978781
:10E63000FF1F83C7679313F7270011EF918B99CFC3
:10E64000B7E70400BC4F1306000A89451785FF1F72
:10E650000345C594829713452400D5BD9787FF1FB6
:10E660009387C7849C4383C787031787FF1F230FA4
:10E67000F792EFF0FFDDC5B793F7050291C7EFF012
:10E680003FDD13450402E1B593F7850091C7EFF034
:10E69000BFD61345840065BD93F7150091C7EFF011
:10E6A0007FBB1345140065B593F7450091C7EFF0A4
:10E6B0007FBA1345440061BD93F7050485C397876E
:10E6C000FF1F83C7278D81CBEFF07FAC9147178762
:10E6D000FF1F232BF78C1345040495BD93F7050109
:10E6E0000145E38607E69787FF1F9387A78AD84BE4
:10E6F00091476310F7049787FF1F9387E7869C4332
:10E7000013D727008583D98F858B91E7B7E704005E
:10E7100083A7071D8297B7E70400FC4F9145178533
:10E72000FF1F0345A587829785471787FF1F232D66
:10E73000F7861345040121BD9787FF1F238CA796F9
:10E740008280EF329FAE9787FF1F23AB07849787A6
:10E75000FF1F23A9078485471774FF1F130404753F
:10E760001787FF1F2322F7841C4083C7870317875F
:10E77000FF1F230DF782EF90FFDF39C19757FF1F6F
:10E7800023AAA7EC1C4017050000130525DB83C74F
:10E7900087031787FF1F230BF7801757FF1FA30758
:10E7A000F7EA9777FF1FA387077EB7E7040083A7E1
:10E7B000070882979777FF1F2382A77E6F303FA9B4
:10E7C000B7C7898E938767ED1757FF1F2324F7E894
:10E7D00055BF1777FF1F0347E77B795555E39777B9
:10E7E000FF1F9387277B03C7170005079776FF1F37
:10E7F000A382E67A03C717008D463377D702977650
:10E80000FF1FA389E67883C617001777FF1F13073A
:10E81000E769184393F6F60FA9EA8347870317774A
:10E82000FF1F2305F77885471777FF1F2304F77627
:10E830009777FF1F938747739C430145998BA9E303
:10E84000EF32BF9E37E404007C48C1451775FF1FB7
:10E850000345C57482973C4885451775FF1F0345DE
:10E86000E573829701456F309F9E83C717008546E9
:10E870006395F600834797035DB78347A70345B7C2
:10E8800082809777FF1F83C7E770A1CBEF32FF9994
:10E8900037E404009777FF1F238E076E7C48854579
:10E8A0001775FF1F0345856F82977C4C914517753F
:10E8B000FF1F0345A56E82977C4891451775FF1F82
:10E8C0000345C56D82973C48C1451775FF1F034539
:10E8D000E56C829701456F309F9779558280EF32C2
:10E8E000DF942A84035565FFEF906FF69777FF1F3B
:10E8F0009387476AD847BE841DEBEFA05F989C487A
:10E90000232004008DEB9777FF1F23AD876897774F
:10E91000FF1F23A78768B7E70400BC4B894517751D
:10E92000FF1F0345A567829701456F305F92630A19
:10E9300087001843D1B780C39777FF1F23A487664A
:10E94000D9BF7955DDB7EF325F8E9777FF1F938779
:10E95000A776884323260500232405005105EF8070
:10E96000D02E6F30DF8EEF325F8C1774FF1F1304D1
:10E97000A4741C40411189CF9C472302B5002AC6CC
:10E980001CC1EFF05FFC1C409C4B99C33245829741
:10E9900041016F30DF8BEF325F894111444D328589
:10E9A00032842EC6EFA00FF92AC42285EFA0EFF91A
:10E9B00003A84400630C0800B24583574400184084
:10E9C000224683D54500AA862685029841016F30EC
:10E9D0001F88EF329F85404D1DC408C09705000079
:10E9E0009385E50213054401EF8090189777FF1F88
:10E9F0009387876C9C43014589E79777FF1F23AD79
:10EA0000876A6F30DF847D55EDBFEF321F820111C1
:10EA100068009305F00F02C602C802CA02CC02CEFB
:10EA2000EFF07FF405616F309F829777FF1F938728
:10EA3000A7689C43D847A1679D076311F702EF328F
:10EA4000CFFE01113285EFA0EFEE230AA100814530
:10EA50006800EFF05FF105616F306FFF828097779C
:10EA6000FF1F938767659C43D847A1679387770308
:10EA70006311F702EF326FFB01113285EFA08FEBCC
:10EA8000230AA10081456800EFF0FFED05616F30BA
:10EA90000FFC82809777FF1F938707629C43D847BC
:10EAA0009547631CF702EF324FF80111328532842B
:10EAB000EFA04FE8230AA1002285EFA00FE98357BA
:10EAC0004400231BA10081453ECC1C4068003ECE83
:10EAD000EFF07FE905616F308FF78280930785FF44
:10EAE00089CF8327C5FF91CBDC4B81CBEF32EFF38E
:10EAF000032585FF82976F308FF58280EF32EFF22A
:10EB00002A843285EFA00FE3BD4763EBA7001844CA
:10EB10009377F5000345B70041995D8DA305A700E4
:10EB20006F30EFF2EF326FF001117C003ECAB70791
:10EB300007003ECC7C003ECE5C4D8DCF2A841385F1
:10EB40008700AE84EF807004A1652A899D0548087E
:10EB5000EF80FFBD9305803EB345B902480893F5A9
:10EB6000F50FEFA0CFD2014781465008A685228538
:10EB7000EF807FDC05616F308FEDEF320FEBEFF050
:10EB80007FFA6F30CFECEF324FEA01117C00AE8498
:10EB90003ECAA165B70707002A843ECC48087C001E
:10EBA000938575033ECEEF809FB81C44480883C50B
:10EBB000B700BD89EFA0AFCD500801478146A685BB
:10EBC0002285EF805FD705616F306FE8EF32EFE5A8
:10EBD0002A84AE84EFF09FF2A6852285EFF0BFFA7B
:10EBE0006F30EFE6EF326FE4EFF0FFF96F302FE6B2
:10EBF000EF32AFE30329C5014111630409022A84FE
:10EC00003285B284EFA00FD32AC62685EFA0EFD3BA
:10EC1000832749002A8691C7DC4781C7B2452285F0
:10EC2000829741016F30AFE2EF322FE0444D81CC4B
:10EC30002A843285EFA06FD1DC40AA8589C79C4722
:10EC400099C3228582976F308FE0EF326FDC032A01
:10EC5000C501411163030A062E89AA8495453285B0
:10EC60003284EF80DFAC85452285EFA0CFBDAA8935
:10EC7000CA852285EFA0EFC283274A009DC7DC43E7
:10EC80008DC72285EFA0AFBA83274A001040835674
:10EC90004400DC437115A307A100B2961307F100ED
:10ECA0004E86CA852685829701C52380090031A03A
:10ECB0008345F1002285EFA00FB941016F308FD855
:10ECC000EF32AFD665711C083EC2B70780013EC463
:10ECD0001C0832893EC62A84AE84EFF07FF14A8553
:10ECE000EFA0AFC68357A10089CFAA855000228527
:10ECF000EFF0BFF5014781465000A6852285EF80E1
:10ED00009FC359616F30AFD4EF328FD065711C084B
:10ED10008329C5013EC2B70780013EC41C082A846E
:10ED2000AE8432893EC6EFF03FF0638409024A8523
:10ED3000EFA0AFC18357A100AA8581CF50002285E3
:10ED4000EFF0BFF0014781465000A6852285EF8095
:10ED50009FBE59616F300FCFEF322FCD65711C0808
:10ED60003EC2B70780013EC42A841C0832853EC6D5
:10ED7000AE84EFA08FBD8357A10089CFAA85500034
:10ED80002285EFF09FEC014781465000A685228541
:10ED9000EF807FBA59616F308FCBEF320FC9444D8E
:10EDA00091E88347450093B71700B307F0403E85CD
:10EDB0006F30EFC91845FD577DDB9707000093873B
:10EDC00007032A845CCB97050000938565D11385E2
:10EDD0008400EF80E05980C003474400814761FB15
:10EDE0001777FF1F232C972CD9B7EF326FC28329D7
:10EDF000C5014111032985008147638B090803245C
:10EE0000090191452A8A2285EF807F9285452285D6
:10EE1000EFA06FA38945AA8A2285EFA0CFA2AA847A
:10EE2000EF809F9683A749002A8B9DC79C438DC77F
:10EE30002285EFA0CF9F83A74900A306A100104021
:10EE4000835644009C431307D100B296D68513061F
:10EE5000E1005285829709CD83570B002380F4008F
:10EE6000A183A380F40023800A00A306010029A83F
:10EE70008357E10022852380F4008345D100A183DC
:10EE8000A380F400EFA02F9C8347D100B337F0009C
:10EE90000347B900920701453D9BD98FA305F900AF
:10EEA00041016F302FBAEF324FB841111DE997770A
:10EEB000FF1F9387A720804305C8044013098400DF
:10EEC0009DC55C4099C79C4B89C726852EC68297F5
:10EED000B2459307803EB385F5024A85EF806055C1
:10EEE00021A0404DAA8479F841016F304FB64A8580
:10EEF000EF80A0555C40EDDBDC4BFDD7268582978B
:10EF0000E5B7EF328FB22A843285EFA0AFA2AA858F
:10EF10002285EFF05FF96F308FB3EF320FB12A84A3
:10EF2000AE84EFF01FFEA6852285EFF0BFBF6F30E5
:10EF30000FB208413355B50005898280EF32EFAE3C
:10EF40001774FF1F130484191C5C0111231701009F
:10EF50008D83858BA303F1008327040B2318010005
:10EF60002319010003D7C7013ECA3C002314E10066
:10EF70007D572315E1000357C4023ECC02CE231671
:10EF8000E100EF802FE38357E101231EA10093F7F7
:10EF900007E093E71710231FF1009777FF1F83C740
:10EFA000871685C305470145638AE70083478403C5
:10EFB00093E727001777FF1F230EF71405616F30C3
:10EFC0000FA9814717D700001307C71B85461306F3
:10EFD000710085454808EF70E04B6DF1834784036D
:10EFE000F59B1777FF1F2307F71285471777FF1F3A
:10EFF000230BF710E1B7EF324FA0977DFF1F938DE2
:10F00000ED0D03A6CD0639712A8981478144930607
:10F0100000023357F600058B01C7850493F4F40F03
:10F020008507E398D7FE83A70D0B2317010223184A
:10F03000010203D7C7013EDA3C102314E1027D57D9
:10F040002315E10203D7CD023EDC2319010223166A
:10F05000E10202DEEF800FD68357E103231EA102F7
:10F06000014593F707E093E71710231FF102977705
:10F07000FF1F83C74709A9EF9777FF1F83C797092A
:10F080003EC69779FF1F938969050144014D9D4A4A
:10F09000054B954B177CFF1F130C8C0B977CFF1FA8
:10F0A000938C8C0A03DAC90563090A00EA856314A4
:10F0B00059036685EFF0FFE71DC1050DA1478909DA
:10F0C000E312FDFE2DE09777FF1F23A107080145FE
:10F0D00021616F304F966285EFF0BFE579DD3247F1
:10F0E000B3878400E3F0E7FE9C00130614000604D7
:10F0F0003E9413178A0093578A00D98FC207C183A1
:10F10000A30EF4FCA183230FF4FC03A70D07B31790
:10F11000AB01D98F1777FF1F232AF702630476010B
:10F12000328461BF15449777FF1F83C7A7FD1387FC
:10F1300017009776FF1F2387E6FC93161400230E13
:10F14000F10017D700001307E70381478506700811
:10F15000CA854818EF700034E34705F68347C101BC
:10F1600005451777FF1FA30FF7F89777FF1F238C2D
:10F1700027F9B9BFEF32CF890111AA892E84EFD0C8
:10F18000EF9C2A899774FF1F938444F56399090AB9
:10F190009C5C414793F707036393E70A1777FF1FC8
:10F1A0000347B7F6894763ECE70883A7040B2317E7
:10F1B00001002318010003D7C7013ECA3C002314F5
:10F1C000E1007D572315E10003D7C4023ECC23198B
:10F1D00001002316E10002CEEF80CFBD231EA10067
:10F1E000EFC06FCD8357C101230FA100914613D704
:10F1F0008700A207D98F2312F1009777FF1F83D7CB
:10F2000087F113D78700A207D98F2313F10017D7EF
:10F2100000001307A7F68147500095454808EF7096
:10F22000602705889317240003C484036D985D8CC0
:10F230009777FF1F238087EE05616F30AF80EF70F7
:10F24000B0781775FF1F130565EDEF80002083A7C9
:10F25000040B9775FF1F83D525EB03D5C701EF106E
:10F26000E0279777FF1F83C7E7EA93F60702014776
:10F2700089E61777FF1F035727E99776FF1F239D1E
:10F28000E6E81777FF1F130727E4184309CBC18B64
:10F2900099C789451775FF1F035505E702979777AB
:10F2A000FF1F23A307E69777FF1F238E07E49777B7
:10F2B000FF1F23AB07E89777FF1F23A907E897777E
:10F2C000FF1F23A707E883D7840393F7270C93E74F
:10F2D00017001777FF1F231FF7E283572903A18B1E
:10F2E00099C3EF70E03F11C49777FF1F23AA07E08F
:10F2F000A1B78D471777FF1F2324F7E0EF902FA5C5
:10F300009305803EB305B5021775FF1F130505E190
:10F31000EF80201215B79777FF1F938727DCD8530C
:10F3200025C791C99777FF1F238F07DC9777FF1FAA
:10F3300023AE07E08280EF225FEF83C7F70241111F
:10F340002EC685071777FF1FA301F7DC9777FF1FEE
:10F350002395A7DC9D471777FF1F2323F7DAEF904C
:10F360000F9E2A84EF90AF9DB24501E5EF902F9D4F
:10F37000AA85B305B4401775FF1F130525DAEF8082
:10F38000400B41016F20BFEC82809777FF1F93876E
:10F39000E7D4D85331C7EF225FE903C7F702050767
:10F3A0009776FF1FA383E6D611CD8C5F0D470145ED
:10F3B000898185899776FF1F23A4E6D4EFF09FDB30
:10F3C0006F20FFE885479305C0441775FF1F13059D
:10F3D000E5D41777FF1F2325F7D2EF808005CDB73F
:10F3E0008280EF229FE41777FF1F0347C7D185472D
:10F3F000631EF7009777FF1F938747CE83C7870366
:10F4000093C787001777FF1F2306F7D01775FF1FD5
:10F410001305C5D0EF806003EF807FEF9947177722
:10F42000FF1F232FF7CC9777FF1FA38007CE977777
:10F43000FF1F238A07CCEF90AF8F93074006330559
:10F44000F5029777FF1F23A3A7CC6F205FE0977784
:10F45000FF1F83C727CCC18B99C7EF221FDDEFF0B9
:10F46000FFAD6F20DFDE695582809777FF1F93879E
:10F47000E7C6DC5381CBEF225FDB8545EFF09FCF02
:10F480006F20FFDC82801777FF1F130727C5014617
:10F490008146BA852148631E06019DCA2390A600B5
:10F4A00083C7850393E717001777FF1F2304F7C669
:10F4B00005A08357C705631DF502F8598547B39723
:10F4C000C70093C7F7FFF98F1777FF1F2322F7C8ED
:10F4D0009C5D9183858B85C79777FF1F83C7A7C2E4
:10F4E00099EFEF229FD41D45EFF0FFB06F203FD67C
:10F4F00081E699E39306C7050506090769BF82807F
:10F50000EF223FD08605AA84B309B500977AFF1F82
:10F51000938A8AC3054B977BFF1F938B2BC3214C88
:10F52000639434039777FF1F938747BB9C5F918356
:10F53000858B89CB9777FF1F83C7E7BC81E7214580
:10F54000EFF07FAB6F207FCF03DA0400630B0A0478
:10F550001779FF1F130989B80144CA8C8357C9055D
:10F56000639D4703A2855685EFF0BF9C11E5A285F8
:10F570005E85EFF01F9C05C903A74C07B3178B00EE
:10F58000D98F1777FF1F2325F7BC83C78C0393E719
:10F5900017001777FF1F230FF7B605040909E31FAC
:10F5A00084FB8904B5BF231E0904C5BF1777FF1F5D
:10F5B000034767B58547631AF700EF221FC7EFF0CF
:10F5C0005FE2EFF0BF976F209FC88280814785453B
:10F5D0001306000293861700B397F500E98F13F71F
:10F5E000F60F89E7B687E397C6FE01473A85828022
:10F5F000FD4785457D56B396F50013871700E98EC4
:10F600001377F70F89E6FD17E397C7FE01473A85A1
:10F61000828089E901473A85828001473A85410124
:10F620006F20FFC2EF227FC041112AC62E852EC453
:10F63000EFF0DFF9A2457D158547B397A700E39E5C
:10F64000F5FC32469377360099C3719A1106977785
:10F65000FF1F938767A894433E871778FF1F1308FF
:10F66000E8A689EA832708009107F19B9776FF1F98
:10F6700023A4F6A6032588001843B307A700B3F711
:10F68000B702B387F540FD15FD8D83274800AA9585
:10F69000B306B600E3F3F6F8E371D5F82E97977743
:10F6A000FF1F23A9D7A23DDB3A858145EF20FFBA92
:10F6B0002A87ADB718419777FF1F938727A123A407
:10F6C000070098C35841D8C39777FF1F23A607A008
:10F6D0008280EF22FFB3AA8401441779FF1F130928
:10F6E000E99F9309400EEF807FD56345A400014553
:10F6F0006F205FB5330534038327090B3E9583578D
:10F70000C501E38797FE0504F9BFEF229FAF977904
:10F71000FF1F9389A99C3E84BA848347060003A7F0
:10F72000090041119D83058B3D8F83C74401AE8A3B
:10F730002A89F99BD98F238AF4001C44B6852312A9
:10F7400004001CC02285328A36C6EF90DF8FB24695
:10F75000D2853686EF90900BDC4883A509000840DF
:10F76000858B56869D8DEFD03FCC61E918407D5545
:10F770008347570003476700A207D98FC207C18795
:10F780002394F4006358F00A83C7440193F70703F6
:10F79000B5CBD0489377160003A609001D8E977746
:10F7A000FF1F938767CA9C43ADEB814641A003A727
:10F7B0000B0093172A00BA971840944383475700C9
:10F7C0008345670033F65601A207CD8F6311F60219
:10F7D000834737000346470003472700A207D18F1E
:10F7E0004207D98FBD82B3F76701638AF604050A21
:10F7F000EF80DFC3420593170A014181C183E3E82B
:10F80000A7FA41BFA16A370B0200014A977BFF1F8D
:10F81000938B8B9AFD1A7D1BE1BF83C744011307AD
:10F820000003854693F70703E391E7F8A2854A852D
:10F83000EFD0FFCF41016F205FA06155E5BF795543
:10F84000D5BFEF22FF9C9764FF1F938464719C4097
:10F85000D9EF9777FF1F9387E7869C436399070C3F
:10F86000EF80DFBE930780023305F5028945EFF094
:10F870005FDA41C99777FF1F23A8A790EF801FBCCD
:10F880009307400E3305F5029145EFF09FD835C937
:10F890009777FF1F23ACA78EEF805FB201CDEF807B
:10F8A000FFB191450E05EFF0DFD621CD9777FF1F11
:10F8B00023A0A78EEF801FCB11CDEF80BFCAD94701
:10F8C0003305F5028945EFF0DFD405CD9777FF1FAB
:10F8D00023AAA78AEF809FB591450A05EFF07FD351
:10F8E0000DC19777FF1F23A9A78C014521A8EF80A1
:10F8F0003FC2930780063305F5029145EFF07FD1B3
:10F9000001E565556F201F949767FF1F23A8A77E09
:10F910000144130A80061769FF1F1309297CB14AA5
:10F92000EF801FBF6364A4029C40E38407F2EF8072
:10F930003FBE9307A0043305F5028945EFF07FCD64
:10F9400069D19777FF1F23ADA78619BFEF805FBBF3
:10F9500089450605EFF0FFCB4DD5B30944030327D6
:10F9600009024E9708CBEF80BFB833055503914588
:10F97000EFF03FCA59D58327090205041374F40F29
:10F98000CE9788DB71BF9767FF1F938727758847DE
:10F9900005898280C167FD176319F5009767FF1F0E
:10F9A0009387C77303A5070B8280EF221F88EFF0B0
:10F9B0005FD26F20DF89814709C58347E501B337EF
:10F9C000F0001767FF1F1307677118470983058B3E
:10F9D00019C393E727003E858280EF221F852A8482
:10F9E000EFF07FFD8347E401AA851305940899E3AE
:10F9F000130504039766FF1F9386466E9442130611
:10FA000015021307840213059504EFD0CFC06F20B1
:10FA10001F84EF22EFFF9764FF1F9384246C9844A8
:10FA20002A892E840983058B9C4019C76314F5002D
:10FA30006380050E014401A2E3FEA7FE1387A7021F
:10FA4000E36AA7FE850763FCA70883A9440BEF8040
:10FA5000FF961316350081454E85EF201F8097676E
:10FA6000FF1F23AD27679767FF1F23AB076649CCAE
:10FA70009C4493E747001767FF1F2325F7669767A6
:10FA8000FF1F2389076C630F040C9767FF1F23A7D1
:10FA9000276501440549EF807F926341A40AEF8006
:10FAA000FF9493050006B3C5A502B7F73600938708
:10FAB00007E81765FF1F1305256A4169014493098B
:10FAC000400E7D19B385F502EF70B016EF801F97D9
:10FAD000634FA4080145EF3040700544A9A863981E
:10FAE000A7029DE583A9440BEF805F8D13163500B7
:10FAF00081454E85EF206FF69767FF1F23A0275F94
:10FB00009767FF1F23AE075C9C44ED9BADB785C58F
:10FB10001767FF1F034707649307F005E3FCE7F04F
:10FB200021F8EF60F03C6DD19C4493E70702176722
:10FB3000FF1F2329F75A22856F20CFF083A7440B9C
:10FB4000131534003E958357050081CB834725006C
:10FB500099C721468145EF204FF005042DBF2301B1
:10FB60002501E5BF9767FF1F23AC07560DBF33057F
:10FB7000340383A7040B3E958357C5016384270193
:10FB8000EFF0BFE5050499B7EF222FEAEF801F865B
:10FB9000130400063345A4029764FF1F93840454A2
:10FBA00083C784073E951375F50F9767FF1F23835F
:10FBB000A75A9307F00563E7A7020545EF30E06118
:10FBC000EF80DF823345A402B7F53600938505E860
:10FBD000B305B5021765FF1F13050558EF707005D3
:10FBE0006F20EFE69C4405458983858B81CBEF90A0
:10FBF0004F8888408145EFF0DFE1DDB7EF30E05D11
:10FC0000C5B7EF22EFE0130495082A891306900583
:10FC1000A28513050503EF90603F1306900581450B
:10FC20002285EF208FE34A85EF30C0548144176A64
:10FC3000FF1F130AAA4A930A8002EF803F8163C420
:10FC4000A4006F202FE0338454038327CA0A3E9414
:10FC5000035704008357C9016317F7028347440021
:10FC60009DC3930964014546CE8513055400EF906A
:10FC7000E039454681454E85EF202FDE228523025F
:10FC80000400EF30005785044DBFEF220FDA97676D
:10FC9000FF1F9387E72C9C432A8491C70DC503550A
:10FCA000C501EFE00FC29767FF1F9387E7799C4379
:10FCB00089CBEFB0DFD085476315F5002285EF5083
:10FCC000C05D6F20CFD841657D15E1BFEF22EFD534
:10FCD0001764FF1F13048440444093871400176780
:10FCE000FF1F232FF73EEF30605E1C448983858B16
:10FCF0009DE75840B7E7B0009387075063F1E702EC
:10FD00000145EFF01F9D01CD0545EF809FF60840AE
:10FD100085450505EFF0FFCF0145EFF01FF726857C
:10FD20006F20EFD2EF22CFCEA1642A8901449769D8
:10FD3000FF1F93896948FD14338AA500EF800FEFF8
:10FD40006344A4006F200FD003A709009317240079
:10FD5000BA979843658F42074183634C2701635AE2
:10FD6000470123800700A380070023810700A381A8
:10FD700007000504E1B7EF224FC883594500C54786
:10FD8000411163F537310441C1E5338534018347BF
:10FD900085FF034795FF0348B5FFA207D98F0347A7
:10FDA000A5FFC207220733670701D98F0347C5FFA5
:10FDB0000348D5FF2207336707010348E5FF0345E2
:10FDC000F5FF420722083365A800498FB98F1767EE
:10FDD000FF1F1307273C1768FF1F1308A83D3A852C
:10FDE000832807006384172B1107E31B07FF17679E
:10FDF000FF1F1307273C18431318270042951CC107
:10FE00000507A1473367F7029767FF1F23A4E73A67
:10FE100093F735001397470083474601C16B368936
:10FE200093F7F7FCD98F32842E8A230AF600814A91
:10FE3000176CFF1F130C8C2AFD1B976CFF1F938CF4
:10FE40002C12176DFF1F130DAD37EF802FDF63C727
:10FE5000AA00E154268541016F20EFBD1308400E32
:10FE6000B3870A0303280C0BB30DF800638E0D2033
:10FE700083D7CD01638A772183A70C00014B639759
:10FE800007169767FF1F9387E7239C436390071626
:10FE900083C7040003C70D0493F7F707631BF71A22
:10FEA000CA872287CE86268693859D0613851D04E4
:10FEB000EFF0BF85631F051883D7CD010327090025
:10FEC0002320B4012312F400FD572313F4008347C9
:10FED000170093F6F7078347D40093F707F8D58FF9
:10FEE000A306F40093F7F707B337F000B307F04029
:10FEF0002307F400834717009D83939637008347B9
:10FF00004401DD9BD58F230AF400834737008346E5
:10FF10004700A207D58F83462700C206D58F1CC88D
:10FF20008347770003478700A207D98F2315F40082
:10FF30000D476304EA00BD5491DF93870710C207A1
:10FF4000C1831307B00FBD54E376F7F0EF800FC9FC
:10FF50008144E31105F09766FF1F83C62626938729
:10FF600016001767FF1F230BF7241767FF1F1307E0
:10FF7000A724231BD400939726001443035784001F
:10FF8000E175BE96A1671386F7FFB377C700984265
:10FF90006D8FD98F9CC21848F18F3E07D98F9CC2B4
:10FFA000EF80CFC89767FF1F83C7472133F5A702AC
:10FFB0009767FF1F2384A72071BD9307A004B30890
:10FFC000FB0283270D00BE9803D7080083D7CD011D
:10FFD000631DF70083C7040003C7880093F7F70782
:10FFE000630BF70083C7FD019DEB050BEF804FD23C
:10FFF000E345ABFC71BD9385980113859800CA87D2
:020000040001F9
:100000002287CE86268646C6EFF02FF0B24879F9D1
:100010008347440193E74700230AF40071BD83C777
:10002000040003C7980293F7F707E310F7FCCA87A9
:100030002287CE8626869385A8031385A802EFF033
:10004000CFEC45F58347440193E72700230AF400EA
:10005000C1B783C7FD018DCB83C7040003C79D09CA
:1000600093F7F7076312F702CA872287CE862686A0
:1000700093852D0C1385AD09EFF02FE911E583472A
:10008000440193E7270049BF850AC1B3FD54D9B3A2
:10009000EF222F97797183544500AA8B2E84B28A60
:1000A000EF80CFBB590563499504B7E4040003A969
:1000B0000407EF80AFBA59054205418102992A89A8
:1000C00005CD2AC623180100EF804FB95905231921
:1000D000A1006146814528089769FF1F938909009F
:1000E0004ACAEF208F972302810203A48900058862
:1000F00019E4BC544A85829745616F200F947400BF
:100100003008D6855E85EFF01FC765F56800EF8083
:100110007FF1176AFF1F130A2A3383270A00AA8474
:10012000035B010189CB89476397FA00835501027C
:100130005E85EF50203003552102EF704FC819E55E
:1001400003552102EF708FD43334A000931764005D
:100150000344C1022C0868001374F4FB5D8C230671
:100160008102EF60B056E9576314F5028356E1024D
:100170009767FF1F938747049C4313972600617678
:10018000BA979843718F98C39767FF1F2388D70248
:10019000831721026345F00085476396FA00B25742
:1001A00093F7070C95E7D247C2040347C102C18009
:1001B000BE9426C62318610113770703C147631D48
:1001C000F70083475102054793F7F7076390E70469
:1001D000B7E70400BC5739BF92570544A18393F792
:1001E000F707E377F4FE15C78347C1021307000240
:1001F00093F707036397E700EFB06FFC8547E319B8
:10020000F5FC8347C10293F7070389CFEFB0AFCA6C
:1002100021A8EFB08FD7E30985FCEFB04FFAE319BF
:1002200085FAD9B7EFB0EFD8AA8501460545EF703A
:100230007FF82A8451DD8347C102414793F70703C2
:100240006384E70232478347170093F707F8A30058
:10025000F7003247925783461700A18393F7F707B9
:10026000FD17D58FA300F70003560101B245130B0C
:10027000C4005A85EF80DFDFE24A1306900583470A
:10028000C10283C4EA01918BB384C40213851404B0
:10029000569595C35444B3879A0083C7070403C790
:1002A0000600137707F82380E600584483460700CA
:1002B000D58F2300F700B25703A609008146858B2E
:1002C0001D8EDA85EFD0EF9B15E9B25783A50900A3
:1002D000484413869406858B56969D8DEFD0CF9417
:1002E00011ED83270A0099EFB257054791838D8B53
:1002F0006387E7049DCF09476389E7042285EF8080
:10030000DFF8F9B5EFB0AFEB85476309F500834738
:10031000C102414793F70703E398E7FC83552102A5
:100320005A85EF40907C69D183172102E35EF0FA91
:10033000F1B7EFB08FC57D151335150061D10146BA
:1003400081452285EF70FFEF55BFEFB04FE7E5B76E
:10035000EF12BFED9764FF1F9384C4D92685EF8009
:100360009FEB2A8419E16F109FEE1305C400054628
:100370008145EFF0FFD12285EF803FF1C5B7EF1245
:10038000DFEA4111AE842A84930795031307150110
:100390009306F10005466C00268523060100EFD088
:1003A000CFBE1DEDA68541462285EF8030468347AE
:1003B000F1009305140226852308F400EFD06FC8DE
:1003C00005E19767FF1F938727089C4389EF130672
:1003D000940497C50000938565DB2685EFD08FD404
:1003E00041016F10DFE61306940297C50000938564
:1003F00065DA2685EFD00FD379D9DDB7EF125FE14B
:100400009767FF1F938747DB8043AE84B289368AA4
:10041000AA8AEF80AF811316250081452285EF104F
:10042000DFE39767FF1F238B07D89767FF1F93872B
:10043000E7CA03A4070B13F714003E89230FE40057
:10044000CE8525C713059408EFF07FF301C55555F8
:100450006F105FDF8947A30FF4009767FF1F938733
:10046000A7FE9C4303278900858093B71700860762
:100470002300F402231E54019767FF1F23A047C7E0
:1004800085889377B7FF99C0936747001767FF1F69
:10049000232AF7C42285930700061767FF1F230B43
:1004A000F7CAEFF08FD3014565B713050403EFF0EA
:1004B0001FED45D569BFEF125FD7FD572310F5003B
:1004C0002311050023120500231305001306200441
:1004D00081452105EF107FD86F107FD7EF125FD3D2
:1004E0004111AA8401441769FF1F130969CD9309BB
:1004F000A0042EC6EF80CF81B2456344A4006155AD
:100500000DA033053403832709003E95835725004A
:10051000639CB7008357050063989700EFF0BFF91D
:10052000014541016F101FD20504E1B7EF125FCE04
:100530009767FF1F938707B99C434111AA842E84B4
:10054000B28903592500C1C39767FF1F83D7C7BB73
:10055000639B2707EF700F862A8903D52400930534
:100560001002B305B40285472302F10093578900B6
:10057000A302F10093578500A303F10083D7440041
:100580002304A100254613D787002305F10083D754
:100590006400A304E1004E8513D78700A305E100A2
:1005A0002306F1001387950093879501A105B38673
:1005B000B400A6974C00269723032101EFD0EF9CAF
:1005C00041016F103FC8EF60FFFE51BFEF125FC4E3
:1005D0004111AA8401441769FF1F130969BE9309D9
:1005E000A0043AC636C432C22EC0EF707FF28245F4
:1005F0001246A24632476344A400615599A0B3074E
:10060000340303250900AA9703D8070003D5C401C2
:100610006310A80495E91DEE91CA03C6E401930591
:1006200010023306B60225063E9690C2014511CB54
:1006300083C6E40113061002B386C602E506B69728
:100640001CC341016F101FC003D52700E305B5FC93
:10065000050441BF83C5E40113051002B385A5025B
:10066000BE9583C585002300B6007DB7EF125FBA43
:100670005C4141112A8403DA2700C167FD17AE846B
:100680003289630CFA002685EF807F9A8D4763EDEF
:10069000A7007D5541016F10FFBA2E85EF803F996D
:1006A0009D47E3E2A7FEF5B75C40268583D547006A
:1006B000EF809F90835584002685EF80FF8F8D45C6
:1006C0002685EF803F8EAA89EFF04FE09357050112
:1006D0002380F90093578500A380F9002381A900A6
:1006E0005840C167FD178345A7006314FA0093E5DE
:1006F00005082685EF801F8F9767FF1F9387879CCC
:100700009C430840D9CF8347B400858BD9CB780070
:100710003400130671008145EFF05FEB1DC983477C
:10072000B400184093069005F99BA305F400834795
:10073000E701B387D702B306F70083C60604A30315
:10074000D1009386170493879706BA96BA9736C452
:100750003EC61764FF1F130464981C440C40268592
:100760008983858B9D8D834771009E05DD8D93F573
:10077000F50FEF803F871C44104022458983858B0D
:10078000CA861D8EA685EFC0DFCFE31505F01C4499
:100790000C40324689838840858B9D8DEFC0DFC831
:1007A000D5BD8347B40013079005F99BA305F4005A
:1007B0008347E501B387E7023307F50003470704E2
:1007C000A303E10013871704938797062A973E95A2
:1007D0003AC42AC6BDBFEF12BFA3032A4500930740
:1007E000F00FAA840347AA00AE89328436896316C3
:1007F000F700EFB06FAB2305AA00938AC90001464A
:10080000D6852685EFF09FE62A8A21E51767FF1F28
:10081000130787C31843DC4039C383C6A7000547C5
:10082000638FE60283D547005685EF40102C05C93B
:10083000DC40839747006354F00201CC1C4089C719
:100840004A868145014582975C4081C7CA8501453A
:1008500082974E85EF807FA352856F10BF9EDC404C
:1008600003D54700EF60BFD501E9DC4003D5470061
:10087000EF60DFE181471DCD19C41C4089C74A865E
:100880008145014582974E85EF807F9FAA85176538
:10089000FF1F13052586EF80DF9511C45C4081C7DB
:1008A000CA85014582971765FF1F1305E583EF6031
:1008B000F0368547D84085460346A700E30BD6F8B7
:1008C000031747006353E000C9F74A86A2854E85A7
:1008D000EF703F97BDBFEF12BF93AA840144176921
:1008E000FF1F1309E98D9309A004130A9508EF70FF
:1008F0003FC26344A400014535A033053403832778
:1009000009003E958357250099E30504CDB70357A9
:10091000050083D7C401E31AF7FE52868545EFF040
:10092000FFC065D56F101F92EF129F8EAA840144FD
:100930001769FF1F1309C9889309A004EF705FBDF1
:100940006344A4006F101F9033053403832709000C
:100950003E958357250081CF835705006399970003
:1009600093059502130610022105EF80206A050405
:10097000F1B7EF129F8B0347E5012A848347F50106
:100980006307B70089E781452E856F105F8C230FC1
:10099000B400054781C9E398E7FE8947A30FF40037
:1009A0008545DDB7638BE7020947E39FE7FC2285B6
:1009B000EFF02FA59757FF1F9387C7709C4399E7C8
:1009C0009757FF1F9387C7599C4389C70355C40195
:1009D000EFF09FF5A30F0400E1B755D6C9BFEF12A2
:1009E0003F83EFA0FFEE85476312F508EF80EFCC61
:1009F0001764FF1F130444A51C4081CBEFA03FFCEC
:100A000089476304F5001C4082979757FF1F93871F
:100A1000676B9C43B9CF82979757FF1F93874754C3
:100A20009C4391C382971754FF1F1304246B8327A1
:100A3000040B83D4C701EF60FFB78327040BAA859B
:100A4000144003C6E7011C448983858B99C3136650
:100A5000260026854169EF40C03D8144D9497D1972
:100A6000EF705FB063CAA4006F10CFFDEF800FCAB4
:100A700041B7EF705F884DB7B38734030327840A0B
:100A8000BA9703D527006308250103C6470183D51C
:100A90000700EF40A03B8504E1B7EF126FF7014478
:100AA0009754FF1F938484631309400EFD59EF7020
:100AB000FF98634FA40401449754FF1F938404627A
:100AC00013098002FD59EF707F98634CA404014420
:100AD0009754FF1F938484605949FD59EF709FA874
:100AE000634AA40497F5FFFF9385450A1755FF1F36
:100AF00013058566EF60D00797050000938585850F
:100B00001755FF1F1305455EEF6050056F108FF3FB
:100B10003307240383A7040B0504BA97239E3701E8
:100B200079B73307240383A7C40A0504BA9723902F
:100B3000370151BF3307240383A7840A0504BA97FA
:100B40002391370161BFD441038735008547335670
:100B5000F5026377E600A54899E7238006008280C6
:100B6000B387E702EDB73358F502038735003375D5
:100B7000F502B3D7E7021307000363DA080103C6DF
:100B8000050013077003118A19E213077005850623
:100B90004297A38FE6FEC9B718451C416376F7005C
:100BA0005C41BA972380B7001C4585071CC582802D
:100BB000EF12AFE74111AA872E85B285368636C679
:100BC000829763480500B246158D3335A000330582
:100BD000A04041016F10AFE7EF128FE305694111AB
:100BE0002A8A2320060001448149975AFF1F938ACD
:100BF000AA5F056B7D1932C62EC4EF703F85AA84AB
:100C0000EF70DF832695A24532466346A4004E85E9
:100C100041016F102FE303A70A0093171400BA973E
:100C200003D707003377670101E71CC20504E1B76A
:100C300003D707009356D700858AE39946FF337799
:100C40002701E315B7FEBE89D5B7EF120FDE0111FC
:100C50002EC6B2843689EFB02FEE2A84615501C8C2
:100C6000B24589E9232E04002320040201450561D1
:100C70006F10EFDDA1463008CA852685EFF05FF3DF
:100C80007DF5835781010357A101231EF40083578B
:100C9000C1012310E4022311F4028357E101D207BA
:100CA000D1832312F4028357E1011397370163566E
:100CB0000700FD57231FF4005DBF231F040045BF3D
:100CC000EF120FD51754FF1F130444418327040B61
:100CD00003D7C701C167FD17630EF7109757FF1FB2
:100CE0009387C7769C4381C70545EF406077C1690C
:100CF0000149930A400EFD19175BFF1F130BCB74BC
:100D0000EF70CFF3634BA90E1757FF1F03478744BC
:100D10009307F00563E4E702EF704FED93050006DB
:100D2000B3C5A502B7F73600938707E81755FF1F2D
:100D300013058542B385F502EF60A06F8145170565
:100D4000000013058520EF60DFF8EFB0EFDE01CD86
:100D50000357C50109CB0357E50111C783470502B6
:100D600099C3EF60A06BEFB06FDE31C51757FF1F5F
:100D70000347074B9757FF1F9387874A0DCF03C73A
:100D800017002304E50003C72700A304E50003C7F9
:100D900037002305E50003C74700A305E50003C7A7
:100DA00057002306E50003C7670083C77700A30643
:100DB000E5002307F5001C4493E717001757FF1FB2
:100DC0002322F7325C4085E7EF708FEF0DC1EF70A3
:100DD0002FEF44402A89EF70AFEE33F5A4025C4058
:100DE000FD17CA97898F1757FF1F232BF72E014531
:100DF000EF70DF9F01456F10EFC4B30459038327E1
:100E0000040BBE9483D7C40163883703138A040399
:100E1000D2855285EFF0AFD605E183C7F40199CFB3
:100E2000938594082E85EFF08FD509C91306900598
:100E300081455285EF106FC20509D9B583270B0094
:100E4000268593B7170086072380F402EFE0FFB8EA
:100E5000E5B7854763F8A7009307F5FFBE9533050F
:100E6000A040E98D2E8582809841C167BA9713D73B
:100E700007016304A7009CC182804207998FE5BFE8
:100E8000EF12AFBA41112EC63284B684EFB00FCC48
:100E9000E15701C9B24591E99757FF1F23820738EF
:100EA00081473E8541016F108FBA9D461756FF1F3F
:100EB00013061637A6852285EFF09FCFAA8775F116
:100EC00005479756FF1F238DE634E1BFEF124FB45D
:100ED000411191E99757FF1F23A407200144228560
:100EE00041016F102FB6B68532858D467000EFF048
:100EF0003FCC2A846DF58347D1000347E1001759A1
:100F0000FF1F1309A91DA2074207D98F0347C1007C
:100F1000D98F1757FF1F2325F71CEF706FDA61D1A8
:100F2000EF700FDA83244900AA89EF706FD933F587
:100F3000A40283274900FD17CE97898F1757FF1FFB
:100F40002320F71A69BFEF124FAE1C45AA8491CF38
:100F5000D84B01CF83D7470089CBEF601F92AA857A
:100F600009C588446105EF60C04C9757FF1F938700
:100F700067159C43014489EF6F106FAD9C481317B0
:100F80001400BA9703D5070019C1EFE0CFCF0504CD
:100F9000EF70CFC7E344A4FEC5B7EF120FA901114C
:100FA00085E9EF605FDA01449757FF1F23A4071C10
:100FB0009757FF1F23A2071C9757FF1F23A0071C4B
:100FC0009757FF1F23AE071A228505616F102FA8C0
:100FD000B6873285C9467000BE85EFF07FBD2A8492
:100FE00065F541469305E1001755FF1F1305851868
:100FF000EF80C0010355C100EF608FD7F1B78DE1DD
:101000009757FF1F23AC070C9757FF1F9387070DB8
:101010009C470145ED9B1757FF1F2325F70C828046
:10102000EF12AFA04111B685328595463000EFF042
:101030003FB815EDA2471757FF1F2321F70A97570F
:10104000FF1F9387A7099447B24713F7B6FF13F61C
:10105000170019C213E74600858393F7F7079756E1
:10106000FF1F23A1E6081757FF1F2305F70E4101B5
:101070006F10EF9DEF12CF9903841500DC412A8990
:10108000AE8485070387F7FF19C36340800C83870D
:10109000240091C7635580007D14620461849C40E4
:1010A000370700FF0907F98F370700100907639218
:1010B000E70A6355800079146204618483C70400E1
:1010C000858B95E39379F40F4E8A93178A01E18714
:1010D000634AF008A2876353040081473384F940D0
:1010E0007D14620461848385240081C54A85EFF004
:1010F000BFAA9C40370700FF0907F98F3707001088
:101100000907639AE706930500034A85EFF0DFA815
:1011100083C7040093058005918B99E393058007AD
:101120004A85EFF07FA783C70400858B81CB1374BA
:10113000F40F93178401E1876347F004C04005046E
:101140008305F4FFA1E96F10EF8F7D1462046184C1
:101150000DBF370700080907E392E7F6E35080F672
:101160007D1499BF930500024A857D1AEFF0DFA236
:10117000137AFA0F99BF370700080907E395E7FAD2
:101180009305000371BF930500034A85EFF0DFA0CC
:101190007D1471BF4A85EFF03FA055B7EF12EF887D
:1011A000EF70CFAA2A84EF706FA9229589450605B2
:1011B000EFE02FC6E55711C59757FF1F23A6A702DB
:1011C00081473E856F10AF88930700026306F500E4
:1011D0005D1513355500828005458280EF124F83DF
:1011E0004111AA892A89130419008304F4FF32C625
:1011F0002EC42685EFF05FFDA245324659E19307E4
:10120000D0026392F4088304040005481304290003
:101210009377F6FEC9E793070003639FF40E8307F5
:1012200004001307800593F7F7FD6399E70683042D
:10123000140041460904B70600806314080093C6F1
:10124000F6FFB3FEC6028147254F654EFD5F33D3DF
:10125000C602138704FD6368EF06BA8463D5C40829
:10126000630DF5017D55636AF3006394670063C6FF
:101270009E000545B307F602A69705048304F4FF14
:10128000C9BF22898DB79307B0020148E392F4F8F1
:10129000830404002A88130429009DBF01CA8947DA
:1012A000E31BF6F893070003E397F4F883070400C1
:1012B0001307200493F7F7FD639BE70483041400EE
:1012C000094609048DBF13E704021307F7F9636C9D
:1012D000EE009388F4FB1307700363741E01130779
:1012E0007005998CA5BF7D576300E5026304080073
:1012F000B307F04091C519C19309F4FF23A035014C
:101300003E8541016F001FF4B687FDF5D5BF9304FC
:10131000000315F2214605B719FE294629BFEF0241
:101320003FEF011161540DC53284AE8941468145BC
:101330003689EFF0BFEA93140501C180639E09006E
:101340002685EF30102B014401C58145EF20501652
:10135000228505616F001FEF2285CD467000CA858A
:10136000EFF01F852A846DF52685EF30902809E976
:101370000356C1008345E1012685EF20500B01C9CA
:1013800041469305E1001105EF705048D1B75D5417
:10139000C1B7EF02FFE70111E15401CDB284AE897C
:1013A000414681453689EFF07FE32A84639709003F
:1013B0008144268505616F00FFE82685D1467000CF
:1013C000CA85EFF0EFFEAA846DF58357C100EDD317
:1013D000EF700F8E4205931704014181C18363F9B9
:1013E000A702EFB08FB64204E14741803304F40214
:1013F00041460C082A9413054400EF70304183578E
:10140000E1002311F4008357C1002310F40055B705
:10141000E55445B7EF02DFDF7971E15415C5328439
:10142000AE8941468145B684EFF05FDB13190501B3
:1014300013590901639E09004A85EF4010658144F4
:1014400001C58145EFB02FB1268545616F009FDF53
:10145000A6859306300270002285EFF06FF5AA840E
:1014600065F54A85EF4070622A8411E54A85EFB040
:101470004F8C2A8431C58357C1002311240193095D
:1014800064002310F4008347E1009305F100414616
:101490002302F4004E85EF70703713097401414642
:1014A0009305F1014A85EF707036930554004E851F
:1014B000EFC04FBF930564014A85EFC0AFBE69B767
:1014C000DD5459B7EF02DFD4797111E5E154268577
:1014D00045616F003FD7B284AE8941468145368968
:1014E000EFF0DFCF131A0501135A0A015285EFE01E
:1014F0006FCA2A846398090071D98145EFB02FB46F
:101500008144F1B72685930610027000CA85EFF07A
:101510002FEAAA844DFD31C8B2479305D100414658
:10152000858B230FF400B24713050403858393F7DB
:10153000F707A30FF400EF70702D41469305D1011A
:1015400013059408EF70902C59B73304690383A7EF
:101550000A0B3E948357C401638337030509EF6088
:10156000FFEDE344A9FEDD549DB7C1690149975AD7
:10157000FF1F938AAAB6130B400EFD19CDB7231E89
:10158000440159BF49CDEF02BFC84111B289AE84B1
:1015900041468145368AEFF07FC4931A050193DAFC
:1015A0000A010149175BFF1F130B4BB3EF601FE1EB
:1015B000634AA9000145ADCC81441759FF1F1309A7
:1015C000E9B181A883274B0B131439003E9483574C
:1015D0000400638857050509D1BF8327490B13947D
:1015E00034003E948357040085E72310540191464C
:1015F0007000D2854E85EFF0AFDB1DE9B24713973F
:101600008700E1832183858B58C02301F4000DA05E
:101610008504EF60BFDAE3C2A4FC5D5511A86155F3
:101620008280F1F4214681452285EF001FC30145E8
:1016300041016F003FC11971D2C4130AC10686CEA1
:10164000A2CCA6CACAC8CEC6D6C2B6D6BAD8BEDA48
:10165000C2DCC6DE52C463810524FD151C102ACCF1
:101660002ECA02CE3EC89304B0021549A94983058B
:101670000600130416009DE1F2465247E24763FB61
:10168000E620B697238007007245F6406644D644AC
:101690004649B649264A964A096182809307500214
:1016A0006386F5004808EFF02FCFF5A88357C100F7
:1016B00023070100014593F7C70F2316F100814569
:1016C00001480147014681469308D00213030003F5
:1016D000130E300205048307F4FF99C7638C970447
:1016E00063C3F404638BC70501CA0346C100858A3E
:1016F000799AD18E2306D100630908008346C10080
:10170000098BF59A558F2306E10019C12307B10013
:10171000138707FD1377F70FA54663E2E6068146B8
:10172000A545294535A0E38717FBE39F67FA0546E2
:10173000FD564DB70545854571BF05487D5759BFD5
:10174000B386A60205048307F4FFBA96E206E18693
:1017500013F7F70F130607FD1376F60F63E5C500C1
:10176000138707FDF1BF1306F7F91376F60F636EC3
:10177000C902138797FAE30537FDA306D1001307C3
:1017800090066385E704634BF706130780056384BF
:10179000E70A6345F702E38107EE1307500293055A
:1017A0005002E381E7F02286D9B51307F7FB1377E0
:1017B000F70FE364E9FC138797FC75BF1307300646
:1017C0006386E70A13074006E39FE7FC03250A0048
:1017D000A947A307F100930A4A006358050093073D
:1017E000D0023305A0402307F1006C00EFF0AFB545
:1017F0006C004808EFF01F88568A75B7130730074A
:10180000638EE7066341F7021307F006638EE70471
:1018100013070007E399E7F80347C10013672700A0
:101820002306E10009A813075007638BE70213079B
:101830008007E39AE7F6938787FA414793B7170043
:10184000A307E100139727008347C100ED9BD98FC1
:101850002306F100930A4A006C0003250A0079B7B9
:10186000A947A307F100FDB7A147E5BF83050A001B
:101870004808930A4A00EFF02FB2BDBF83270A0041
:101880006C0048083EC8EFF0EFFE1C10930A4A00B7
:101890003EC89DB7BA97FDB30145C5BBEF02FF989F
:1018A0002A88368583464800BA8703475800A2062F
:1018B000D98E328717B600001306069089E517B651
:1018C000000013062690BE85EFF0FFD66F003F980C
:1018D0009757FF1F938747949C4381CFEF02FF9454
:1018E000D843B2862E861847AA853E8502976F0098
:1018F0001F9661558280EF025F938357050039710F
:101900002A84231EF1008347450093056500414664
:101910001305F101230FF100EF70406F930574017F
:1019200041461305F102EF70606E8356240017B62E
:10193000000013066691E5450A85EFF0DFCF6C08DD
:10194000130630020A85EFF0BFF821616F003F9067
:10195000EF02BF8D39712A849305050341461305B3
:10196000D101EF70A06A9305940841461305D10296
:10197000EF70C0698347E4010347F4018356C40153
:10198000858B0607D98F17B600001306A68CE54590
:101990000A85230EF100EFF01FCA6C08130610022F
:1019A0000A85EFF0FFF221616F007F8AEF025F8608
:1019B00037040001B70400FF0111814A1749FF1FD6
:1019C0001309C9717D149389F4FF17BA0000130A33
:1019D000EA8CEF60BF9E63C5AA0005616F009F8619
:1019E0008327490B13973A003E978347370095CFDB
:1019F0005C43A30107005286B3F687008247E545A2
:101A00004800E58FD58F3EC083462700B3F73701E6
:101A1000858AE206D58F835607003EC0EFF0BFC12E
:101A200011468A854800EFF0BFEA850A5DB7EF02EC
:101A3000CFFF01468145EFF0BFE96F005F8183571B
:101A40006500638E071A1D71A2CCA6CACAC886CECD
:101A5000CEC6D2C4D6C2DAC05EDE801013F717003D
:101A60003289AA8431CBF99B2313F500EF601F99CB
:101A700006053D0541990A8BC16A3301A1408A8B55
:101A80008149014AFD1AEF607F97634CAA0C7947A0
:101A9000930604FB17A600001306467FCA85268519
:101AA000EFF0DFDF638F090C13961900DE85130555
:101AB00004FBEFF0FFE15A8183D7640013F727009E
:101AC00021CBF59B2393F400EF605F9406053D0561
:101AD00041998A8A3301A1400A8B8149014AEF600A
:101AE000FF926345AA0A6547930604FB17A6000008
:101AF0001306467ACA852685EFF05FDA6387090AFE
:101B000013961900DA85130504FBEFF07FDC56818C
:101B100083D7640013F7470005CBED9B2393F400B4
:101B20006547930604FB17A600001306E676CA85F0
:101B30002685EFF0BFD69C4481C703D747003DEB15
:101B4000130504FBEFF0BFEE130104FAF640664400
:101B5000D6444649B649264A964A064BF25B256169
:101B60008280DC4413171A00BA9703D70700630872
:101B7000570193971900DE972390E7008509050A1E
:101B800019B7130504FBEFF09FEA35B79C4813170C
:101B90001A00BA9703D7070019C793971900DA9765
:101BA0002390E7008509050A1DBF130504FBEFF02C
:101BB0001FE8B1BF2314E4FA03D767008326C4FAF1
:101BC0002146520751832315E4FA370700F0758F39
:101BD0009447930584FA130504FB92069182558F6E
:101BE0002326E4FA83C7770013F707018347F4FA43
:101BF000BD9BD98FA307F4FAEFF09FCDB1B78280D8
:101C0000EF022FE01744FF1F1304444D0444797181
:101C100093F7F4FB1747FF1F2326F74C93F70404B1
:101C2000A1C78588A1E097A9000093892967EF6083
:101C3000EFF863DBA4028327440B139934003E9929
:101C40008356090091CE4E86E5454808EFF0BF9EC9
:101C50004808EFF0DFDD214681454A85EF00EFDFE0
:101C60008504F1B7EFF09FD41C4413F7F7F79746BC
:101C7000FF1F23A9E64693F707086397071E1C4436
:101C800013F7F7EF9746FF1F23AEE64413F707104D
:101C90006318071E18449377F7DF9746FF1F23A3A7
:101CA000F6449376072095C6058B630A07201840F3
:101CB0008983858B3ACA0347840715464C08060773
:101CC000D98F17A500001305255A230CF100EFF05A
:101CD0003FC01C4413F7F7BF9746FF1F23A4E640FD
:101CE00093F707408DC3835744000D464C08231AD1
:101CF000F1008357640017A5000013052557230B37
:101D0000F100EFF0FFBC1844FD749387F47FF98F66
:101D10009746FF1F23A8F63C9317470163DF070090
:101D2000EFA08FE119C98356C5016391061A17A563
:101D3000000013052554EFF09FCF1C447D777D17DD
:101D40007D8F9746FF1F23AFE63813973701635AFD
:101D50000702858B6388071CEFA04FDF1DC1184564
:101D60008347E5001D463ACA0357C5004C0817A52E
:101D700000001305A550231CE100230DF100EFF036
:101D80003FB51844F977FD17F98F9746FF1F23AB2E
:101D9000F6349317270163D9070081451705000022
:101DA000130525CAEF50FFF21844E177FD17F98FAC
:101DB0009746FF1F23A8F6329317070163D3070244
:101DC000EFA0BF982A84814417A900001309894B0A
:101DD000EF600FEE939704014205C183418163EAEE
:101DE000A71445616F006FC583A70A0093141900FB
:101DF000BE9483D7040033F767011DCF13961701F4
:101E000033F77701B3F637016352060417A60000D3
:101E10001306864309E717A600001306A643E54507
:101E20004808EFF05F814808EFF07FC083D70400D7
:101E3000B3F747012390F4000509EF602FE1AA846E
:101E4000EF60CFDF2695E341A9FA15BD368519C7A6
:101E5000EF40A04361DDEFF01FAAC9BFEFD09FB3F1
:101E600071D5EFF0FFAED9B785697D7A0149974A00
:101E7000FF1F938A6A37056B896BFD197D1A75BF41
:101E8000858B9DC7EF500FF3231AA100414697455C
:101E9000FF1F9385252E13056101EF70201749461A
:101EA0004C0817A500001305A53BEFF07FA2DDB39A
:101EB00017A500001305C53AEFF07FB7E1BB17A5E2
:101EC00000001305653AEFF09FB621B50357E50111
:101ED000C17785073E978357A101FD14133717007B
:101EE0003207E58FD98F231DF100231AD1008356C5
:101EF0000502035725022146231BD100231CE100C4
:101F0000035745028566FD16758FFD76F58FD98FCF
:101F10004C0817A500001305E535231DF100EFF06F
:101F20003F9B21BD17A5000013054535EFF03FB0DD
:101F300089BD5C4813F7E7FF58C8858B89CFA68613
:101F40004A86C9450A85EFF00FEF8357040099E7E9
:101F50000A85EFF0DFAD850461049DBD231AF10011
:101F6000835724009305440041462808231BF100B1
:101F7000EF70C00951464C080A85EFF07F95E1BF2C
:101F8000EF02AFAA85473395A7009747FF1F9387B6
:101F9000E7149C47411181455D8D9747FF1F23A39F
:101FA000A7149377057085E393576500858BA1CBC4
:101FB000C167938707887D8D05EDEF606FD193052D
:101FC000803EB305B5021745FF1F130525222EC617
:101FD000EF50A03BB24519C16349B50085C517450F
:101FE000FF1F1305A520EF50C04441016F002FA62D
:101FF000EF600FCE2A84EF60AFCEE360A4FCEF6009
:102000002FCE75BF0145EFF0BFBFC5B7EF02EFA1FF
:102010007971AA8601441749FF1F1309290C36C696
:10202000EF60CFB9B246635CA4028327490B9314D7
:102030003400BE9483D704006396D70285C617A6E2
:1020400000001306A625E5454808EFF0CFDE480856
:10205000EFF0FF9D214681452685EF000FA04561E9
:102060006F00EF9E050465BF19C22320060081475B
:1020700001C59306D00389E53E8582808505050567
:10208000838705000307050099CF6394E700E39772
:10209000D7FE8147D5B79306D0038547E30ED7FC1B
:1020A00093371700D1BF9307F002E316F7FE854779
:1020B00061D6050508C2C9B799C123A005008147AB
:1020C0000DC11308D0031306F0023307F500830691
:1020D000070081CA638706016397C60099C1050797
:1020E00098C13E8582808507CDB731C9EF026F91D7
:1020F00041112E8A6C002A89368BB28A97A400007F
:102100009384840DEFF05FFB2A8C0144A689B14BC8
:1021100088406286CA85EF70E01701ED0E044E9488
:102120005C403245DA865686D285829741016F003F
:10213000CF900504A104E31D74FD6155C5BF7D5515
:10214000828099E561558280615505616F008F8FAE
:10215000EF020F8C2E8A2A8401118145B2845285A8
:102160004146BA893689EFF06F8793150501C18121
:102170001376F50FA1812285EF507FB12A8469D5AE
:1021800052854C08EFF05FF3524A2A8BE30E0AFAAD
:102190002A8697A500009385650F5285EF70800F02
:1021A000AA8A0DED7D5AEF606FA563C5AA0099E874
:1021B000014561BF5C4413971A00850ABA972390C2
:1021C0004701D5B74C442EC6EF604FA3B245131656
:1021D00015004E850299E34DA0FC85BF5A8697A550
:1021E00000009385250B5285EF70C00A0DE1032A8C
:1021F0000401EF60AFA11316150081455285EF0071
:10220000CF85DDD40C482EC6EF604FA0C1B75A86EB
:1022100097A50000938545085285EF70A00741E11E
:102220001C44A5CF81ECD443370700E0758F944759
:10223000D8C33707001F758F98C701BFA146300864
:10224000CE854A85EFE0DF96E31105F01844835709
:1022500081017D762312F7008357A10193964701F0
:1022600083576700D182F18FD58FF2467D767D1638
:10227000F182858AB206F18FD58F2313F700834749
:10228000E1018356C1012305F7008347B7002314FA
:10229000D700FD8BA305F7004DBD7D557DB55A8652
:1022A00097A500009385C5F25285EF60B07EE31DCF
:1022B00005E81C4CE38A07E89C43E38707E8CE86E1
:1022C0004A86A6852285829749B5EFF21EF63687A3
:1022D000B2862E86AA850545EFF0BFE66FF03EF781
:1022E000EFF2BEF43687B2862E86AA850145EFF05E
:1022F0005FE56FF0DEF5EFF2BEF1411199C123A069
:1023000005009747FF1F938727F0804381441DC82E
:102310002E89AA8931141DC40C4070004E85EFF03F
:10232000BFD419CD81E8A284630C0900B2472320F1
:10233000F90039A08C4008400146EFF0FFD265F566
:10234000404869F8268541016FF0DEEF184111CB56
:10235000EFF2BEEDAE873E85B285368602976FF00E
:102360001EEF35558280EFF25EEC8357C50013D720
:102370000501C205B387E7021841C1814849BA95F2
:10238000BE95EFF0BFFC6FF09EEC584111CBEFF221
:10239000DEE9AE873E85B285368602976FF03EEB6A
:1023A00035558280184509CBEFF23EE8AE873E8571
:1023B000B28502976FF0BEE9355582805C4599C7BA
:1023C000EFF2BEE62E8582976FF07EE8355582806B
:1023D000EFF21EE483290500035AC5002A84484908
:1023E000AE848145EFF09FFD2A890DE193D504016C
:1023F000B38545030356C4004848CE95EFF09FFAD5
:102400002A8909E548488545EFF05FFB4A856FF06A
:102410007EE3EFF2FEDF2A890441035BC5004849F1
:1024200079712E848145B28A368AEFF03FF941E115
:1024300093590401B3896903420441802694A29907
:1024400003440901330480403374440111CC032553
:102450004901A2865686CE85EFF03FF3AA8431E18A
:10246000330A8A40A299A29A8144630C0A025286D6
:10247000D685080803244901EF60503983460901D5
:102480001C089305F00F338646413385470136C655
:10249000EFF0BEDCB2461008CE852285EFF0FFEEED
:1024A000AA84032549018545EFF05FF12685456142
:1024B0006FF05ED9EFF27ED72E864C41A1462A847A
:1024C000EFF03FF5AA8403450401A145EFE07F98B2
:1024D0005C403385A74048C026856FF05ED78147B2
:1024E00097A60000938646CC6393C700828033870B
:1024F000F500034707008507398D135745003697C8
:10250000034707001205398D1375F50F1357450062
:102510003697034707001205398D1375F50FE9B794
:10252000EFF2BED02A84AA851D461305F00FEFF006
:102530001FFB834774003385A7403335A0006FF03D
:102540001ED1EFF29ECE4111A1463000EFF0BFE167
:1025500009ED03578100C167FD1705456317F700B3
:102560002800EFF0FFFB3335A00041016FF03ECEB5
:10257000EFF21ECAAE848C414111A1462A89034460
:102580000501EFF05FDEAA8939E9A1452285EFE078
:102590005F8C9C400357C9002A8AAA97939607012B
:1025A0009CC0C182098F639CE602C16513D70701F5
:1025B000B385B74011E78355E900FD15C205BE9507
:1025C0008CC0A1460A864A85EFF0FFD9AA8901E9A5
:1025D0000A85EFF0FFF401C9832749009CC04E85AE
:1025E00041016FF03EC60357C90083572100804068
:1025F0003307474163DBE70033FA470363170A00F9
:102600004177798C3E9480C0D9BF03450901A1452B
:10261000417AEFE01F84098CAA8A80C0337A440192
:10262000417B63648A0081495DBFA1463000A28579
:102630004A85EFF05FD3AA895DF12800EFF05FEEE5
:1026400011E98357A1000357C100337A6A0180C0A2
:10265000BA973E9A33045441E9B7EFF21EBD2A847B
:10266000AA851D461305F00FEFF07FE7A303A40032
:102670006FF0FEBDEFF2FEB82A84034505015D71DF
:10268000A145EFE00FFD5C402A8B0355E400417942
:10269000B3F727016C003EC6EFE00FFD8355C40081
:1026A000B247A1463008BE95B385654122852EC844
:1026B000EFF07FCBAA84634B05002808EFF05FE6BC
:1026C00011C9B2452285EFF0BFD0AA842685616189
:1026D0006FF0BEB6C2470357A101417C338B6741FF
:1026E000B3F72701BA973EC810100C082285C24BD9
:1026F000EFF01FE8AA8479F90810EFF07FE22DE9E6
:102700005C403ECA30104C0822855249EFF05FE62B
:10271000AA844DFD03578102835701026316F70017
:102720002810EFF0FFDF09C55840D247E31CF7FC43
:1027300063902B058357410285CF83572102B3FA5B
:102740008B010810BE9A1C442311F102EFF0FFF038
:1027500083490401035A4102B309304193F9090244
:10276000631B0A000C102285EFF0DFD4AA8439FD28
:10277000E31C7BF7B9B74E8963733A015289CA8665
:102780001018D6852285EFF01FBEAA8421F16309B7
:1027900009000C44CA8610182285EFF09FC7AA844E
:1027A00003450401CA85EFE0CFEA1C443E9508C406
:1027B000E39E04F0330A2A41CA9A5DB7EFF25EA5A0
:1027C000411191E5FD54268541016FF0BEA7C44932
:1027D00083D725014CC904C12316F50003C70501A1
:1027E0002A842317E50003C5150193160701130773
:1027F00000022308A400C182E366A7FCE1D7B3E48A
:10280000F402E9F08547E3FFD7FAA145EFE06FE472
:10281000AA89014A01498357C400931509012285F9
:10282000BE95B38535412EC2EFF0BFD119ED0355EA
:10283000E4004C00050AEFE02FE39245420A2285AE
:10284000135A0A01EFF0FFCF09E905098357E400A5
:10285000420913590901E360F9FC8357E4006394CA
:102860004701D1548DB7639427039245A1463000A8
:10287000B38535412285EFF01FAF35E12800EFF039
:102880003FCA11C50355E4004C00EFE0EFDD92476D
:10289000C17A3387374158C04177F98F1CC44C4007
:1028A0001C4463EEF500A14630002285EFF0BFAB7B
:1028B0001DE52800EFF0DFC6032A44001DC15C407F
:1028C0000355E4004179B3F727014C003EC2EFE025
:1028D000AFD992452285EFF0DFC6635C0502AA847A
:1028E000DDB512450359A100035BC10033F5AA0011
:1028F0002A9903450401DA85EFE0AFD54A9508C46B
:102900006314450163130B04330A3A412322440143
:1029100079B709C58547A308F40075B54C402285F1
:10292000EFF01FAB4DFD48408357C4008609337557
:10293000A9003E953305354148C03375250108C4CB
:102940002285EFF03FD379D559BF4D5549BF834715
:102950001501C9CFEFF2FE8A2A8403450501411112
:102960002E8AA145BA893689328BEFE08FCE835704
:10297000C4000605898F7D5563E727075C408144C5
:102980003EC230004C002285924AEFF07FBE21ED1E
:10299000835B810063994B012800EFF07FB801E56C
:1029A0008504C204C18058409247630BF702E3FAE2
:1029B00099FC8356C10061559DC663E63403C17519
:1029C000B3FABA006373D900CA868355A1005A8648
:1029D0002285D695EFF03F9919E50355C10021A056
:1029E0006155E3884BFD41016FF03E85495582807A
:1029F000EFF2BE830147EFF09FF56FF05E85EFF2D7
:102A0000DE823284B2862E86835545000841EFF07F
:102A10003FFE635385002A8422856FF05E83EFF2C8
:102A2000CEFD834715013971C954BDC7034B05015C
:102A30002EC62A84A1455A853689328AEFE06FC1B5
:102A40000D473307E5028357C400AA8DFD54998FC3
:102A500063E427056304090063000A045C403ECA7E
:102A600030084C082285524DEFF09FB0AA8945ED01
:102A70008357810132476397E7002808EFF05FAA88
:102A8000630605105840D247E31CF7FC8144631BE2
:102A9000090019A0814499E7268521616FF0AEF9FC
:102AA000E35CA0FE5A85CA85EFE0AFBA014B11C5C1
:102AB000330BB501420B135B0B01014D7D5CC17BF8
:102AC000930C44008357E4006380A70D1C444440EA
:102AD0003307FB0063EBE40432472311F1020810D3
:102AE000FD572310E102231221032303F102EFF02B
:102AF000DFB6630909000C44CA8652862285EFF0CE
:102B00005F91AA8903450401CA85EFE08FB41C4494
:102B10003E9508C4639909000C102285EFF09F9937
:102B2000AA89CA8435D9CE8485BF03450401A1454D
:102B3000EFE02FB2B387A4002311F1028357C40042
:102B4000B3F4740123108103BE94898C44C008102F
:102B500023120102EFF07FB00C102285EFF09F9559
:102B6000AA840355E400E685EFE00FB05C40B3F7BC
:102B700077011CC4E39204F22285EFF0BFAFAA8470
:102B8000E31C05F0050D3DBFC15439B78357C101A2
:102B9000E30209F0E39827F1C177034C0401B3770E
:102BA000FD00035DA101330C8041137C0C023E9DAE
:102BB000D28ACA8CE28B63F38C01E68BDE8610101E
:102BC000EA852285EFF02FFAAA84E31B05EC5E86E6
:102BD0000C105685EF602041AA84E31505ECB38CF8
:102BE0007C415E9DDE9AE3970CFC7DB5EFF2EEE34F
:102BF00081460146EFF0BFE26FF06EE5638C050E93
